:020000040800F2
:10500000804F0020D550000805DA00089FCA00082C
:105010000000000000000000000000000000000090
:1050200000000000000000000000000045EF000844
:105030000000000000000000E9DA0008850F010808
:10504000E7500008E7500008E7500008E750000864
:10505000E75000081D7C0008E7500008277C000886
:1050600000000000E7500008117B0008E75000082E
:10507000E750000851CF0008B1230108E7500008AD
:10508000E7500008E7500008E75000080000000063
:10509000E7500008E7500008E7500008E750000814
:1050A000E7500008E7500008E75000089123010886
:1050B000A1230108E75000080000000000000000E4
:1050C0000348854600F046FD00480047A14001081E
:1050D000804F00200448804704480047FEE7FEE771
:1050E000FEE7FEE7FEE7FEE749100108C1500008B1
:1050F00030B50B46014600202022012409E00D4670
:10510000D5409D4205D31D469540491B25469540F7
:1051100040191546521E002DF1DC30BD70B500243B
:105120002546002801DA01244042002901DA012540
:105130004942FFF7DDFFAC4200D04042002C00D0D6
:10514000494270BDF0B51FB40646002082B0054646
:105150004024019100901BE0019922460F46304601
:1051600000F020F8049A059B801A994110D310464C
:105170001946224600F042FB361A8F41019722461B
:1051800001200021009F00F039FB38184D410090AC
:105190002046641E0028DFDC019B00982946324629
:1051A00007B0F0BD10B5202A04DB0846203AD040F5
:1051B000002110BD0B46D340D0402024A21A9140BC
:1051C0000843194610BD03460B439B0703D009E073
:1051D00008C9121F08C0042AFAD203E00B78037032
:1051E000401C491C521EF9D27047D2B201E0027035
:1051F000401C491EFBD270470022F6E710B513464B
:105200000A4604461946FFF7F0FF204610BD421E2D
:105210005378521C002BFBD10B781370491C521C85
:10522000002BF9D1704730B505462A460B46107859
:105230001C78521C5B1C002801D0A042F7D0002C27
:1052400003D0002802D06D1CEFE7284630BDCAB25B
:10525000401E4178401C8A4202D00029F9D100202A
:105260007047421C0178401C0029FBD1801A70470E
:1052700010B5002200E0521C835C8C5CA34201D17B
:10528000002BF8D1D8B2E1B2401A10BD30B50446B7
:105290000020034600E05B1C934203D2E05CCD5C3F
:1052A000401BF8D030BD03460A780270401C491CF0
:1052B000002AF9D11846704730B50546002003464C
:1052C00000E05B1C934205D2EC5CC85C201A01D163
:1052D000002CF6D130BD70B506460DF0C1FC046857
:1052E00005460A220021304600F0FEFA2C6070BD0F
:1052F00070B502464A40D50F40004A00ED0740080D
:105300005208002814D0002A12D0C40DD30D410237
:105310000120C0055202490A520AE41A091812185B
:105320007D34914201D3641C00E04900002C01DA75
:10533000002070BD0023914201D3891A0343400825
:1053400049000028F7D100290AD0914202D1012159
:10535000C90705E0914201D2012101E00121C943C1
:10536000E005C018401900F0F7FA70BDF0B5074627
:105370000846584087B0C00F049048000E465900B8
:1053800040084908BC1A884105D2384631461E46B5
:1053900017460B4602465800400810434CD0300DCB
:1053A000039040055900400D490D0590401A0290A8
:1053B000402872DA18030121000B09050843019007
:1053C00004980092002805D001995242002088419B
:1053D00000920190029840210A1A0199009800F069
:1053E0000DFA05460C466B4607CB00F017FAC019BC
:1053F0007141039A0E0D0023D71756401A467A4082
:10540000164344D0049A002A2DD0029A012A039A06
:1054100015DC1205C01A914101263605001C7141A8
:10542000D20F059ED2070093019202962A46234688
:1054300000F0E0FA07B0F0BD38463146FAE716054D
:10544000224A0F46B218C01AB74101210905001CB3
:105450004F4100187F41114618187941E20F10435F
:105460006D19644113E0E2076D0815436408C20733
:105470001443039A01261205C01A91413605001CF7
:105480007141CE07400830434908C01851412A46AF
:10549000234600F0A2FACDE7FFE70498012240007E
:1054A000C117121A00238B4104983146C417381AC9
:1054B000A141EEE730B40124E407634030BC55E776
:1054C00030B40124E407614030BC4FE70000E0FF46
:1054D000F0B51FB488B00B99099800244840099989
:1054E000C00F490049080991C0070B990090490075
:1054F00049080B9109990898A64608431CD00B99B6
:105500000A98084318D0099801244000420D480029
:10551000410D099824050003000B204309900B98C6
:105520000003000B20430B9050181C494018002228
:1055300001901446104605E0002001460DB0F0BD74
:10554000032801DA034600E003239C46C11A0AAE91
:105550000AE05F0008ADED5B4F00F75B7D4300277D
:10556000AA187C41491C5B1E6145F2DD410004AB79
:105570005A522104120C0A43240C401C0828DFDB79
:10558000019802900099704601910090059B049A41
:105590000799069800F02EFAD0E700000DFCFFFFF7
:1055A000F0B50C465C4085B0E40FE40703944C0072
:1055B0000026640859009446490802460296224390
:1055C00021D062460A431ED06200570D4A000E03E6
:1055D0002303550D012402462C492405781B1B0B7F
:1055E000360B401823432643614600901C46501A50
:1055F000B44103D30098401C009002E09218009838
:105600005B41002803DA0020014605B0F0BD002010
:10561000012109050746864611E064461D46141B14
:10562000B54106D36546521BB341744607430C434C
:10563000A646CD0740084908284392185B41054615
:105640000D43EAD11046184313D060461946504026
:105650007140084306D06046101AB34106D20122B9
:10566000002306E000220123DB0702E00122D243EF
:105670005310009874460105381C6141029C039D3B
:105680000019694100F0A9F9BFE70000FD0300001F
:1056900070B54B005B0803430BD04B005C0D00263C
:1056A00033466542B341D417AD1AA34102DB002053
:1056B000014670BD12053018514170BD10B5002271
:1056C0009623114600F050F910BD00000EB5C21728
:1056D000C10F5040CA0740180021054B02930192A8
:1056E00000910A460B4600F085F903B000BD0000AA
:1056F000330400000EB505490291002100910A46CD
:105700000B46019100F076F903B000BD33040000B0
:10571000410040020122400AD205090E80187F296B
:1057200001DA00207047962903DC9622511AC840FE
:1057300070479639884070474A0009030123090BD6
:105740001B051943094B10B5520D9A4201DA00208E
:1057500010BD064B34339A4203DC9A1AFFF722FD40
:1057600010BD03495118884010BD0000FF03000020
:10577000CDFBFFFFC20FD207400040080BD0C10D88
:105780000723DB01C91840020905400A1143C2087A
:1057900040071143704700200146704710B50029AB
:1057A00004DB0124E40740428C412146002B04DB4A
:1057B0001C460123DB075242A341994200D190428B
:1057C00010BD0000CB0FDB07490010B549080246A9
:1057D0000A4307D00A0D07240903E401090B121B31
:1057E000002A01DC002010BDC900440F0C43C10099
:1057F000E018D205801800F0AFF810BD10B5202ACF
:1058000004DB0146203A9140002010BD9140202346
:105810009C1A0346E3401943904010BD10B5202A5E
:1058200006DBCB170846203A1041C1170B4306E0B0
:105830000B461341D0402024A21A91400843194638
:1058400010BD00000FB400B589B00CA900910B99F0
:105850000023CB60204B214A069307920422019239
:105860001F4A02921F4A089202466B46002000F02F
:1058700020FA09B008BC04B0184770B586B00646D7
:105880000020C0430190002015460C460091029173
:1058900004903246694604A8FFF7D4FF02460498F4
:1058A0002118002D05D0002801D0084600E0204630
:1058B0002860049800280DD0002A02DD0098884254
:1058C00008D0081B0190009432466946029404A84F
:1058D000FFF7B8FF06B070BD095F0008295F000838
:1058E000FFFFFF7F815B0008F7B5009C0F46002695
:1058F0002578641C002D05D000F03EF90068405D5D
:10590000C007F5D12B2D02D02D2D18D0641E39469D
:105910002046029A00F01AFB002F04D03968A142F9
:1059200001D1009939607105022400290BDA404247
:10593000002803DD0DF094F90460A007FEBD0120EE
:1059400080020643E3E70028F8DA0DF089F90460E5
:105950000048FEBDFFFFFF7F002904DA401C49001C
:1059600001D140084000704770B40024050C05D1F7
:105970001024000402D1002921D01124050E01D1E8
:1059800000020834050F01D10001241D850F01D14B
:105990008000A41C002801DB4000641C002908D002
:1059A00020252E1B0D46F540A14000D001212943A2
:1059B000084301061B1B000ADB1D02D5002070BC3A
:1059C0007047DB05181880180029F8DA401C4900D8
:1059D000F5D170BC40084000704710B5002B08DAC4
:1059E0000024401C614192185B411A4301D14008D8
:1059F000400010BDF0B51FB482B005460C0003D0C6
:105A000008460DF0CFF802E00DF0CCF82030024649
:105A1000009021462846FFF7F1FE049B059A0446B4
:105A20000F4618431143084314D0184610431BD0A7
:105A3000009840210A1A18460599FFF7B3FB05465E
:105A40000E46009A05990498FFF7D8FE084305D042
:105A5000012004E02046394607B0F0BD0020C11700
:105A600005430E432C43374300990E986305401AB3
:105A70007905E40A00220C43FD0A0A3002D5002011
:105A80000146E9E70105101969410C9C0D9D0019BB
:105A90006941FFF7A2FFDFE7F8B505464800400877
:105AA0000C46284304D06000184A400D904201DDA6
:105AB0002846F8BD15493539884210DC88420BDB91
:105AC000290D200308432903014305D0E00F1049A5
:105AD000C00741180020F8BD00200146F8BD161A85
:105AE0004020821B28462146FFF788FE074600918A
:105AF000284621463246FFF755FB3A46009BFFF702
:105B00006CFF3246FFF77AFEF8BD00003304000058
:105B10000000F03F4A0009030123090B1B0519434C
:105B20000A4B10B5520D9A4202DA0020014610BD10
:105B3000064B34339A4203DC9A1AFFF733FB10BD4D
:105B4000034BD218FFF75AFE10BD0000FF03000000
:105B5000CDFBFFFF064C0125064E05E0E36807CCB0
:105B60002B430C3C98471034B442F7D3FFF7ACFA00
:105B7000C0570108E057010800487047304C010841
:105B800010B50446FFF7F8FF0068005DC007C00FBE
:105B900010BD0000FFB5087889B01546FF2805D074
:105BA000491C2D2804D00022002407E000240BE02B
:105BB0000122F9E70A235C430419491C0878FF28ED
:105BC000F8D1002A00D06442002004902A780146CF
:105BD0002D2A01D02B2A0FD16D1C2D2A02D0002294
:105BE000049209E00122FBE700260A2233466D1CDD
:105BF00000F0FFF9381871412F78FF2FF4D10C9A7B
:105C0000A218069202460A4304D0FF23069A913353
:105C1000DA4205DA002109980A4606C00DB0F0BD47
:105C20000024B74AB54D2646079200F02FFA02909D
:105C300006980391002801DA474200E0074639053B
:105C40000020AF4A001C51410191009012E0F8077A
:105C500007D022462B4630460799FFF739FC064607
:105C6000079122462B4610461946FFF731FC0446A1
:105C70000D467F10002FEAD10698019B0028009A5C
:105C80000399029806DAFFF78BFC3246079BFFF771
:105C900087FC05E0FFF71CFC3246079BFFF718FC6A
:105CA000049A002A02D00122D2075140099A03C265
:105CB000B4E7FFB591B0002009900025ED432E20F8
:105CC0009E685C681F460190B9696D1C12988847F0
:105CD0000090396A88470028F6D10098401C0AD005
:105CE0000D20C0018443002E12DD00982B2809D01E
:105CF0002D280DD103E00020C04315B0F0BD0120D8
:105D000080020443B9696D1C12988847761E009082
:105D100003A9600501D52D2000E02B206A461073F1
:105D2000491C0CA80F9102900AE0B9696D1C1298E9
:105D3000884700900120400204431398761E0560B6
:105D4000002E02DD00983028EFD00199009888429B
:105D500046D18020044308E00998401E09900120A4
:105D6000400204431399681C0860B9696D1C761ED3
:105D70001298884700903028EED031E0019988428F
:105D800005D1200603D480200443761E1EE000982F
:105D90000DF008F9002826D001204002044307A98D
:105DA0000F980331761E88420BD200980F99303835
:105DB00008700F98401C0F90200607D50998401EC8
:105DC00003E0200602D40998401C0990A00502D5E2
:105DD0001399681C0860B9696D1C12988847009077
:105DE000002ECBDC59E0002E57DD0098652801D04D
:105DF000452852D1A00550D5032000028443B9693B
:105E00006D1C761E129888470090002E0CDD2B2802
:105E100004D02D2808D1FF2001300443B9696D1C3E
:105E200012988847761E0090E00501D52D2100E0EC
:105E30002B21029801700298401C0290019025E0ED
:105E40000120400204430EA902980131761E8842C7
:105E50000ED20098029930380006000E087003D167
:105E60000299019881420AD90298401C029006E0EA
:105E7000E00501D5234801E0224840420990B96974
:105E80006D1C12988847009013980560002E04DD61
:105E900000980DF087F80028D2D1F9691298884748
:105EA0000F99FF200870029903AA087000200A9039
:105EB0000B900CA90AA8099BFFF76CFEA00502D461
:105EC0000120C04319E72420044209D0E00713D180
:105ED00038680B9A0A99031D3B60006806C00BE006
:105EE0000B990A98FFF76EFC0146E00704D1386869
:105EF000021D3A60006801602846FEE6000014407A
:105F00000000F03FF1D8FFFF4268002A08D0016886
:105F10000B78491C002B03D0521E06C01846704750
:105F20000121C160881E70474268002A0BD0C368F7
:105F30000168002B07D183688B4204D0491E521C94
:105F400006C0002070470020C0437047F7B582B0FC
:105F5000029C00272078641C15460197302802D047
:105F6000002D15D015E020780127641C782804D076
:105F7000582802D0002D09D00BE0002D01D0102DA3
:105F800007D1002710252078641C02E0082500E0D6
:105F90000A250026009610E0009901276943081899
:105FA000020C294680B2714300908E183804864254
:105FB00001D3012001902078641C294600F056F896
:105FC0000028E9DA0398002805D0002F01D0641ECC
:105FD00000E0029C04600198002806D00CF040FE0E
:105FE00002210160C81E05B0F0BD009930040843CD
:105FF000F9E7F0B51FB486B0002000900190029040
:106000000698069980B204900798090C02040014BF
:10601000114307900027089D099806913E463C468B
:1060200003900398A9B20204000C039004982D0C6D
:106030001543484300212246FFF7E0FBC719714191
:1060400010340E46402CECDB3846029AFFF7D6FBA4
:10605000009A019B801800905941029801911030DC
:1060600002904028CCDB00980BB0F0BD3A2800D25B
:106070003038202302469A43412A01D3104637384C
:10608000884201D30020C043704700000EB5054A86
:1060900002920022009213460192FFF7ABFC03B07C
:1060A00000BD00003304000070B58C180578401C5A
:1060B0006B075B0F01D10378401C2A1106D10278CF
:1060C000401C03E006780E70401C491C5B1EF9D191
:1060D0002B0705D40023521E0DD40B70491CFAE780
:1060E0000378401CCB1A921C03E01D780D70491CEC
:1060F0005B1C521EF9D5A142D8D3002070BD000010
:1061000038B50446064805490068FEF7F1FF6043CC
:1061100000E0401E00900028FBD138BD40420F0037
:106120009C000020F8B50446006881688907890F43
:10613000012902D10168C90727D18168144A1026B4
:1061400011400125002913D1816829438160012074
:10615000FFF7D6FF02F0F0FF074611E002F0ECFF78
:10616000C01B0A280CD920680068C043C00707D0AC
:10617000606D30436065A06D2843A0650120F8BDC7
:1061800020680068C043C007E8D10020F8BD0000C7
:1061900017000080F7B58EB00D4630224A4901A89D
:1061A000FFF711F80E98494C8068372D416B09684C
:1061B0000D91E7691DD019DC444A0C23D2690021F6
:1061C0005A4301ABD618042D2BD008DC002D18D073
:1061D000012D20D0022D24D0032D38D121E00E2D09
:1061E00057D00F2D64D0362D31D102E0383D072D28
:1061F0002DD81098002F4FD0012F51D0022F5CD1F5
:1062000052E0E1612162019A029904F017FE206ACE
:10621000401C206251E004F035FE0D9806F05EF857
:106220004BE02A4AD7697F1C042D0DD0B268022D9D
:1062300010D002252A4217D0E7612162042F0BD328
:1062400021490022503917E0327A5207F4D4012054
:1062500011B0F0BD0125EDE70C214F43F918DA59D3
:10626000496804F0EBFD28E0206A401C2062032806
:1062700006D315490022A0390E9805F03DF91CE01F
:106280000E200090124A00210E9B0D9805F01AF97D
:1062900013E09A587168E4E703C807F071FB0CE05B
:1062A00003C807F083FB08E003C807F05DFB04E0C8
:1062B000002007F00BFB012801D00020C8E70249AD
:1062C0000022B0390348D8E710480108B800002080
:1062D0001027000010100020FEB5074680680A460F
:1062E000416B384C0968019100250E26A378032ADA
:1062F00061D007DC3449002A0CD0012A12D0022ACE
:1063000006D115E0042A28D00E2A40D00F2A4DD0FD
:106310000120FEBD032061610CF038F9A570E56035
:1063200025612BE004F0AEFD019805F0D7FF42E0B7
:10633000012B0DD02561E168491CE1601ED0E121EF
:10634000626909038A4229D10121A1701FA221E0BB
:10635000032061610CF01AF910E02069E560401C2F
:106360002061052807D00A2808D91D49002238468F
:1063700005F0C2F81FE0E1210903E9E77D223B4671
:10638000D20000210096019805F09CF813E0012B43
:1063900004D014A2154904F051FD0CE003210020A3
:1063A00007F0A4FA0E4900222031E0E7002007F0B0
:1063B0008DFA012801D00020FEBD094900221039C4
:1063C0000B48D5E7B800002000C2010041542B491A
:1063D00050523D3131353230303B26570D0A0000E6
:1063E00070470108415445300D0A00008813000031
:1063F0001010002038B504468068164B022915D0CD
:1064000004DC002908D0012904D10CE003290DD0B7
:106410000A2911D0012038BD516819600EA2114916
:1064200004F00CFD14E004F02DFD11E000222046E4
:10643000196805F061F80BE00020009003CA6B4674
:1064400009A206F019F9022802D1009807F0CCFA47
:10645000002038BD4401002041542B4353510D0A04
:1064600000000000881300002B4353513A2025649C
:106470002C252A0D0A0000001CB500230093C26BD6
:1064800052680192C06B42685168044A936051603F
:106490006A46024905F030F800201CBD4801002082
:1064A00010B5044607F098FA012802D00020C04336
:1064B00010BD2046FFF7E0FF002010BD10B50446D8
:1064C0008068002907D001290AD002290BD00329AE
:1064D00009D0012010BD09A20B4904F0AFFC0BE06C
:1064E00004F0D0FC08E00221084607F0FFF9002282
:1064F0000649204605F000F8002010BD41542B430A
:1065000046554E3D300D0A0088130000B047010883
:1065100000B5E1B0FF21813168460CF02DFB6846E3
:1065200004F09CFE002061B000BD000010B594B0E6
:1065300000216846417202210172234803904802FB
:10654000049022480590642006900820079002A934
:1065500003200BF0A1FF0024E443002820D11C48B5
:1065600005F0D0FE00281BD11A4809901A480A905D
:1065700039200B9019480C9019480D9019480E902D
:106580001248802164300F90803011901048109193
:106590001291139009A9144804F0A0FC002802D01D
:1065A000204614B010BD01210F48019100900F4BFF
:1065B0000FA21149074804F045FF1049054804F0AF
:1065C00079FF0020EDE70000140A0020140E0020DF
:1065D000B00000201010002078440108CD7300089E
:1065E0009175000835740008780F002040460108B6
:1065F00041495237383045004047010811650008CD
:1066000010B505490869002803D0898A012202F0E3
:106610008CFD002010BD0000F80F002010B50549CA
:106620000869002803D0898A002202F07EFD00203C
:1066300010BD0000F80F0020C3000348C150181817
:106640008280002070470000F80F002010B5054937
:106650000868002803D08988002202F066FD002027
:1066600010BD0000F80F002010B50549086800288B
:1066700003D08988012202F058FD002010BD0000DF
:10668000F80F002010B503468068154C002907D08C
:1066900001290CD002290DD0092918D0012010BDE4
:1066A0000021A1630FA2124904F0C8FB15E004F019
:1066B000E9FB12E0A06B012805D00E490022184624
:1066C00004F01AFF09E00B4900223031F7E7044BD0
:1066D00003CA383308A205F0CFFF002010BD000028
:1066E000B800002041542B43474154543F0D0A0049
:1066F00088130000C04701082B43474154543A20F7
:1067000025640000F0B599B00C460646202110A87B
:10671000FEF772FDB5683C22686B5649076801A810
:10672000FEF751FD07F0A4F8052253A10090FEF7F3
:10673000C3FD00281CD0052251A10098FEF7BCFD26
:10674000002815D0052250A10098FEF7B5FD0028BD
:1067500010D005224EA10098FEF7AEFD002807D00C
:1067600005224DA10098FEF7A7FD002804D008E0FF
:106770004BA202E04CA200E04DA2202110A806F09E
:106780006EF800224C4801A9032C3DD006DC002CF9
:106790000BD0012C15D0022C69D119E0042C17D094
:1067A0000E2C5ED00F2C62D158E002634263044687
:1067B0002846019A029904F041FB606B401C60631B
:1067C0004CE0284604F05EFB384605F087FD45E0C6
:1067D000042C04D0022C0FD0032C15D02BE0036B1B
:1067E0000C245C436418247A640740D5426314E0A7
:1067F00020490022603925E0036B0C2463435B18B9
:106800001B7ADB0707D116E0036B0C2463435B188C
:106810001B7A9B070FD54263036B5B1C0363052B3D
:10682000E6D20C204343CA585818416810AB28469A
:1068300004F004FB12E0416B491C4163032905D3BA
:106840001E490022304604F057FE07E00E2000905B
:1068500033461B4A0021384604F034FE002019B0AC
:10686000F0BD006B0C2250430A584018DDE70120B0
:10687000F5E70000404801083436303030000000B1
:106880003436303032000000343630303100000011
:1068900034363030360000003436303033000000FB
:1068A000434D4E4554000000554E494E455400009E
:1068B00043544E4554000000B800002040470108F2
:1068C0001027000010B58268002912D0012910D0CD
:1068D0000F2901D0012010BD07490B78012B03D0EF
:1068E000104600F0F5FD04E000220A70034904F0B0
:1068F00003FE002010BD0000B8000020C0470108C2
:1069000008B50F2925D006DC002922D0012908D09E
:10691000042904D108E01A290BD0272916D0012018
:1069200008BD0AF02BF814E000220B4904F0E4FD46
:106930000FE00020009003CA6B4608A205F09CFE01
:10694000012806D100980AF0F9F802E0094901206F
:106950000870002008BD0000504701082B51495520
:1069600052433A2022636C6F736564222C25640DB8
:106970000A000000B800002010B58068002907D088
:10698000012905D00F2901D0012010BD00F082FDA2
:10699000002010BD10B5002909D0012907D0042915
:1069A00001D0012010BD0022024904F0A5FD002005
:1069B00010BD00005047010810B504468068324BF6
:1069C0009AB0022916D004DC002909D0012904D18B
:1069D0000DE003290ED00B2912D001201AB010BDF2
:1069E0005168196029A22E4904F028FA4AE004F0FF
:1069F00049FA47E000222046196804F07DFD41E095
:106A0000002014461890169013901490159007903B
:106A1000129003CC18AB23A2083C05F02DFE0128F0
:106A200030D1189800282DD112AB069307AA15A9CA
:106A300014A803AB07C310AA13A816A900920191CA
:106A4000029003CC0EAB1BA205F016FE092819D14B
:106A500010980CF05BFE099108900E980CF056FE11
:106A60000B910A9068461699018608A813998174BB
:106A70001499C17415990175079941751299817519
:106A800006F010FF0020A9E78401002041542B43A9
:106A9000495047534D4C4F433D312C310D0A0000B6
:106AA000881300002B43495047534D4C4F433A2025
:106AB000256400002B43495047534D4C4F433A2027
:106AC000252A2C25702C25702C25642F25642F2534
:106AD000642C25643A25643A25640D0A0000000000
:106AE0001CB500230093C26B52680192C06B4268D0
:106AF0005168044A936051606A46024904F0FCFC04
:106B000000201CBD8801002010B5044606F0C2FE1E
:106B1000012802D00020C04310BD2046FFF7E0FF4F
:106B2000002010BD10B504468068002907D0012957
:106B30000AD002290BD0032909D0012010BD09A2D7
:106B40000B4904F07BF90BE004F09CF908E0032109
:106B5000022006F0CBFE00220649204604F0CCFCC1
:106B6000002010BD41542B4346554E3D310D0A00C7
:106B700088130000C047010810B50446002905D05D
:106B800001291DD00F2908D0012010BDFFF75EFD9F
:106B90000221002006F0AAFE12E0002006F096FE78
:106BA000012803D10221002006F0A0FE002006F0FB
:106BB00095FE012804D100220249204604F09CFCE5
:106BC000002010BD70470108F7B582B002980E266C
:106BD0008468274D606B00290068019008D0012966
:106BE00015D00E2916D032293FD0012005B0F0BDB6
:106BF0000027E7622169204688470028FAD0E7622B
:106C00006F70FFF723FD00961A4A029B23E005F000
:106C100065FB2AE068787D24E400002806D001287E
:106C200009D002280FD003281FD119E00120687075
:106C3000FFF71AFD03E002206870FFF7E1FC009601
:106C40002246029B07E003206870FFF7E7FC192249
:106C5000029B009652010021019804F033FC04E0ED
:106C600000220549029804F047FC0020BEE700001E
:106C7000B8000020B80B00008047010800B585B0BF
:106C8000002923D0012921D0042904D0352907D097
:106C9000012005B000BD00220D4904F02DFC15E0D7
:106CA000002002900390049003A904A80191009091
:106CB00003CA02AB07A205F0DFFC032806D102AB32
:106CC00007CB0AF00DF8029809F0ACFF0020E0E7CE
:106CD000504701082B524543454956452C25642C05
:106CE00025643A0D0A256500002903D0012901D049
:106CF000012070470020704770B5054684680B007E
:106D00000BF07FFF05040D1111111C0006F0BEFDF4
:106D100003460BA20C49204604F090F80CE02046F4
:106D200004F0B0F808E0104606F01CFE0748002208
:106D30004168284604F0E0FB002070BD012070BDD2
:106D400025730D0A0000000088130000F4000020E5
:106D5000FEB586680346706B3F4F006801900125C1
:106D600000203C7907294DD006DC00290CD00129F0
:106D70000DD0022906D111E008294AD00E2951D0A0
:106D80000F2960D00120FEBD3871B8624FE0304657
:106D900004F078F8019805F0A1FA5AE02E4A916AB9
:106DA000526A491C002C02D0012C0ED051E078719F
:106DB000012A07D0052A05D0B962642919D9002211
:106DC000264912E03D71B86235E07871012A04D09D
:106DD000052A02D0B962F8620BE0F86A401CF8623A
:106DE000032806D31D4900228031184604F084FB95
:106DF0002FE00E207D22009012010021019804F066
:106E000061FB26E0002C24D1134B03CA243314A2C7
:106E100005E0012C1DD1104B03CA243314A205F048
:106E20002BFC16E0002C02D0012C04D011E078627B
:106E30007D7113A202E078627D7114A2164930467A
:106E400003F0FCFF05E07879002802D1304600F01D
:106E500021FB0020FEBD0000B800002050470108C3
:106E60002B435245473A20252A2C25640000000078
:106E70002B43475245473A20252A2C256400000021
:106E800041542B435245473F0D0A000041542B43C8
:106E9000475245473F0D0A00881300007FB505465D
:106EA0008068214C37292BD00CDC02291FD004DC50
:106EB000002912D001290DD116E0032917D0362957
:106EC00008D11DE038291BD0392919D03A2917D00B
:106ED0003B2915D0012004B070BD1346A26013A257
:106EE000174903F0ABFF1DE003F0CCFF1AE0A068E8
:106EF00009F024FE00221349284604F0FDFA11E0AF
:106F00000020039001A8009003CA03AB0EA205F075
:106F1000B3FB022806D10FA1029A0198FEF7CCF923
:106F20000028E4D00020D6E72C01002041542B4358
:106F30004950434C4F53453D25640D0A0000000065
:106F400030750000F047010825642C2025700D0ADB
:106F500000000000434C4F5345204F4B0000000001
:106F6000F7B584B0049800268568474C686B3629CD
:106F70000068039010D00CDC02297ED004DC0029CC
:106F800015D001297DD134E0032939D00E2978D1DB
:106F90006EE03739042974D801A80396009003CA1B
:106FA00003AB3AA205F068FB022866D134E0104634
:106FB000226009F08BFD0746206809F077FD064640
:106FC000206809F0ADFD012811D033A06946C1C188
:106FD00032A23A492846236803F030FF0E20009081
:106FE000374A0021049B039804F06CFA45E035A071
:106FF000ECE7284603F046FF039805F06FF93CE004
:10700000206809F0B9FD6068401C606003282FD338
:1070100000222D4966602DE02068039988422CD11A
:107020002AA1029A0198FEF747F900280ED02BA159
:10703000029A0198FEF740F9002807D02AA1029A87
:107040000198FEF739F9002805D016E0666020683F
:1070500009F0ACFD0CE0206809F08EFD6068401C72
:107060006060032804D303206060206809F00CFDF1
:1070700021490022049804F03FFA002007B0F0BD37
:10708000FFE70120FAE700002C01002025642C20F6
:1070900025700D0A000000005544500041542B4358
:1070A000495053544152543D25642C222573222CBF
:1070B000222573222C25750D0A000000881300007C
:1070C00020BF02005443500040470108414C524544
:1070D00041445920434F4E4E45435400434F4E4E7A
:1070E000454354204F4B0000434F4E4E45435420E0
:1070F0004641494C00000000F04701087FB50646B4
:1071000085680020374C362910D00CDC022964D069
:1071100004DC002915D0012962D126E0032929D0F9
:1071200010295DD12AE03739042959D8039001A8E4
:10713000009003CA03AB2CA205F09EFA02284CD1A2
:107140002BE01046E26009F0CFFC002845D005F0A6
:1071500035FC2061002840D04068009025A22A49D3
:107160002846E36803F06AFE37E02061284603F012
:1071700089FE32E0E06809F0E1FC29E003F00AFF53
:10718000012803D1206903C804F0B4F820691F491D
:107190000CC8284603F07EFE1FE0E0680399884291
:1071A0001BD11BA1029A0198FEF786F8002807D090
:1071B00019A1029A0198FEF77FF80028DAD00CE0B6
:1071C000E06809F091FC002807D0216905F0CAFBAE
:1071D00000221449304604F08FF9002004B070BD3D
:1071E0000120FBE72C01002025642C2025700D0ACE
:1071F0000000000041542B43495053454E443D2567
:10720000642C25750D0A000088130000204E000034
:1072100053454E44204F4B0053454E442046414970
:107220004C000000F0470108F8B50546002405F0C1
:1072300099F8204609F066FC03281AD0204609F088
:1072400061FC04281DD0204609F05CFC052814D000
:10725000641C032CEDDB1C4F03217869401CFDF7F7
:107260005DFF0C460026084609F04CFC06280DD0B0
:107270001EE00421204609F0BBFD22461349E86BBD
:1072800012E0124922461039E86B0DE0204609F061
:107290002BFC00280CD005F091FB002808D00B49EE
:1072A0007C6122461031E86B04F026F90020F8BD1D
:1072B0000321601CFDF732FF761C0C46032ED2DB47
:1072C0000020C043F8BD00002C0100209C480108AC
:1072D000F8B58568274E6A6B0B001468264AD77884
:1072E0000BF08FFC10090D141721232323232323D4
:1072F000233823253B230020D07090611EE02846D0
:1073000003F0C0FD204604F0E9FF2BE000221B49FA
:107310001DE00E2103467D220091D200002120466F
:1073200004F0D0F81EE0012FF0D00120F8BD012FAD
:10733000ECD091690A2907D2491C916110A231460B
:10734000284603F07BFD0DE00C490022103104F0CB
:10735000D3F807E00120D07004E0002006F0B6FA70
:10736000012801D00020F8BD044900224039074817
:10737000EDE7000088130000B8000020A0470108D6
:1073800041542B4350494E3F0D0A0000101000207D
:1073900010B50446022006F099FA012802D0002018
:1073A000C04310BD084A00231360E06B4168516080
:1073B000496818329360516003491A46183104F045
:1073C0009BF8002010BD0000F400002010B5032041
:1073D0000BF010F810BD000005480649406804E0B5
:1073E000884201D10120704740680028F8D17047D9
:1073F00010100020E047010810B50446022006F0F6
:107400006DFA012802D00020C04310BD084A0023B5
:107410001360E06B416851604968283293605160A5
:1074200003491A46283104F067F8002010BD000017
:10743000F400002070B50D4614461146284605F0AC
:1074400001F901280DD1285D00280AD1002C04D0B3
:1074500028192038C07F0A2809D0294605A003F042
:1074600021FF2246294603200BF04AF970BD294628
:1074700004A0F4E75B41542053656E645D202573DE
:107480000D0A00005B41542053656E645D20257336
:107490000000000010B5044600F05CF8002815D08C
:1074A0002046FEF7FDFF002810D0204600F03EF9F0
:1074B00000280BD02046FFF76BFF002806D020469F
:1074C000FFF79AFF002801D00020C04310BD000044
:1074D00070B5054604F046FF0446284600F03AF829
:1074E00000281BD02846FFF79FFE002816D028460C
:1074F000FEF7D6FF002811D02846FFF705FB00282D
:107500000CD01048104A8168611A914207D98460F2
:1075100000220E490E4803F0EFFF002070BD284600
:1075200000F004F90028F9D02846FFF731FF0028C1
:10753000F4D02846FFF760FF0028EFD00020C043BA
:1075400070BD0000B80000201027000000480108AE
:107550001010002010B5002006F0C0F9012803D15A
:107560000321002006F0C2F9002006F0AFF901283F
:1075700002D00020C04310BD00220349034803F09D
:10758000BBFF002010BD0000604701081010002064
:10759000FEB50446002668460670002C12D0E0684E
:1075A00000280FD0606A00280CD02746A06A4D4DF5
:1075B0002037002806D078E0E268694620469047E8
:1075C000002802D00020C043FEBD68460178E06A72
:1075D000626A431CE3621154E16A606A4654E06ADD
:1075E00009280BD1092240A0616AFDF74FFE00284F
:1075F00004D10120287001F09FFDE860287801285F
:1076000003D0022801D0032809D101F095FDE968D3
:10761000401A384988424DD82878012809D0C0B28C
:107620000A2822D0684600780D2823D00A2824D0C2
:1076300026E031A1606AFDF7F6FD0290002834D003
:10764000019601AB2DA2E16A606A05F015F80228E7
:1076500030D1019800282DD0626A0299891A081841
:10766000C01CA8600A2028701FE0E16AA868814257
:107670001BD11FE00120387405E0387C012806D0BA
:10768000387C022805D0E06A01280ED109E00220EA
:107690003874E06A022801D03E740BE0E6623E7462
:1076A00003E0606A00783E2804D0A06AE16A401EC8
:1076B000814281D3E16A606A04F0C4FF01280CD1E1
:1076C000E06A002805D0616A08182038C07F0A28BF
:1076D00006D00EA0616A03F0E5FD2E700020FEBD0D
:1076E0000EA0F8E7A00000202B524543454956451F
:1076F0002C000000DC0500003A0000002B5245433E
:10770000454956452C252A2C25643A005B415420D6
:10771000526563765D2025730D0A00005B4154209D
:10772000526563765D2025730000000010B50446A5
:1077300006F010F9012802D00020C04310BD084A0D
:1077400000231360E06B4168516049680832936020
:10775000516003491A46083103F0CEFE002010BDE7
:10776000F4000020F1B54A4A484884B0117801720B
:10777000517841724749C71D0978474CF971217DFD
:107780000173617D41730026354668460CF0CDFAE1
:1077900004206946320E2D02154332020E5C164358
:1077A000401EF7D526636563E17814204143FF222C
:1077B0000498913250430818FF30D7300104C8179D
:1077C000891968410206080A1043E0610CF0DFFAEB
:1077D000E069002540084000010E0002E163A0635B
:1077E0002A48636B2130226B0CF0D0FD2748E36BF5
:1077F0002530A26B0CF0CAFD244828492130898924
:107800000181274821490078387021207872029838
:1078100000220007000FF874C91D26200CF098FB09
:10782000002126200CF0A6FB01200CF0F7FAA07036
:107830001C4801F02FFEE08164216170FF3091301F
:1078400080B20121C9032082884201D3401A2082DC
:10785000144801F01FFEA081134E0AE0114801F008
:1078600019FE80B2A081218A884202D389198842F8
:1078700006D300210F200CF019FAA0610006EDD507
:107880000A48217A455405B0F0BD0000493E002069
:10789000880000208C000020D8020020C038002082
:1078A0008E00002030070020983A00007C3F002026
:1078B00010B5064CE078401CC0B2E070642804D9D2
:1078C0000020E07000F032FE207010BD00000020AB
:1078D00010B500231A4603E0845CE3189BB2521CE7
:1078E0008A42F9D3D84380B210BD0000F1B500241C
:1078F000084E094D09E06000811902226846FDF733
:10790000C5FC002804D0641CA4B2687A8442F2D377
:107910002046F8BDA43F0020D8020020014840784E
:1079200070470000A401002000B587B01C21684604
:10793000FDF762FC012168464170022101700D488B
:107940000190C8010290C000049040200590694653
:1079500000200AF0A1FD07480749203801610749C6
:10796000C1610749816107494161074804F092FB01
:1079700007B000BDF0290020B17A0008A57A000800
:10798000E17A0008EF7A0008502400207CB5444CCE
:10799000607800280AD0002501280AD00126022894
:1079A00033D0032804D16846057060E004F0E6FA9D
:1079B0007CBD6846057001A9022001950AF05AFDB8
:1079C0007D26F6000AE06846007803280DD0656041
:1079D000334601226946019803F0EDF8694600201C
:1079E0000AF008FD0028EED07CBD6068002808D0B1
:1079F00004F0B8FC6168401AC828E9D9002060701A
:107A0000E6E704F0AFFC6060E2E76846057001A9B4
:107A1000022001950AF02EFD08E068460078032850
:107A20000BD0A560684600780AF056FF6946002032
:107A30000AF0E0FC0028F0D07CBDA068002809D046
:107A400004F090FCA168401AC828EBD9A670002069
:107A50006070E7E704F086FCA060E3E76846007822
:107A600003280BD0E560684600780AF035FF6946C8
:107A700000200AF0BFFC0028F0D07CBDE0680028A0
:107A800009D004F06FFCE168401AC828EBD9A67051
:107A900000206070E7E704F065FCE060E3E70000C9
:107AA000A401002010B5014600200AF0A3FC10BD7F
:107AB0000FB400B5FFB082B0012183AB4902684624
:107AC000829A0BF059F86846FDF7CBFB02466946EF
:107AD00000200AF015FE7FB002B008BC04B01847C1
:107AE00001B50122694600200AF00AFE08BD10B562
:107AF0000446FDF7B6FB0246214600200AF000FED0
:107B000010BD00000149487000207047A40100200A
:107B100010B5024801F002F810BD0000B4090020C1
:107B200030B5446C1C252C400125A540046C6560D3
:107B3000046863608368102B036803D09960006851
:107B4000C26030BD9A600068C16030BD7D2100B563
:107B5000C900484300F001F800BD002140E000BF2B
:107B600000BF00BF00BF00BF00BF00BF00BF00BF1D
:107B700000BF00BF00BF00BF00BF00BF00BF00BF0D
:107B800000BF00BF00BF00BF00BF00BF00BF00BFFD
:107B900000BF00BF00BF00BF00BF00BF00BF00BFED
:107BA00000BF00BF00BF00BF00BF00BF00BF00BFDD
:107BB00000BF00BF00BF00BF00BF00BF00BF00BFCD
:107BC00000BF00BF00BF00BF00BF00BF00BF00BFBD
:107BD00000BF00BF00BF00BF00BF00BF00BF491C07
:107BE0008142BCD37047000010B506F0BFFE2020D4
:107BF00009F022F901200BF0ADFF002009F01CF97B
:107C000004480BF04BFE04480CF0C8F800200CF0C0
:107C1000FDF810BDCC0200208380000010B50120CB
:107C200001F094F910BD10B50120800201F08EF929
:107C30000120400301F08AF910BD72B6FEE7000092
:107C400010B5084900224A6107494B684C15234387
:107C50004B604B68082423434B60C009C00102609D
:107C600010BD0000FC090020002002407FB5002468
:107C70000D460646039401F0A7F8E809029003A90F
:107C800001960094684601F037F80749002806D0AD
:107C90000120088001F06CF8002004B070BD0C8059
:107CA00001F066F80120F8E7D001002010B50023AC
:107CB00002E0C45CCC545B1C9342FAD310BD0000BC
:107CC00010B5214A00219069C305204804D54169B7
:107CD000022319434161911593699B0505D54369B9
:107CE0000124234343616302194393695B0505D56E
:107CF0004369082423434361E301194393691B0546
:107D000005D54369042423434361630219439369FE
:107D10009B0405D54369102423434361630219433F
:107D200093699B0304D5446920231C434461194390
:107D30009369DB0305D54369402423434361A002D3
:107D40000143916110BD000000200240FC090020A9
:107D500070B5054601F0F0F90646184C0AE0681CBB
:107D600008D0002D04D001F0E7F9801BA84201D90A
:107D7000032070BDA069C007F1D1A069800701D5BB
:107D80000220A061A069C00511D4A06980050ED4AD
:107D9000A06940050BD4A069000508D4A06980043F
:107DA00005D4A069800302D4A069C00303D5FFF7FE
:107DB00087FF012070BD002070BD00000020024040
:107DC000F8B51746002605460C4600F0FDFF0BE00F
:107DD00029460220226800F0D9FF0849002848807F
:107DE00004D1241D2D1D361DBE42F1D300F0C0FF6D
:107DF000BE4201D20020F8BD0120F8BDD001002014
:107E00000FB4F8B504460D460026002C04D1401EE0
:107E1000F8BC08BC04B01847E06A002800D1F7E7B6
:107E200009A80090E76A29462046009B089AB847AF
:107E30000646002000903046EAE7FFB504460D46AE
:107E4000002100260023214600BF11E0D800115078
:107E5000D80080184660D80086185B1C68684F6898
:107E6000B84204D103980660002004B0F0BD496810
:107E70000029EBD1481EF8E7F8B505460026002793
:107E80002E0CAFB20848046809E02088B04205D142
:107E900000223946204603F071FA02E06469002CA2
:107EA000F3D100BFF8BD00000C04002070B5022122
:107EB0000B4801F035F90B490B4D002805D0012086
:107EC0000870288A401C288270BD0024074E0C7060
:107ED0003078022801D101F053FB34702C8270BD40
:107EE00000040050F901002000000020FA010020E9
:107EF00010B5827F5118C9B28177182914D3183967
:107F00008177417F0122491CCCB24477017F0B006D
:107F10000AF077FE0D0A080B081908190808190855
:107F2000191E0A001F2C10D810BD817E8B0703215B
:107F3000002B03D01C2CF7D9427702E01D2CFBD874
:107F400010BD017710BD1E2CFCD94277491CF8E703
:107F50001F2CF7D942770277418B491C418310BD12
:107F600010B5054B64220549054802F024FE962011
:107F7000FFF7ECFD10BD0000B80B0000240000204E
:107F8000A408002010B586B003AA009201AB0FA28E
:107F900004F072FB0024E443022811D104990398F1
:107FA00004F001FBC3B201980121027803E00198BB
:107FB000405C4240491C02988842F8D89A4202D05C
:107FC000204606B010BD0020FBE700002425702AE3
:107FD00025700D0A0000000010B588B000F038FAD6
:107FE000164C0122A188206801F09FF80A2000F0B9
:107FF00065FEA1880022206801F097F80A2000F0B1
:108000005DFEA1880122206801F08FF801206946F9
:108010004870022008700A49019141020291094901
:10802000039104210491059069460AF035FA20462F
:108030008821103004F096FA08B010BD68230020A3
:10804000681F002099010020F3B51F488DB001275B
:108050000E46077028216846FDF7CEF831460D9888
:10806000FFF790FFBC1E002807D10AAB17A23146CC
:108070000D9804F001FB0F2802D020460FB0F0BD90
:108080000A98002401781D488519203D302916D012
:108090001B488368002B03D0324600200D99984777
:1080A000112118480902016017480770EC77AC7776
:1080B000B21E12480D99FDF786F80020DEE7114840
:1080C000046011480470F1E70700002024252A2CE1
:1080D000252A2C252A2C252A2C252A2C252A2C2514
:1080E000702C252A2C252A2C252A2C252A2C252AB9
:1080F0002C252A2C252A2C252A2A0000243D002064
:108100009801002018000020F8010020F3B5002598
:108110004468ED43066883B0092C0AD322462E2119
:10812000304604F00FFC070003D0B81B0190042870
:1081300002D0284605B0F0BD0221304604F0A7FB6E
:10814000FDF7D8FA054600910221B01C04F09FFB10
:10815000FDF7D0FA029001980E46241A641E2146BB
:10816000781C04F094FBFDF7C5FA0E4F04E00022E2
:108170003B46FDF715FA641E002CF8D102460B466B
:1081800031460298FDF7F2F80022074BFDF708FA96
:108190002A46009BFDF7EAF8049AD160906000201F
:1081A000C8E700000000244000004E40F3B5002561
:1081B0004468ED43066883B00A2C0AD322462E2178
:1081C000304604F0BFFB070003D0B81B0190052820
:1081D00002D0284605B0F0BD0321304604F057FB1D
:1081E000FDF788FA054600910221F01C04F04FFBD0
:1081F000FDF780FA029001980E46241A641E21466B
:10820000781C04F044FBFDF775FA0E4F04E00022E1
:108210003B46FDF7C5F9641E002CF8D102460B461B
:1082200031460298FDF7A2F80022074BFDF7B8F996
:108230002A46009BFDF79AF8049A516110610020CC
:10824000C8E700000000244000004E40F3B59BB09A
:108250000F465E4C1B98FFF795FE0026F64300255F
:10826000002801D02576A0E010AB079313AA0EA931
:1082700015A804AB07C319AB03930CAA17A90AA846
:108280006B4607C308AB52A239461B9804F0F4F9B9
:108290000D2872D10B980A9901286ED108784128CF
:1082A00006D02576207E012805D000201DB0F0BD27
:1082B00001202076F6E7089F2E213846099A04F01F
:1082C00041FB002871D0C01B06286ED10221384620
:1082D00004F0DDFAA0770221B81C04F0D8FAE077A8
:1082E0000221381D04F0D3FA202108551198109F5F
:1082F00006285AD10221384604F0C9FA60770221D3
:10830000B81C04F0C4FA20770221381D04F0BFFA2B
:108310007D21090140186083214617A8FFF7F6FE6A
:10832000002842D1214619A8FFF740FF00283CD180
:108330000F9F0E990A2F38D2002F0FD03A4603A86C
:10834000FCF741FF03A8C5550BF0E0F92B4A2C4B75
:10835000FDF7BEF8FDF7F0F9208000E02580284603
:10836000149F139D002F0DD03A462E21284604F06D
:10837000E9FA002802D0411B01E016E03946284600
:1083800004F085FA60800D980C9901280DD800281A
:1083900007D00878532804D10122E068D207504062
:1083A000E06016981599012801D930467EE700282B
:1083B00007D00878572804D101226069D2075040BD
:1083C000606108212046FFF793FD6EE7002400203E
:1083D00024252A2C25702C25702C25702C25702CFA
:1083E00025702C25702C25702C25702C25702C25A3
:1083F0002A2C252A2C252A2A000000006F1283C06F
:10840000CAA1FD3FC3000248C150181882807047BE
:108410006823002008B500206946087003E068461C
:10842000007800F023F86946022009F0E3FF0028F5
:10843000F5D008BD10B505490020087001220520BF
:108440001103000700F071FE10BD0000980100202C
:1084500010B505490120087001030520002200071E
:1084600000F063FE10BD00009801002070B5204DA3
:1084700000262C462B78611C8034002B08D0224625
:108480005268022B0CD0032B09D10A2813D02CE000
:10849000242804D102222A7070540120606070BD2B
:1084A00050546168491C61607E291ED20D28F6D1A6
:1084B0000320287070BD50546068401C60604654B2
:1084C0000CA1681CFCF7AFFE002804D0681C616892
:1084D000FFF7BAFD09E009A1681CFCF7A4FE00281B
:1084E00003D0681C6168FFF7B1FE2E7070BD0000FC
:1084F000782300204747412C00000000524D432CB8
:108500000000000010B5084800F05EFA0A21064895
:1085100000F0F6F9044800F0E1F8800503D50248C0
:1085200000F0DEF880B210BDC4060020F8B5FFF7F9
:10853000E9FFFDF7C3F8274E3146FCF7D9FE264C7C
:1085400026490025206188423EDB2078244F002800
:1085500015D02570FFF7D6FFFDF7B0F83146FCF7D0
:10856000C7FE2061FDF706F900223B46FCF7A2FF9B
:1085700000221C4BFCF7ACFFFDF724F9A06020693A
:10858000FDF7F8F800223B46FCF794FF164A174B1C
:10859000FCF79EFF06460F46A068FDF7EBF8124A6F
:1085A000134B5242FCF794FF32463B46FCF7DEFE8B
:1085B000FDF708F90F49A060884201DDA16004E0E1
:1085C000FF21C905C84200D3A560A068FDF7A0F847
:1085D000C0B2F8BD00401B44BC0100200000604058
:1085E00000000C4000E064403333333333B3304099
:1085F000CCCCEC3F0000C84210B5104C607800288D
:1086000012D1012149020E4800F08AFD00280BD149
:108610000C480078002807D1A079002804D1E0791F
:10862000002802D00020607110BD6079401CC0B2EB
:1086300060710528F8D900F0A3FF10BD00000020EC
:1086400000040050FA010020F8B506460D464036F9
:10865000317C01290DD00121317401688A685207EB
:1086600009D5416D2022114341650020307401205D
:10867000F8BD0220F8BD174B6A68D80547109A422A
:10868000154C8A6A2B6812D05B035B0B1A438A6213
:108690002968490305D5A1680143A1600A20FDF7B7
:1086A0002FFD2868800312D5A06838430EE05B03D5
:1086B0005B0B9A438A622968490302D5A16881430A
:1086C000A1602868800302D5A068B843A06000209C
:1086D0003074F8BD0110000000270140406D704764
:1086E0000068006C7047000070B5040006D0606D33
:1086F000264600254036002802D006E0012070BD45
:10870000A5653574204600F0D3F8606DC00603D42B
:1087100021688868400705D5606D102108436065B1
:108720003574EBE7606DFF22013290430222104363
:10873000606588688207920F5B48012A02D10A6847
:10874000D2072BD1032362689B079A4205D05B4274
:108750009A4202D05B009A4209D10A6992009208BB
:108760000A6121680A6963681A430A610CE00A69B0
:10877000920092080A6181680F22920491438160FD
:1087800081686268114381602168CA6818239A432E
:10879000CA602168CA68A3681A43CA608168012256
:1087A0005206914381608168A28E52061143816016
:1087B00020688168C90004D481680122120711432E
:1087C00081602068C168394A1140C1602069E16850
:1087D000022825D000200143204620300278037B68
:1087E00052035B001A431143226B1143A2699203A7
:1087F0001143E269D20311432268D3681943D1605F
:10880000616A0A46FF3AC23A05D0A26A1143226859
:10881000D3681943D16042780121012A02D00BE0CC
:108820000420D8E70078002823D0606D2022104370
:108830006065A06D0843A065E06B012820681FD02B
:108840000169C90703D0016949084900016120682D
:108850004169C908C900416120684169A26B11439F
:108860004161A565606D80088000401C6065002046
:1088700070BD2068C26801231B041A43C260DBE795
:108880000269FF239B009A43026120680269236CFE
:10889000A66C1A43636C33431A4302612068026971
:1088A0000A430261D3E70000002701401902FEFFDE
:1088B00010B586B0044614216846FCF79DFC0E49AD
:1088C0002068884216D10D48416B4215114341631F
:1088D000C16A01221143C162C06A69461040059015
:1088E0000220009003200190002002900520000744
:1088F00000F038FB06B010BD00240140001002401B
:10890000F8B504464069254640350E4608280BD088
:108910002068C068C00709D0606D202108436065E9
:10892000002028740120F8BD082700E00C2700F083
:1089300003FC009015E0701C13D0002E05D000F051
:10894000FBFB0099401AB0420BD9206800683842FE
:1089500007D1606D0421084360650020287403205E
:10896000F8BD206800683842E5D0606D01214902F9
:10897000084360652068C16809058A0F0C21002A38
:108980001BD12022125D002A17D10268120714D5CC
:10899000826853070122002B08DB43688B43436046
:1089A000606D130298431043606506E0606D2023FC
:1089B00018436065A06D1043A065A069002801D12F
:1089C000206801600020F8BD70B5044621680020D1
:1089D0008968490721D425464035297C01291CD0C6
:1089E00001212974E169012904D02046FDF79AFB91
:1089F000002811D1616D0A4A1140FF220132114352
:108A000061650021A165297422681C21116021681B
:108A10008A6804231A438A6070BD022070BD00007A
:108A2000FEF1FFFF30B5014620314A790023022ACA
:108A300004D00422C2630B71012030BD02681468A7
:108A40000E25AC4314600268146864086400146066
:108A5000446C1C22144001221546006CA540456060
:108A60004A7118460B7130BD70B5002401462031A3
:108A70004A79022A03D00421C163012418E0026864
:108A800013680E25AB431360026813685B085B0034
:108A90001360436C1C221340012215469D40036C59
:108AA0005D604A7100220A71816B002900D08847FD
:108AB000204670BD70B5040029D0206801684908BF
:108AC000490001601348256814212818FCF710FBA1
:108AD000800060641048206400202860626C1C21C3
:108AE0000A4001239340226C53600B4A8032936A00
:108AF000656C0D400F21A9408B439362E0622063B7
:108B00006063A063E06320346071207170BD012058
:108B100070BD0000F8FFFDBF00000240F0B4016C22
:108B20000D6801680C68466C1C2304221E40174621
:108B3000B7402F420ED067070CD50C68A40602D4AC
:108B40000C6894430C60416C19408A40016C4A6087
:108B5000016B1AE00227B74002462F402032002F57
:108B600017D0A70715D50C68A40605D40C680A25EC
:108B7000AC430C6001215171446C02211C40036C18
:108B8000A140596000211171C16A002918D0F0BCC0
:108B900008470827B7402F4212D0240710D50C6889
:108BA0000E25AC430C60446C01211C400B46A340D5
:108BB000046C6360C163517100211171416BE4E782
:108BC000F0BC704770B504003CD01F4825681421E4
:108BD0002818FCF78DFA800060641C48206402218C
:108BE000204620300246417129681948E368014057
:108BF000A06866691843236933431843A36918437F
:108C0000E3691843236A1843084328600121A068D8
:108C10008903884210D00D488030836A656C1C211E
:108C20000D400F26AE40B3438362656C63680D4010
:108C3000816AAB400B4383620020E06301215171E4
:108C4000107170BD012070BDF8FFFDBF0000024033
:108C50000F80FFFFF8B504468C46203001790025CF
:108C6000012909D00126067141790027012905D083
:108C7000077102252846F8BD0220F8BD0221417186
:108C8000E7632068016849084900016061462046A1
:108C9000FEF746FF206B00282068016801D00E22F5
:108CA00005E0042291430160206801680A22114313
:108CB00001602068016831430160DBE770B504465C
:108CC00000F03AFA0546601C02D0044800782418E7
:108CD00000F032FA401BA042FAD370BD9000002091
:108CE00070B5054600F028FA044600F025FA001B8E
:108CF000A842FAD370BD0000F8B51A4E0546307C84
:108D00000F46012807D0012030741748FFF720F8DC
:108D1000010002D021E00220F8BD0020C0433860ED
:108D20006C6814E02046FEF78BFF0F48FFF710F841
:108D300001460E48426808239A4342604268431540
:108D40009A434260002901D03C6006E08034A86864
:108D50006A68C0018018A042E4D800203074084638
:108D6000F8BD0000FC09002050C3000000200240B4
:108D700005484168022211434160416801221143C4
:108D8000416000207047000000200240F8B50C4C04
:108D90001646207C0F46012808D00120207409487F
:108DA000FEF7D6FF0025002802D006E00220F8BD1D
:108DB00065613E600348FEF7CBFF2574F8BD0000F7
:108DC000FC09002050C3000011484168C9070BD0BE
:108DD000EFF3108172B60F4AC2600F4AC26081F38E
:108DE00010884168C9070ED1416889070DD5EFF396
:108DF000108172B6094A0261094A026181F3108842
:108E00004068800701D501207047002070470000AE
:108E100000200240EFCDAB8905040302BFAE9D8C5C
:108E200016151413F0B5002262E0012393401C468E
:108E30000C405CD09608304DB6007519AF68AC4652
:108E400095072E0F0F25B540AE463D4005273F073D
:108E5000B84201D1002719E0284FB84201D10127BB
:108E600014E0274FB84201D102270FE0254FB84246
:108E700001D103270AE0244FB84201D1042705E0BD
:108E8000224FB84201D1052700E00627B740AF4284
:108E900012D11F4D2E68A6432E606E68A6436E60E9
:108EA000EE68A643EE60AE68A643AE606546AD6868
:108EB0007446A5436446A560056856000324B44083
:108EC00025430560D508AD002D182E6AAC46550720
:108ED000EF0E0F25BD40AE4365462E62C568A54323
:108EE000C56045689D4345608368A3438360521C09
:108EF0000B46D34099D1F0BD000001400004005062
:108F000000080050000C005000100050001C0050E1
:108F10000004014010B5012189020B4C884207D1A1
:108F200008F036F8A089401CA08105F07BF910BD3F
:108F30000128FCD108F02CF86078012801D100F05C
:108F40001FFB0020E08110BD0000002010B5044987
:108F50004A69024202D04861FFF7DCFF10BD000001
:108F600000040140F8B5002303240125C2E0324685
:108F70002E469E40B446324079D00E79B607B60FE1
:108F8000012E01D0022E17D186682746B6465E0014
:108F9000B74000967646BE43B646CF68009EB740BF
:108FA00076463743876046686746BE430F79FF06BB
:108FB000FF0F9F40374347600E79F643B6070ED048
:108FC000C6682746B4465E00B646B7406646BE430E
:108FD000B4468F687646B74066463743C7600E7919
:108FE000B607B60F022E14D1DE08B600361800966A
:108FF000366A5F07B446FE0E0F27B646B740664690
:10900000BE43B4460F697646B74066463743009E76
:10901000376206682746B4465E00B646B7406646E5
:10902000BE430F79B446BF07BF0F7646B7406646CA
:10903000374307604E68B603B60F5AD0304F7E6B89
:109040002E437E639F082F4EBF00BE190096B66860
:109050000F27B4469E07360FB646B7406646BE4356
:1090600005273F07B446B84202D100271AE040E086
:10907000254FB84201D1012714E0244FB84201D155
:1090800002270FE0224FB84201D103270AE0214F07
:10909000B84201D1042705E01F4FB84201D105278E
:1090A00000E006277646B74066463743009EB76025
:1090B0001A4EB6684F689643FF0200D51643174F05
:1090C000BE60FE684F689643BF0200D51643134F3B
:1090D000FE607E684F689643BF0300D516430F4F6E
:1090E0007E603E684F689643FF0300D516430B4AE7
:1090F00016605B1C0A681646DA4000D037E7F8BDF8
:109100000010024000000140000400500008005020
:10911000000C005000100050001C005000040140E2
:109120000069084000D001207047002A01D0816109
:1091300070478162704700000148806870470000F6
:109140009000002070B504000FD021681548086019
:1091500021681548086003CC41602068083C2168FC
:109160008860FFF7E9FF05460CE0012070BDFFF7BE
:10917000E3FF401B2A2805D92068C068400701D0BA
:10918000032070BD2068C0684007F0D120680269E4
:10919000E1688A4201D0016101E0044901600020D8
:1091A00070BD0000CCCC000055550000AAAA0000FC
:1091B000006802490160002070470000AAAA000070
:1091C0000248816802788918816070479000002009
:1091D00010B50848002401684022114301600320B3
:1091E00000F00AF8002801D0012401E000F09CF909
:1091F000204610BD0020024070B504460D4D7D2074
:109200002978C000FBF774FF01460B480068FBF7A4
:109210006FFF01F0AFF8002809D1042C07D200221B
:109220002146401E00F0A8F900206C6070BD0120AE
:1092300070BD0000900000209C0000207047704727
:10924000F8B507F0A5FEFFF7D7F904F0B1FC012748
:109250007F0239461F48FFF763FF1F4E00251F4C52
:10926000002810D0307800280DD1607A401CC0B2A0
:109270006072022807D965722562E561A5616561A2
:1092800006F070FB05E06369A269E169206A06F0F7
:109290004BFBFEF70BFE09F027FC6089401C608148
:1092A000E089401CE08107F03BFBFEF701FB3946FB
:1092B0000848FFF735FF002808D13078002805D18D
:1092C0002562E561A561656106F04CFB0448FFF786
:1092D0006FFFF8BD00040050F601002000000020E0
:1092E0002007002070477047704710B5044600689B
:1092F0000168C943C90708D18168C943C90704D1B6
:10930000012141602046FFF79BFF20680168C943A7
:10931000890708D48168C943890704D402214160C0
:109320002046FFF78BFF20680168C943490708D42E
:109330008168C943490704D404214160204600F0F4
:10934000F1F820680168C943090708D48168C94356
:10935000090704D4082141602046FFF7C3FF2068B5
:109360000168C943C90608D48168C943C90604D441
:10937000102141602046FFF762FF20680168C94361
:10938000890608D48168C943890604D42021416034
:109390002046FFF7A9FF20680168C943490608D4A1
:1093A0008168C943490604D4402141602046FFF743
:1093B0009AFF10BDF8B5040005D025462035A87BDE
:1093C000002802D006E00120F8BD00206873204686
:1093D00000F048F80220A8732068C26884466368D9
:1093E000012B04D00120A16AC005814201D11E20B9
:1093F000824319486169814201D0184802401848E7
:10940000A668024018463043676A266A3E433043E6
:10941000A66A30431043002B18D0012B03D0012241
:10942000D205964203D12369E2681A4310430A4ADF
:10943000914205D0A2691143E269024308461043F4
:109440006146C8600120A8730020F8BD2369E26965
:109450001A431043E3E70000FFFF00003F1FFFFF38
:10946000FEF119FF10B50068084988420CD1084880
:10947000816BC20411438163002211460D2000F06C
:109480007BF80D2000F06CF810BD0000007C00405F
:10949000001002400068C06970470000F8B504463B
:1094A0000220254620351746A8731D480268C304CC
:1094B0001A4302602068C2689B121A43C260206887
:1094C0000269012632430261226810205060206840
:1094D00081611021204603F0B9FD03281FD02168C7
:1094E00008204860206847610821204603F0AEFD4F
:1094F000032814D0204603F033FDA87B03280ED0A8
:1095000020688168314381602068016931430161CD
:1095100020680169042211430161AE730020F8BD87
:1095200000040140704700000448416B01221143D0
:109530004163816B02041143816370470010024054
:10954000002809DBC106C90E0120884003490860D4
:10955000BFF34F8FBFF36F8F7047000080E100E0D3
:10956000002805DBC106C90E0120884001490860BA
:109570007047000000E100E010B509F04FFB10BD9E
:10958000BFF34F8F04490348C860BFF34F8F00BF3C
:10959000FDE700000400FA0500ED00E00248016864
:1095A000821511430160704700700040F0B5154A04
:1095B0001368154D54152D6A2340ED07ED0F002B50
:1095C00004D0002D02D01668A64316601668B608AF
:1095D000B600064316600D48076904263743076145
:1095E00001290DD040BF20BF20BF0169B1430161F7
:1095F000002B04D0002D02D0106820431060F0BD75
:1096000030BFF2E7007000400000014000ED00E0D4
:10961000F8B5044600780027594D800674D5584E99
:10962000403EB06BC00004D4B06BA9050843B063E2
:10963000012754480168C90511D4016882151143F6
:109640000160FFF779FD009005E0FFF775FD0099D7
:10965000401A642837D84B480068C005F5D53268F1
:109660000321090560680A400140914208D0810346
:10967000890F032904D13168890301D50120F8BD80
:109680002A69032109040A4022D0084090421FD0D1
:109690002078800631D528692A6988430121C904C8
:1096A0000A432A612A698A432A612861C0050FD5C5
:1096B000FFF742FD009008E0FFF73EFD0099411AD8
:1096C0003148814201D90320F8BD28698005F3D5CE
:1096D0002078800611D561688803800F032805D1A2
:1096E00032680005824301400A4332602869032240
:1096F00061681204114008432861002F04D0B16B47
:10970000012000078143B1632078C00705D0E868D5
:10971000A168800880000843E8602078800705D5AC
:10972000E8680C218843E1680843E8602078400736
:1097300006D5E86803218902884321690843E86067
:109740002078000706D5E86803210903884361698A
:109750000843E8602088C00506D5E86803210904AD
:109760008843A1690843E8602078000606D5E868C8
:10977000032189048843E1690843E8600020F8BDBB
:10978000401002400070004088130000F8B50E46FB
:10979000050038D05E480068C007C00FB04214D240
:1097A0005B4C20684008400030432060FFF7C4FC59
:1097B000074605E0FFF7C0FCC11B564881427AD836
:1097C0002068C007C00FB042F4D12878524C8007FF
:1097D00005D5E068F0218843A9680843E06028784F
:1097E000C00752D06868022806D0032807D0216835
:1097F00001280AD0890504E02168890301E0216875
:109800008901002903DB0120F8BD4907F9E7E16878
:10981000890889000143E160FFF78EFC074668680C
:1098200002280AD0032814D001281ED029E0FFF70F
:1098300083FCC11B374881423DD8E0680007800F98
:109840000228F4D121E0FFF777FCC11B31488142A7
:1098500031D8E0680007800F0328F4D115E0FFF746
:109860006BFCC11B2B48814225D8E0680007800FA4
:109870000128F4D109E0FFF75FFCC11B25488142B4
:1098800019D8E0680007800FF5D121480168C907A1
:10989000C90FB14217D90168490849003143016035
:1098A000FFF74AFC074608E005E0FFF745FCC11B4F
:1098B0001848814201D90320F8BD15480068C00747
:1098C000C00FB042F1D12878400706D5E0680721E3
:1098D00009028843E9680843E0602878000707D553
:1098E000E0680721C90288432969C9000843E0608C
:1098F00000F03AF8E168094A0906090F515CC840CE
:109900000749086007480068FFF776FCF8BD0000CB
:109910000020024088130000001002405444010857
:109920009C00002094000020044805490068C96894
:10993000044A4905490F515CC84070479C0000200B
:10994000001002406D440108044805490068C968D8
:10995000044A8904490F515CC84070479C000020AC
:10996000001002406D44010870B51A4AD3681A49C4
:109970000C2018408D0004280CD04E00082810D070
:109980000C2810D050680004410F0120C003491C6E
:10999000884070BD1068C00601D5084670BD2846D5
:1099A00070BD304670BD98020C4C000F205C1B024D
:1099B0009C0FD368641CDB0301D5314603E01268B9
:1099C000D20600D4294609F004F922460023FBF709
:1099D000B9FB70BD0010024000093D00644401085D
:1099E000FEB505007ED0F74CE7680C20E66807401E
:1099F0000120000406402878C00747D0082F05D072
:109A00000C2F0AD101200004864206D12068800371
:109A10003CD568680028E5D038E00120696800047A
:109A2000814203D121680143216011E00523012215
:109A30001B0492049942216802D111432160F1E78D
:109A4000814321602168014000912068904320609B
:109A5000686800280DD0FFF76FFB009005E0FFF766
:109A60006BFB0099401A64287ED820688003F6D5E5
:109A70000CE0FFF761FB009005E0FFF75DFB00994C
:109A8000401A6428F0D820688003F6D4287880072C
:109A90005DD5E868810604D5226820210A4322604A
:109AA00088430923042F0DD00C2F01D1002E09D09B
:109AB00000283CD02168994301432160FFF73CFB1B
:109AC000064628E02168490701D500288AD0616848
:109AD0001F22120291432A69120211436160216818
:109AE000994300E091E101432160FFF73DFFE16808
:109AF00009060A0FB449895CC840B4490860B448F3
:109B00000068FFF779FB002874D120E0FFF714FB11
:109B1000801B0228A8D820684007F7D560681F215D
:109B20000902884329690902084360600FE0206840
:109B3000400840002060FFF7FFFA064604E0FFF708
:109B4000FBFA801B02288FD820684007F7D42878BA
:109B5000C00661D5002F0DD0A86900284BD0206821
:109B6000FF210131084300E0C6E02060FFF7E4FA7E
:109B700006462DE02068800502D5A8690028A5D0FA
:109B80006068072149038843296A08436060606868
:109B9000297F0002000A090608436060286A410B19
:109BA0000120C003491C8840E16809060A0F864964
:109BB000895CC8408549086085480068FFF71CFB40
:109BC000002817D128E0FFF7B7FA801B0228A1D898
:109BD00020688005F7D56068072149038843296A12
:109BE000084360606068297F0002000A0906084394
:109BF000606011E0E1E02168FF20013081432160D5
:109C0000FFF79AFA064604E0FFF796FA801B02284F
:109C100072D820688005F7D428786E4E000724D5C6
:109C200068690028306910D0012108433061FFF7CE
:109C300083FA009005E0FFF77FFA0099401A0228A6
:109C40005AD830698007F6D50FE0400840003061EF
:109C5000FFF772FA009005E0FFF76EFA0099401ADC
:109C6000022849D830698007F6D42878400765D59E
:109C700000200290A06BC00006D4A06B0121090750
:109C80000843A0630120029053480168C90511D41C
:109C90000168821511430160FFF74EFA009005E05C
:109CA000FFF74AFA0099401A642825D84A48006804
:109CB000C005F5D5FF20AA680130824203D1316981
:109CC0000143316111E001218902002A07D00523F7
:109CD0001B029A4203D132690A433261EFE73269CB
:109CE00082433261306988433061A86800280FD010
:109CF000FFF722FA009007E05EE0FFF71DFA0099F7
:109D0000411A3648814257D830698005F5D50DE0B3
:109D1000FFF712FA009006E0FFF70EFA0099411AD9
:109D20002E48814248D830698005F5D40298002831
:109D300004D0A06B012109078843A063686A00284A
:109D400065D00C2F4CD0012636060228206805D09D
:109D5000B0432060FFF7F0F905462FE0B0432060E4
:109D6000FFF7EAF9074604E0FFF7E6F9C01B02280F
:109D700022D820688001F7D4E96AA86AE26808431B
:109D8000296BFD231B049A4311430843E0602068BC
:109D900030432060FFF7D0F9054604E0FFF7CCF927
:109DA000401B022808D820688001F7D52FE0FFF774
:109DB000C3F9401B022801D90320FEBD20688001A1
:109DC000F5D424E000100240544401089C00002017
:109DD00094000020401002400070004088130000F2
:109DE0000128EAD0E06801210904AA6A01409142F1
:109DF0000BD10F218904EA6A0140914205D1032168
:109E000089050840296B884201D00120FEBD002051
:109E1000FEBD000070B5040005D0254620356878E9
:109E2000002802D006E0012070BD002028702046E6
:109E300000F046F8022068702068C168C943C9066E
:109E400037D5CA214162216853204862204604F078
:109E50005DF9002827D120688168184A1140816087
:109E6000216888686268A369104322691A43104315
:109E700088602168E068086120680169228912040D
:109E800011430161204604F064F900280BD12168D8
:109E9000CA6C92089200CA646269E169114322683F
:109EA000D36C1943D1642268FF215162002801D08C
:109EB00070BD00200121697070BD0000BFFF8FFFE1
:109EC00000680549884205D10448016901229204CD
:109ED000114301617047000000280040401002401B
:109EE00070B5044621680A48C860FFF725F97D2649
:109EF0000546F60006E0FFF71FF9401BB04201D906
:109F0000032070BD2068C0688006F4D5002070BDB5
:109F10005FFF0100F8B504000ED0FF27606A053727
:109F2000002500280AD02561656126464036A562D5
:109F3000707C002807D00AE00120F8BD6068B842B4
:109F4000F3D0E561F1E73574204600F03FF80221D7
:109F500071742068026840239A4302602123A2683A
:109F600060689B021A4038401043E3688A0213403D
:109F7000184323690B40217D1843C907C90F0843C3
:109F8000A169931019400843E16938231940084337
:109F9000216A802319400843A16A930019400843AD
:109FA00021680860A0690421000C0840616A102340
:109FB00019400843216848602068C1699143C16124
:109FC0006565012070740020F8BD000010B586B0F2
:109FD000044614216846FBF70FF9104920688842AF
:109FE00019D10F48416B821411434163C16A0122A8
:109FF0001143C162C06A002110400590E02000902A
:10A0000002200190032003900291049105206946EB
:10A010000007FEF7A7FF06B010BD000000300140AA
:10A0200000100240FFB5054604464035287C002755
:10A0300081B01646012809D001202874FFF77CF86A
:10A040000090687C012804D0022797E0022005B028
:10A05000F0BD0298002874D0002E72D003206874DE
:10A060000020606502992163A686E686A063A0872A
:10A07000E087606420640122A068D20340219042FE
:10A0800008D1206802688A430260206802680B02D7
:10A090001A43026020680268520602D402680A432A
:10A0A00002600121E068C9028842606828D1002866
:10A0B00001D0012E1ED1206B21680088C86006E007
:10A0C00020688168890709D5216B0988C160206BE8
:10A0D000801C2063E08E401EE0860BE0FFF72CF82A
:10A0E0000099411A0498814202D3401C02D005E035
:10A0F000002803D0E08E0028E2D128E003273BE0CF
:10A10000002801D0012E1FD1206B21680078087330
:10A1100006E020688168890709D5216B09780173F9
:10A12000206B401C2063E08E401EE0860CE0FFF7B1
:10A1300003F80099411A0498814203D3401C03D0CC
:10A14000DCE717E00028D9D0E08E0028E1D12046D6
:10A15000009A049904F03CFE002801D0202060659C
:10A16000A068002803D12068C16880680090606DF5
:10A17000002801D0012701E0012068740020287424
:10A18000384664E7FFB5044683B0012025464035D4
:10A190000090287C00271E4601280FD0012028743B
:10A1A000FEF7CAFF0190687C616801280DD0CA1FC4
:10A1B000FD3A08D1A168002905D102E0022007B0CC
:10A1C000F0BD042801D00227D0E0049800287AD0FE
:10A1D00005980028FBD0002EF9D0687C042801D017
:10A1E00005206874002060650599A163E687A6874D
:10A1F00004992163E686A68620646064206801686D
:10A20000490603D401684022114301600121E0683E
:10A21000C9028842606847D1002801D0012E3CD194
:10A22000206B21680088C860206B801C2063E08E52
:10A23000401EE08631E020688168890710D5E18EF4
:10A2400000290DD0009901290AD1216B0988C1602C
:10A25000206B801C2063E08E401EE0860020009072
:10A2600020688168C9070DD0E18F00290AD0C06835
:10A27000A16B0880A06B801CA063E08F401EE0876C
:10A2800001200090FEF758FF0199411A0C98814275
:10A2900003D3401C01D0032766E0E08E0028CAD11A
:10A2A000E08F0028C7D148E0002801D0012E3ED120
:10A2B000206B216800780873206B401C2063E08EBF
:10A2C000401EE08633E04DE020688168890710D5A4
:10A2D000E18E00290DD0009901290AD1216B09785E
:10A2E0000173206B401C2063E08E401EE08600203E
:10A2F000009020688168C9070DD0E18F00290AD03D
:10A30000C068A16B0870A06B401CA063E08F401E6A
:10A31000E08701200090FEF70FFF0199411A0C9889
:10A32000814202D3401C02D0B5E70028B3D0E08EB2
:10A330000028C9D1E08F0028C6D12046019A0C9987
:10A3400004F046FD002803D00127202060650DE0C1
:10A35000A068002803D12068C16880680090606D03
:10A36000002801D0012701E0012068740020287432
:10A37000384624E7094910B5401E884201D901201A
:10A3800010BD074C60610321081F08F047FC002046
:10A39000A06107202061002010BD0000FFFFFF002A
:10A3A00000E000E0F0B502462032137E012B21D000
:10A3B000012515760223537606687468B368702702
:10A3C000BC430F68274377600068AC07A04208D001
:10A3D000094CA04205D0094CA04202D0084CA04232
:10A3E00004D180244968A343194381605576002035
:10A3F0001076F0BD0220F0BD0004004000080140CE
:10A400000014014002462032137E012B06D00123A6
:10A4100013760068016500201076704702207047AF
:10A4200010B586B0044614216846FAF7E5FE0D49DA
:10A430002068884213D10C48C26A04210A43C262D0
:10A44000C06A084005904020009002210020019140
:10A4500002900491039069460448FEF783FD06B01C
:10A4600010BD000000040040001002400008005031
:10A47000F8B5064604462036307E00270D460128F2
:10A480000ED001203076002A0CD0042A1BD0082AD6
:10A490002FD00C2A3ED00127002030763846F8BD58
:10A4A0000220F8BD206806F00BFE206881690822B2
:10A4B000114381612068826904218A438261206896
:10A4C0008169EA6812E0206806F012FE206882695D
:10A4D0000121C9020A438261206881690122920236
:10A4E0009143816120688169EA68120211438161A8
:10A4F000D2E7206806F015FE2068C16908221143E2
:10A50000C1612068C26904218A43C2612068C169AF
:10A51000EA6812E0206806F01FFE2068C169012287
:10A52000D2021143C1612068C269012189028A43B4
:10A53000C2612068C169EA6812021143C161ABE7D8
:10A5400070B5050005D02C462034607E002802D06E
:10A5500006E0012070BD00202076284600F010F8AB
:10A5600002206076291D286806F076FD0120A0777C
:10A57000A076E076207760776076002070BD0000DE
:10A5800000680449884204D10348816B02221143C8
:10A59000816370470004004000100240704770471C
:10A5A00070B504001BD02420E067206801684908CA
:10A5B000490001602068002505602068456020682A
:10A5C0008560204600F09EF9204680304560E567B2
:10A5D00005602566656660342576002070BD012023
:10A5E00070BD10B508F03EF810BD0000F8B5026867
:10A5F0000446D06911689368A44D06462E4025464E
:10A600008035002E71D0A24FDE07F60F0F40374382
:10A610007ED0C70706D0CF0504D5012717626A6828
:10A620003A436A60820708D5DA0706D02768022213
:10A630003A626A6804273A436A60420708D5DA0733
:10A6400006D0236804221A626A6802231A436A60E9
:10A65000020709D520220A40324305D02368082288
:10A660001A626B6813436B60020509D54A0107D56E
:10A6700001222368D2021A626A6820231A436A60A0
:10A680006A68002A39D0800606D5880604D5A16EEE
:10A69000002901D0204688476868216889684906F2
:10A6A00002D4282108422DD0204606F0F0FE216871
:10A6B0008868400622D5EFF31080012282F31088CB
:10A6C0008A6840239A438A6080F31088606F00286C
:10A6D00014D070498163606FFEF7C6F900280CD072
:10A6E000606F816B08E000E012E0860610D58E06F0
:10A6F0000ED5A16EAFE020468847F8BD2046FFF793
:10A7000070FFF8BD2046FFF76CFF00206860F8BDC1
:10A71000266E012E7DD1C6067BD5CE0679D51023B7
:10A72000136222689068264640064036002849DABF
:10A73000616F086840680004000CE8D0378B8742DE
:10A74000E5D9708308680068800634D4EFF3108080
:10A75000012181F3108811681F01B943116080F352
:10A760001088EFF31080012181F3108821688A6836
:10A77000520852008A6080F31088EFF310800121A4
:10A7800081F3108821688A684027BA438A6080F381
:10A7900010882020286000202066EFF3108001211F
:10A7A00081F3108821680A689A430A6080F3108850
:10A7B000606FFEF737F902206066308B718B401AAC
:10A7C00081B234E0308B718B401A81B2708B0028DB
:10A7D0009DD000299BD0EFF31080012686F31088CE
:10A7E0001668FF272137BE43166080F31088EFF309
:10A7F0001080012282F3108822689668760876001D
:10A80000966080F310882020286000202066A066D3
:10A8100000E010E0EFF31080012282F3108822683C
:10A8200015689D43156080F31088022060662046FD
:10A83000FFF7B4FEF8BDC50208D55B0206D50120BE
:10A84000000510622046FFF7AAFEF8BD030606D5F4
:10A850000B0604D5E16E002900D04CE7F8BD400698
:10A86000FCD54806FAD52046EFF31081012383F387
:10A87000108813684024A343136081F310882021BB
:10A88000C1670021C16600F089FAF8BD0F08000019
:10A89000200100041D13010810B5040003D0E06F6F
:10A8A000002802D007E0012010BD002178200155CA
:10A8B000204600F06DF82420E06720680168490810
:10A8C00049000160204606F0FBFE0128ECD0606ADA
:10A8D000002802D0204606F05AFC20684168092270
:10A8E000D20291434160206881682A2291438160AD
:10A8F00020680168012211430160204606F0ACFC8B
:10A9000010BD000010B5044600681B4B05221B4912
:10A91000120798420BD1486B01239B03984348636D
:10A92000032149021046FEF77DFA1B200CE0144B70
:10A9300098420CD1886B01235B04984388630C21F7
:10A940001046FEF76FFA1C20FEF7FAFD10BD0D4A07
:10A950009042FBD1886B012212059043886311124B
:10A960000948FEF75FFA04210848FEF75BFA606FBA
:10A97000FEF7A0F80E20E7E7003801400010024083
:10A98000004400400050004000080050000C0050FF
:10A99000F0B587B0074614216846FAF72DFC494BFD
:10A9A0003A68002448480226032104259A421CD113
:10A9B000426B2B031A434263C26A01231A43C262E9
:10A9C000C06A039118400590480200900520019646
:10A9D0000495029469460007FEF7C4FA0022114666
:10A9E0001B20FEF7C9FD1B201FE0384B9A4220D1E7
:10A9F000826B01235B041A438263C26A01231A43F8
:10AA0000C262C06A0391184005900C200090052096
:10AA100001960495029469460007FEF7A3FA002206
:10AA200011461C20FEF7A8FD1C20FEF799FD07B07B
:10AA3000F0BD274B9A42FAD1826B01231B051A43C2
:10AA40008263C26A2A43C262C26A2A400592C36A0A
:10AA500008221343C362C06A019610400590500259
:10AA60000090032003900294694604961948FEF76B
:10AA700079FA032003900620049001960095029431
:10AA800069461548FEF76EFA154D14482860AC600B
:10AA90000D20EC6068606C618020AC612861202032
:10AAA0002C62E8612846FEF78DF8002801D0FDF7FA
:10AAB000C4F87D67002211460E20AF62FEF75CFDF0
:10AAC0000E20B2E700380140001002400044004070
:10AAD0000050004000080050000C00501C000240D4
:10AAE000B409002070B580231B58202B01D0022010
:10AAF00070BD00290BD0002A09D0012483682403EB
:10AB0000A34206D10369002B03D1CB0701D001205A
:10AB100070BD002303660B4B04689C420ED0636833
:10AB20001B020BD5EFF31083012585F310882568F0
:10AB30000126B6063543256083F3108806F0CAFE69
:10AB400070BD00000048004070B580231B58202BCA
:10AB500001D0022070BD00290BD0002A09D00124A9
:10AB600083682403A34206D10369002B03D1CB07DA
:10AB700001D0012070BD002303660B4B04689C428A
:10AB80000ED063681B020BD5EFF31083012585F30C
:10AB9000108825680126B6063543256083F31088A2
:10ABA00006F0EEFE70BD00000048004010B507F052
:10ABB0007BFD10BD7047FFB50446C06F83B01746DC
:10ABC0000D46202802D0022007B0F0BD002D0BD08A
:10ABD000002F09D00120A1680003814206D120691D
:10ABE000002803D1E80701D00120EDE700218420EF
:10ABF00001512120E067FEF79FFA2646403601907A
:10AC0000378277820120A1680003814202D1206946
:10AC1000002802D02F46002511E000270FE0002277
:10AC20008021204606F06CFF002815D1002F17D098
:10AC30002168387888627F1C708A401E7082708A12
:10AC4000019B002806980090E9D10022402120466F
:10AC500006F056FF00280AD02020E0670320B3E763
:10AC600028882168C005C00D8862AD1CE4E720205B
:10AC7000E0670020A8E7000070B50446C06F2028F8
:10AC800001D0022070BD00290BD0002A09D0012379
:10AC9000A0681B03984206D12069002803D1C80789
:10ACA00001D0012070BD20464030E1640282428222
:10ACB00000202546803568602121E167216F002949
:10ACC00018D0154BCB62236F14491963236F1449B5
:10ACD0005963216F134688632668E16C3246283237
:10ACE000206FFDF7B7FF002804D0102068602020F7
:10ACF000E067D6E7216840200862EFF31080012169
:10AD000081F3108821688A6880231A438A6080F35F
:10AD10001088002070BD0000391401088514010856
:10AD20003113010830B5C36F202B01D0022030BD94
:10AD300000290BD0002A09D0012384681B039C4200
:10AD400006D10569002D03D1CD0701D0012030BD0A
:10AD5000C164014640310A824A8200218422C166D0
:10AD600011502121C1679C4202D1016900290FD0F5
:10AD70000849C166EFF31081012282F31088006850
:10AD8000026880231A43026081F31088002030BDDE
:10AD90000149EEE7A71A0108491A010810B507F0A2
:10ADA0001BFD10BD7047F0B585B00446002500209E
:10ADB0000390002602900027002C02D06068002833
:10ADC00001D105B0F0BDA068402800D9F9E7002501
:10ADD0002EE0204600F0E4F82E46002003901FE00D
:10ADE000606A825D02AB2046039900F07AF907465B
:10ADF000022F0DD1606A0090E06A01906068029AAB
:10AE0000D20080186A464168204600F0A7F80AE0A0
:10AE1000002F00D107E000BF761C0398401C039070
:10AE2000E06AB042DCD800BF022F00D103E06D1C05
:10AE3000E06AA842CDD800BF00BFC2E70FB438B562
:10AE400004460D4607A80090E169A069009B069A98
:10AE500007F092FE20620020009009480078012847
:10AE600003D1216AA06900F079FA29462046236AB5
:10AE7000A26900F00FF838BC08BC04B01847000005
:10AE8000B806002010B50446A06B01F027FA002098
:10AE900010BD0000F8B504460D4616461F463A465A
:10AEA000314620466369984700280AD12046FFF7BB
:10AEB000E9FF0094074B2A460021A06B01F0A6FA97
:10AEC00006E00094044B01220021A06B01F09EFAE1
:10AED0000020F8BD1DB000080DB0000870B5044694
:10AEE0000D468021204601F03DFB2868E06368683C
:10AEF0006060A868A060E868E0602869206168690F
:10AF00006061A869A061E869E06100202062286AA8
:10AF10006062686AA0620020E06200213020015572
:10AF2000A86A60632046383001F0ECF9002802D0AE
:10AF30000020C04370BD204600F002F8FAE7000090
:10AF40000146002901D1401E70470348006808608F
:10AF5000014801600020F7E7B406002070B5044600
:10AF60000D461646022D06D0032D05D0042D04D023
:10AF7000052D07D102E000BF00BF00BF2046FFF74C
:10AF800081FF00E000BF00BF32462946E06B00F0C1
:10AF9000F5F970BD0148007870470000B806002040
:10AFA00010B50446012240216018FAF71EF910BDC1
:10AFB00010B50024124804681FE020462169884724
:10AFC000002819D10F480078012810D1E16A606A81
:10AFD00001F038FB012803D1606A00F03FF906E078
:10AFE000E16A606A00F086F907A000F037F92046B0
:10AFF000FFF7D9FE0020E0622468002CDDD110BDEF
:10B00000B4060020B80600200D0A000010B5044662
:10B01000002205212046FFF7A1FF10BD10B5044610
:10B02000002204212046FFF799FF10BD70B50446A9
:10B030000D46204600F02CF8012801D1801E70BD7D
:10B040002268501CE168FAF753F8216023692168EF
:10B050005943A368C81829462269FAF7B4F80020B2
:10B06000EDE710B58160C2600361012444600024F3
:10B07000046010BD10B504462268501CE168FAF760
:10B0800037F86068814201D1012010BD0020FCE743
:10B0900010B504462268901CE168FAF729F8606848
:10B0A000814201D1012010BD0020FCE770B50446AB
:10B0B0000D462046FFF7DEFF012801D1801E70BD3E
:10B0C000236960685843A368C11828462269FAF7C3
:10B0D0007AF86268501CE168FAF70AF861600020AB
:10B0E000EDE7F0B504460D46002600211DE02046A0
:10B0F0004030405C012817D1CF006068C059405DE6
:10B10000904204D000202746403778540CE0761C4B
:10B11000CF006068C0596F1CC05D002804D1002BAF
:10B1200000D019600220F0BD491CA0688842DED81A
:10B13000002E01D10020F6E70120F4E770B50446A7
:10B140000D46002C01D1401E70BD00BF2068A842F2
:10B15000FCD32068401B206062685019E168F9F751
:10B16000C7FF61600020EFE770B504460D46002C74
:10B1700001D1401E70BD20684019206000BFE16809
:10B1800020688842FBD8A2685019E168F9F7B0FF3F
:10B19000A1600020EEE7FFB581B004460D461646DB
:10B1A0000027002E06D00498002803D0E16820680C
:10B1B000884203D30020C04305B0F0BD2168E06899
:10B1C000401AA84202D20020C043F5E7A068401907
:10B1D000E16888420BD9A168E068471A2168E068F5
:10B1E000401AE919884202D20020C043E4E7A2686D
:10B1F000D019E168F9F77CFF316079190498016092
:10B200000020D9E7014648687047014688687047C2
:10B210000246002A01D1401E704700205060906015
:10B220001060D16000BFF7E70146002901D101207D
:10B2300070470868002801D10120F9E70020F7E7EE
:10B240000146002901D1012070470A68C868904270
:10B2500001D10120F8E70020F6E700000FB400B5A7
:10B260000E48FFB0407882B0002805D07FB002B011
:10B2700008BC002004B01847012183AB490268468E
:10B28000829A07F079FC06490246884200D90A46AC
:10B290006946002007F034FAE8E70000A401002026
:10B2A000FF0100000FB400B51048FFB0407882B035
:10B2B000002805D07FB002B008BC002004B01847B9
:10B2C00000226946104607F01BFA012183AB4902B0
:10B2D0006846829A07F050FC05490246884200D928
:10B2E0000A466946002007F00BFAE3E7A4010020B4
:10B2F000FF010000F0B5064616480C46417891B0B3
:10B30000002923D10078012820D10127102C01D950
:10B31000102500E02546402101A8F9F76DFF4023E4
:10B3200001AA29463046009701F0CCF80AA101A8ED
:10B33000F9F76DFF01A8F9F794FF024601A9002073
:10B3400007F0DEF9641B7619002CDFD1002011B064
:10B35000F0BD0000A40100200D0A000010B5064A4F
:10B360005278002A01D0002010BD0A460146002074
:10B3700007F0C6F910BD0000A4010020F7B582B0A7
:10B3800004460D46002700266088012820D1206948
:10B3900000280AD1606800680195009019A2002178
:10B3A0002046E368FCF72CFD12E0A9002069405814
:10B3B00000782D280CD0A9002069405861680968E0
:10B3C0000091019017A200212046E368FCF718FDC8
:10B3D0006668F36829462046049A984707460CE0B9
:10B3E0007068002808D07068C36829462046049A0F
:10B3F00098470746766800E001E0012FF0D000BFD3
:10B4000005B0F0BD46534D3A252D387320535441B5
:10B4100054453A252D323873204556454E543A2529
:10B42000750D0A0046534D3A252D3873205354416B
:10B4300054453A252D323873204556454E543A2509
:10B44000730D0A00FFB581B004460E46174600256D
:10B45000002C01D105B0F0BD30212046F9F7CCFE1B
:10B460000A98A060049820616660E7600021A162EC
:10B4700061620E48008820800B9860800C4800684C
:10B4800060610B48046009480088401C0749088037
:10B49000656806E06560002211462046FFF76EFFF2
:10B4A000AD68002DF6D100BFD4E7000010040020E5
:10B4B0000C0400200246002A01D1401E7047D162D0
:10B4C0000020FBE7FFB583B005460E461C460C9FE7
:10B4D0000020029020880004B9B20843029002982C
:10B4E000044B009031462846059A00F08FFF07B0C4
:10B4F000F0BD0000797E0008F7B596B005460E460F
:10B500006F680024002015903C462AE06C60002201
:10B5100001212846FFF732FFA64205D10021284627
:10B52000189AFFF72BFF1EE0502101A8F9F764FEDF
:10B5300015AB01AA21463046FCF77FFC00280FD14D
:10B540000AE015980068686000212846189AFFF7FD
:10B5500015FF15984068159015980028F1D102E064
:10B560006468002CD2D100BFB46806E06C60002192
:10B570002846189AFFF702FFA468002CF6D119B0EC
:10B58000F0BD016E05E002467C324B1CD35C535487
:10B59000491CC26D8A42F6D8704710B5C26D511E63
:10B5A00005E002467C32545C4B1CD454491E026EAA
:10B5B0008A42F6DD10BD70B505460C46A879002814
:10B5C00002D001282ED100E000BF432C1BD004DCA8
:10B5D000412C0CD0422C22D10FE0442C19D07E2CCF
:10B5E0001DD100220821284600F040FB18E000226F
:10B5F0000321284600F03AFB12E0002204212846ED
:10B6000000F034FB0CE000220621284600F02EFB5F
:10B6100006E000220521284600F028FB00E000BFDC
:10B6200000BF2CE0432C1BD004DC412C0CD0422C5E
:10B6300022D10FE0442C19D07E2C1DD100220821EC
:10B64000284600F081F818E000220321284600F087
:10B650007BF812E000220421284600F075F80CE087
:10B6600000220621284600F06FF806E0002205219E
:10B67000284600F069F800E000BF00BF00BF00BF2F
:10B6800070BD70B504460D46432D46D008DC1B2D19
:10B690000DD0332D25D0412D3DD0422D4DD13BE055
:10B6A000442D3BD05B2D11D07E2D46D124E0207956
:10B6B000002802D0042804D100E000BF012020713E
:10B6C00002E00020207100BF00BF39E0207901288E
:10B6D00002D10220207102E00020207100BF00BFD3
:10B6E0002EE02079022802D10320207102E0002000
:10B6F000207100BF00BF23E02079032806D129462E
:10B700002046FFF758FF0420207102E0002020713E
:10B7100000BF00BF14E000BF00BF00BF20790228B7
:10B7200006D129462046FFF746FF0420207102E09B
:10B730000020207100BF00BF02E00020207100BF88
:10B7400000BF207970BD0000F7B504460D46092DF5
:10B7500002D00020A066E0662B0007F052FA0AFD36
:10B760000646CBFCFBFAF9F8F7FD6079002802D019
:10B77000012837D100E000BFE06D63282FD20B20F5
:10B78000C00120188169029888472046FFF705FF0D
:10B79000029821467C31226E8854206E401C20661F
:10B7A000E06D401CE065266E002709E022467C32F1
:10B7B000905D0B22D201A21891698847761C7F1CEC
:10B7C000E06DB042F2D805E00B20C001201881697D
:10B7D0000820884738467F1E0028F5D100BF00208A
:10B7E000607100E000BF00BF3EE2E06D002806D1BE
:10B7F0000B20C00120184169FEA0884734E260791F
:10B80000002802D0012856D11FE0002120467C30BC
:10B81000E26D81546422616F51430246C832881838
:10B8200021467C31F9F73FFD606F401C6067606F17
:10B830000A2801DB00206067A06F401CA067A06F92
:10B840000A2801D30A20A06736E000BF00BF6422A7
:10B85000206F50432246FF32453281186422E64869
:10B860002018F9F7B0FC266F11E00A21701CF9F7D7
:10B870003FFC0F4664227A432346FF334533D118F9
:10B8800064227243D0186422F9F79DFC3E46616F32
:10B89000084609300A21F9F741FCB142E5D164219B
:10B8A00071432246FF32453288186422D24961181A
:10B8B000F9F789FC00E000BF00BF0B20C001201891
:10B8C0004169CEA08847204600F002FD20467C302A
:10B8D00000F054FC002000F0FBFC00202066E06536
:10B8E000606F0A3020670B20C00120184169C4A096
:10B8F0008847B9E16079002802D0012855D100E0DD
:10B9000000BFA06F002800D150E0A06F0A2803D12B
:10B91000616F206F88420CD1A06F0A2842D0616FFE
:10B920000A31A26F881A0A21F9F7E2FB206F8142DF
:10B9300038D0216F084609300A21F9F7D9FB216771
:10B940006422206F50432246FF3206E01CE1DBE018
:10B9500096E084E076E02BE085E1453281182046D0
:10B960007C30F9F7A0FC20467C30F9F77AFCE065E2
:10B97000E06D20660B20C00120184169A1A0884716
:10B980006423226F5A432346FF334533D0180B22DA
:10B99000D201A218516988470B20C00120184169C3
:10B9A00099A088470120607100E000BF00BF5BE103
:10B9B0006079002802D0012841D100E000BFA06FCB
:10B9C000002800D13CE0616F084609300A21F9F7F0
:10B9D000A5FB206F81422FD0216F481C0A21F9F767
:10B9E00087FB21676422206F50432246FF32453295
:10B9F000811820467C30F9F756FC20467C30F9F758
:10BA000030FCE065E06D20660B20C0012018416924
:10BA10007CA088476423226F5A432346FF33453373
:10BA2000D0180B22D201A218516988470B20C001FF
:10BA30002018416974A088470120607100E000BFB0
:10BA400000BF11E1206E002808DD206E401E206638
:10BA50000B20C001201881690820884704E1E16DAE
:10BA6000206E88420BD222467C32236ED05C0B22A1
:10BA7000D201A21891698847206E401C2066F3E02D
:10BA80006079002802D001283BD100E000BFE06DC2
:10BA9000002833D0206E002830DD0B20C001201894
:10BAA000816908208847266E012709E022467C32FA
:10BAB000905D0B22D201A21891698847761C7F1CE9
:10BAC000E06DB042F2D80B20C0012018816920201F
:10BAD000884705E00B20C0012018816908208847AD
:10BAE00038467F1E0028F5D1206E401E2066204675
:10BAF000FFF747FDE06D401EE06500BF002060716C
:10BB000000E000BF00BFAFE06079002802D001284C
:10BB100037D100E000BFE06D00282FD0206E002854
:10BB20002CDD216EE06D884228D0206E461C012756
:10BB300009E022467C32905D0B22D201A218916965
:10BB40008847761C7F1CE06DB042F2D80B20C00104
:10BB5000201881692020884705E00B20C0012018AB
:10BB600081690820884738467F1E0028F5D1204685
:10BB7000FFF707FDE06D401EE06500BF002060712B
:10BB800000E000BF00BF6FE06079002802D001280C
:10BB900066D100E000BFE06D00285ED0E06E0028B6
:10BBA0000AD10120E06621467C312046E030E26D7A
:10BBB000F9F709FBE06D606642E0A06E00F026FB3D
:10BBC00006462146E031626EF9F776FB002834D153
:10BBD0000B20C001201841690CA08847A06E00F01E
:10BBE00015FB06460B20C0012018416930468847E6
:10BBF000A06E0FE00D0A3E002C0500000D0A0000AB
:10BC00003E0000000D3E00001B5B4A000D1B5B4A1E
:10BC10003E00000000F0FAFA0646314620467C302D
:10BC2000F9F741FB20467C30F9F71BFBE065E06D3E
:10BC30002066A06E401CA06607E0A06E401CA066B7
:10BC400000F0DEFAA16E8842B7D800BF00F0D8FA43
:10BC5000A16E884201D80020A0660020607100E03B
:10BC600000BF00BF00E000BF00BFFEBDF7B5044647
:10BC70000E46330006F0C5FF09F2064EF2F2B0BDE3
:10BC8000D8F1F200E06D632843D2A079012806D1F3
:10BC90000B20C001201881692A20884705E00B206D
:10BCA000C00120188169029888472046FFF775FC7B
:10BCB000029821467C31226E8854206E401C2066FA
:10BCC000E06D401CE065256E002713E0A079012897
:10BCD00006D10B20C001201881692A20884707E07F
:10BCE00022467C32505D0B22D201A218916988470E
:10BCF0006D1C7F1CE06DA842E8D805E00B20C00158
:10BD0000201881690820884738467F1E0028F5D111
:10BD10000DE10CE1E06D002809D1A079002806D1E1
:10BD20000B20C0012018416982A08847FFE0A0795C
:10BD3000002802D001284CD117E0002120467C3099
:10BD4000E26D81540B20C001201841697DA0884715
:10BD50000120A07100202066E06522467C3210217F
:10BD600020460C3000F07BFD34E0002120467C3082
:10BD7000E26D81540020E06522467C32402120465D
:10BD80001C3000F06CFD21461C3120460C3000F0C8
:10BD90008BF900280CD10B20C001201841696DA03F
:10BDA00088470220A07100202066E06560710FE0E6
:10BDB0000B20C001201841696AA088470B20C001F0
:10BDC000201841695BA088470020A0712066E065CB
:10BDD00000E000BF00BFAAE0206E002808DD206E52
:10BDE000401E20660B20C00120188169082088476A
:10BDF0009DE0E16D206E884215D2A079012806D120
:10BE00000B20C001201881692A20884708E02246BB
:10BE10007C32236ED05C0B22D201A2189169884734
:10BE2000206E401C206682E0E06D00283FD0206E2E
:10BE300000283CDD0B20C0012018816908208847BC
:10BE4000256E012715E0A079012808D10B20C0013B
:10BE5000201881692A20884709E029E066E0224607
:10BE60007C32505D0B22D201A218916988476D1C6B
:10BE70007F1CE06DA842E6D80B20C0012018816924
:10BE80002020884705E00B20C00120188169082088
:10BE9000884738467F1E0028F5D1206E401E206658
:10BEA0002046FFF76EFBE06D401EE06500BF3EE000
:10BEB000E06D002839D0206E002836DD216EE06D5F
:10BEC000884232D0206E451C012713E0A07901285A
:10BED00006D10B20C001201881692A20884707E07D
:10BEE00022467C32505D0B22D201A218916988470C
:10BEF0006D1C7F1CE06DA842E8D80B20C001201803
:10BF000081692020884705E00B20C0012018816945
:10BF10000820884738467F1E0028F5D12046FFF7C5
:10BF200030FBE06D401EE06500BF00E000BF00BFD9
:10BF3000FEBD00000D0A757365726E616D653A2075
:10BF4000000000000D0A70617373776F72643A200D
:10BF5000000000000D0A57656C636F6D65210D0AC6
:10BF60003E0000000D0A55736572207665726966A1
:10BF700079206661696C65642E00000038B5002088
:10BF800000900024414804687CE072E000F0EAF987
:10BF90000546684601782046FFF773FB002800D06D
:10BFA00067E0A068281A3A49884205D9A5600220AE
:10BFB000A0710020E0652066A079002802D0012849
:10BFC0002BD100E000BF684600780D2806D16846F6
:10BFD000027802212046FFF749FE1DE068460078FE
:10BFE0000A2819D068460078082805D100220721C0
:10BFF0002046FFF73BFE0FE068460078092805D190
:10C00000002209212046FFF731FE05E0684602784C
:10C0100001212046FFF72AFE29E0684600780D2816
:10C0200006D16846027802212046FFF78DFB1DE00D
:10C03000684600780A2819D068460078082805D193
:10C04000002207212046FFF77FFB0FE068460078BB
:10C05000092805D1002209212046FFF775FB05E0DC
:10C060006846027801212046FFF76EFB00BF00BF43
:10C0700000BF0B20C0012018C1696846884700280E
:10C0800084D02468002C80D138BD00002804002012
:10C0900040771B0003490968016002218171014951
:10C0A0000860704728040020024600207047000006
:10C0B00000BFEFF30580002800D0704707480068F4
:10C0C000002804D1012080F3108800BF00BF03487E
:10C0D0000068401C0149086000BFEEE7140400201E
:10C0E00070B504460D4600F0A3F800280FD000F00C
:10C0F0009FF80B21C90140180069002807D000F003
:10C1000097F80B22D2018018016902A0884700200D
:10C1100070BD00001B5B481B5B4A000070B5024607
:10C120000C4600210023002A01D0002C02D100205F
:10C13000C04370BD0021002316E0C8000D4D2858F3
:10C14000002810D1D8001058CD000A4E7051D800E8
:10C1500080184068CD00AD19686007480068401C31
:10C16000054D28605B1C491C502901D2A342E4D331
:10C170000020DEE73404002030040020F0B595B044
:10C180000446002600E0641C20782028FBD02046CE
:10C19000F9F767F8002801D115B0F0BD2046F9F78E
:10C1A00060F80019461E02E000203070761E3078DC
:10C1B0002028F9D0142301AA2021204600F078FB82
:10C1C0000746002513E0E9000C4A50582146F9F7CC
:10C1D0004FF800280AD1E8000849401801A9426830
:10C1E00038469047002800D105E004E06D1C00F0BF
:10C1F00007F8A842E7D800BF0020CDE734040020AC
:10C2000001480068704700003004002001460548DE
:10C210000068814201D304A07047C800034A105847
:10C22000FAE7000030040020000000003404002081
:10C2300001480068704700002C040020F8B506464D
:10C240000F46002536E0002418E0FFF7F1FF002834
:10C2500013D0FFF7EDFF0B21C9014018006900283A
:10C260000BD0FFF7E5FF0B23DB01C018026928198B
:10C27000C000134B195813A09047641C052C04DA16
:10C28000FFF7BEFF29198842DFD8FFF7D1FF00284A
:10C290000FD0FFF7CDFF0B21C9014018006900281E
:10C2A00007D0FFF7C5FF0B22D2018018016907A054
:10C2B00088476D1DFFF7A4FFA842C4D80020F8BD31
:10C2C00034040020252D3136730000000D0A0000D3
:10C2D00001490860704700002C0400200146202915
:10C2E00002D30020C0437047012218204843044B6A
:10C2F0001A50002218204843C01882600020F2E73C
:10C300007C44002070B505460024002D01D1401E5C
:10C3100070BD00240CE0182060430C490858002828
:10C3200005D1012118206043084A115002E0641C25
:10C33000202CF0D300BF202C05D105A0FEF78EFFE6
:10C340000020C043E4E72C600020E1E77C440020AB
:10C3500074696D65722049442069732066756C6C40
:10C360000D0A000001480068704700001804002012
:10C3700010B5002400BF41E018206043214908584F
:10C3800002283AD118206043401880681E49096885
:10C39000091A182060431B4A8018C06881422CD9B2
:10C3A00018206043114640184069002820D018200A
:10C3B000604340180079002804D10121182060430F
:10C3C00011500AE00221182060430E4A11500E4815
:10C3D0000168182060438018816018226243094B6D
:10C3E000D218106918226243D2185169884704E0B4
:10C3F000012118206043034A1150641C202CBBD338
:10C4000010BD00007C44002018040020F0B5044654
:10C41000059D202C02D30020C043F0BD0226182029
:10C4200060430E4F3E50182060433E468019017114
:10C430000B48066818206043C019866018206043C6
:10C440003E468019C260182060438019436118205D
:10C450006043801905610020DFE700007C44002074
:10C460001804002007480068401C06490860064878
:10C47000026840680021521C484103490A60486034
:10C4800070470000180400202004002000BFEFF3D4
:10C490000580002800D0704709480068002804D0B3
:10C4A00007480068401E06490860054800680028E3
:10C4B00004D100BF80F3108800BF00BF00BFEAE7CF
:10C4C00014040020FFB581B005460C460026002369
:10C4D00000200090002D03D0002A01D0002C02D1B2
:10C4E000002005B0F0BD0A98012801D1032000E02A
:10C4F00002206043401C0499884201D90020F0E7E3
:10C50000002618E0A85D00900099081100F019F8C5
:10C5100019465B1C505400990807000F00F011F8F1
:10C5200019465B1C50540A98012803D12021184653
:10C530005B1C1154761CA642E4D30020D05418464C
:10C54000CFE70146092903DC08463030C0B2704706
:10C550000A2905DB0F2903DC08463730C0B2F6E7AD
:10C560003020F4E770B504460D4629462046F8F71A
:10C5700043FE70BD0146302904DB392902DC084640
:10C5800030380EE0412904DB462902DC0846373802
:10C5900007E0612904DB662902DC0846573800E021
:10C5A0000020C0B2704710B502460B46002406E0DA
:10C5B0001078FFF7DFFF21014418521C5B1E002B8F
:10C5C000F6D1204610BD00B50246002305E01078E4
:10C5D000FFF7D0FF19014318521C10780028F6D13C
:10C5E000184600BD70B588B005460C46002007907F
:10C5F0000690059004902846F8F733FE064604A8F6
:10C6000005A906AA07AB0092019102900AA2314641
:10C61000284600F031F8042803D00020C04308B0B9
:10C6200070BD07982070069860700598A0700498F7
:10C63000E0700020F3E7000025642E25642E2564B9
:10C640002E25640002460B46002100BF10E0505C1E
:10C65000202803DB505C7E2800DC08E0505C0D28BD
:10C6600002D0505C0A2800D101E000207047491C2C
:10C670009942ECD30120F9E70FB4F0B585B0044638
:10C680000020049000222020039000200290002C23
:10C6900002D00C98002805D1002005B0F0BC08BCE1
:10C6A00004B018470DA80490CFE0002908D10C98D9
:10C6B0000078252803D10C984078652800D0C9E07F
:10C6C0000C98007825286ED10C98401C0C900C9882
:10C6D000007803900C98401C0C900398652877D044
:10C6E00004DC2A2807D0642873D113E0702872D0A4
:10C6F0007828F9D13EE008E020780C9B1B7898421E
:10C7000002D0641C491E00E001E00029F4D100BF02
:10C71000521C88E000260196009600230025202068
:10C72000049E20CE049618E02078009E002E05D1AD
:10C730002D2803D10126019600960CE0302809DB54
:10C74000392807DC012600960A265E430746303F5B
:10C75000F31900E003E0641C491E0029E4D100BF86
:10C76000019E012E01D1DE43731C002D00D02B60F1
:10C77000521C58E000230025049E20CE04961FE0A2
:10C780002078302806DB392804DC1E010746303FBC
:10C79000F31913E0612807DB662805DC1F01064654
:10C7A000573EBB190AE043E0412806DB462804DC7B
:10C7B0001F010646373EBB1900E003E0641C491E1A
:10C7C0000029DDD100BF002D00D02B60521C2AE0D3
:10C7D0001BE024E0FFE7049E01CE04960025002321
:10C7E000254609E026780C9F3F78BE4201D05B1CAD
:10C7F00000E003E0641C491E0029F3D100BF0028BB
:10C8000001D005604360521C0DE0049B01CB0493F2
:10C81000002800D00460521C0123029303E0012091
:10C820000290002200BF00BF029801280DD111E044
:10C8300020780C9B1B78984205D1641C0C98401CF6
:10C840000C90491E01E0002204E00C9800780028BA
:10C8500000D02AE700BF0020049010461DE70FB467
:10C86000F8B506460C46002509A80090214630463A
:10C87000009B089A06F080F9054600200090A5422A
:10C8800000D3651E2846F8BC08BC04B0184710B594
:10C8900002460B46002407E01078FFF76BFE0A21E2
:10C8A00061434418521C5B1E002BF5D1204610BD7D
:10C8B000FFB504461D4621460023002D03D0002C61
:10C8C00001D0002A02D1002004B0F0BD18465B1C44
:10C8D000800011500BE00E780198864206D10020AE
:10C8E0000870481C1E465B1CB6009051491C087815
:10C8F000002801D0AB42EED31846E5E770B50646F6
:10C900000025002478213046F8F7A1FC0446002CCD
:10C9100004D158213046F8F79AFC0446002C0BD07D
:10C92000641C05E02078FFF725FE29014518641CEA
:10C9300020780028F6D103E03046F8F7CCFC054615
:10C94000284670BD10B503460C46002100BF05E027
:10C95000585CA04201D1581810BD491C9142F7D330
:10C960000020F9E770B504460D46002C01D0002DDB
:10C9700002D10020C04370BD012120461030FEF7D7
:10C98000DDFB20462030A968FEF7D8FB0020F2E747
:10C9900070B504460D46002C01D0002D02D10020B8
:10C9A000C04370BD012120461030FEF7DDFB20465C
:10C9B0002030A968FEF7D8FB0020F2E710B5044646
:10C9C000002C00D110BD20461030FEF72DFC0128B0
:10C9D00001D10020F6E720462030FEF725FC012893
:10C9E00001D10020EEE720461030FEF70BFC0C21B1
:10C9F000484321684018E5E77CB504460E4600250B
:10CA0000002001900090002C00D17CBD2046103009
:10CA1000FEF716FC002801D00020F6E76B4601AABD
:10CA2000314620462030FEF7B6FB002801D000201A
:10CA3000EBE720461030FEF7E8FB0C214843216865
:10CA40004518A0680199401828606E600098A86099
:10CA50002846DAE7FFB581B004460E461D4600279A
:10CA60000C2068430399884202D3781E05B0F0BDBC
:10CA70000C202F4647432660676060688019A060DD
:10CA80000398C11BE160294620461030FEF7C0FB29
:10CA900020462030E168FEF7BBFB0020E6E7FEE71A
:10CAA000F8B50F460546002412E010482E786100C4
:10CAB000081832090EA16D1C009006F049F8009884
:10CAC0003207120F0AA1401C06F042F8641CE4B2BF
:10CAD000BC42EAD305480D227900425408180A22C4
:10CAE00042700248891C05F02BFCF8BDC03C0020B8
:10CAF0002578000070B501240E4D64030022214604
:10CB00002846FCF712FB002261002846FCF70DFBCB
:10CB10000A2006F07CFE012221462846FCF705FB90
:10CB20000A2006F074FE002221462846FCF7FDFA92
:10CB300070BD00000004005070B501240E4D640368
:10CB4000002221462846FCF7F0FA012291032846EC
:10CB5000FCF7EBFA0A2006F05AFE0122214628468D
:10CB6000FCF7E3FA0A2006F052FE0022214628468E
:10CB7000FCF7DBFA70BD000000040050F1B50024A2
:10CB80000126164F25467603002231463846FCF72B
:10CB9000CCFA0A2006F03BFE012231463846FCF76B
:10CBA000C4FA6006040E012189033846FCF7B8FA7E
:10CBB000002801D0641CE4B2052006F028FE6D1C9C
:10CBC000EDB2082DE0D30098002803D0FFF792FFC4
:10CBD0002046F8BDFFF7B0FFFAE700000004005060
:10CBE000F8B50126164F0546760300223146384631
:10CBF000FCF79BFA0024E80901D0012200E00022A2
:10CC0000012189033846FCF790FA6806050E0A20D0
:10CC100006F0FDFD012231463846FCF786FA0A206F
:10CC200006F0F5FD002231463846FCF77EFA0A2070
:10CC300006F0EDFD641CE4B2082CDCD3F8BD000066
:10CC40000004005070B501220C4D94032146284683
:10CC5000FCF76BFA0122560331462846FCF765FAC9
:10CC6000002221462846FCF760FA0A2006F0CFFD94
:10CC7000002231462846FCF758FA70BD00040050E7
:10CC800070B501240E4D6403002221462846FCF7AE
:10CC90004CFA6600002231462846FCF746FA0A2084
:10CCA00006F0B5FD012221462846FCF73EFA012296
:10CCB00031462846FCF739FA0A2006F0A8FD70BD77
:10CCC00000040050F8B50122144D960300243146AB
:10CCD0002846FCF72AFA062006F099FD01225703A0
:10CCE00039462846FCF721FA062006F090FD07E0B9
:10CCF000641CE4B2FA2C03D9FFF7C2FF0120F8BD8F
:10CD000031462846FCF70CFA0028F1D100223946BA
:10CD10002846FCF70AFA0020F8BD00000004005085
:10CD200010B50A48018C012903D100210184FCF7C8
:10CD300027FC0648064A40380188914202D1C08843
:10CD4000002801D1FCF71CFC10BD000000390020B8
:10CD5000AA55000010B5F9F7E9FB002801D0002022
:10CD6000C04310BD10B5FAF737FB10BD10B5002257
:10CD70000F210248FEF702FB002010BD101000201A
:10CD800010B5044603CC8EB0019100901DA2102175
:10CD900006A8083C05F0C2FE083403CC01910090BF
:10CDA00018A210210AA805F0B9FE0C2206A91748FE
:10CDB000F8F709FA15492C200B39C87513480C22CD
:10CDC0000AA90D30F8F7FFF91048104B7B3841796C
:10CDD00000200290039004900D48059101780D48C1
:10CDE0000B3B8088019100900BA264211846FFF74D
:10CDF00036FD064902460B39002003F0BDFF0EB098
:10CE000010BD0000252E386C660000006F02002067
:10CE100000000020C038002025732C2C2C2C2C3036
:10CE20002C30302C30302E302C2C2C2C2C2C2A302A
:10CE3000302C25582C253032782C25782C25642C44
:10CE400025642C2564250D0A0000000010B5184843
:10CE500000F032F81648401E4178817037212020BA
:10CE600000F071F80321212000F06DF8402122200C
:10CE700000F069F80821232000F065F8AA2130208D
:10CE800000F061F80B4802210187322000F05BF8C6
:10CE90000121332000F057F85F21202000F053F8E3
:10CEA000034800F009F80A2006F0B1FC10BD0000AC
:10CEB00021030020C038002010B501460F2000F0EB
:10CEC00021F8002800D0012010BD10B50446FFF75E
:10CED000B9FE3220FFF784FEFFF7F4FEE0B2FFF761
:10CEE0007FFEFFF7EFFEFFF7ADFE3320FFF778FE82
:10CEF000FFF7E8FE0020FFF741FE0446FFF7C0FE03
:10CF0000204610BD10B50C46FFF7DFFF2070012052
:10CF100010BD70B50D460446FFF794FE3220FFF7B2
:10CF20005FFEFFF7CFFEE0B2FFF75AFEFFF7CAFE43
:10CF30002846FFF755FEFFF7C5FEFFF7A1FE0A20C2
:10CF400006F065FC70BD10B5FFF7E3FF012010BDD2
:10CF500010B50248FCF7C9F910BD000030070020E9
:10CF6000FEB504460027EFF310800290012080F305
:10CF70001088344B2168CA1804D13348C76803208D
:10CF80008004074088680190C868009048698E69ED
:10CF9000002A08D12C4940398A6ACD042A438A6282
:10CFA0008A6AAA438A62014631433CD025492268F5
:10CFB000CA4205D12449CB68032292049343CB6033
:10CFC00025462035002810D021680A6901231A431C
:10CFD0000A61216848610821204600F037F80328DB
:10CFE00000D1A873216808204860002E10D0206866
:10CFF00001690122114301612068866110212046E8
:10D0000000F024F8032800D1A8732168102048609C
:10D010000C482168C14206D10B48C1680322920422
:10D0200091433943C16020680169490849000161A1
:10D0300021680198886021680098C860029880F390
:10D040001088FEBD0084FFBF4010024070B5064648
:10D050000B480D46002409490068F8F749F87D217E
:10D06000C90048433168401E00D103240B682A469A
:10D070009A4301D00028F6D1204670BD204E000012
:10D080009C00002010B50D480B4901600C498160DF
:10D090000C4941600C49C1600C490D4C016121688B
:10D0A00088470C48162240890721FF30D73003F00B
:10D0B0002BFFE06A804710BDB1DA0008D4410020A0
:10D0C00009DA0008C5DA000889DA000861DA000820
:10D0D000044A0108C03800201CB5002118480091FE
:10D0E000164A01910260C163120542608160072205
:10D0F0008263012202610246C16020321170FF2367
:10D100005170C233436281621173016381610422F1
:10D1100041634261C161FBF7E7FA002801D072B6B2
:10D12000FEE7084800908013019069460448FBF729
:10D130008BFA002801D072B6FEE71CBD0024014026
:10D14000C406002002000004F0B587B01421684630
:10D15000F8F752F85448C26A04210A43C262C26A0C
:10D160000A400592C16A01252943C162C16A29406A
:10D170000591C16A02263143C162C16A31400591FD
:10D18000C26A08210A43C262C06A012208400590AF
:10D190000C214648FBF7C9FF812105200022090127
:10D1A0000007FBF7C2FF002210214048FBF7BDFF3C
:10D1B00000223F493F48FBF7B8FF01223E493D4866
:10D1C000FBF7B3FF91210520012209020007FBF7BD
:10D1D000ACFF0920800211273F040024009069461B
:10D1E000019702943148FBF7BDFE1C200090029489
:10D1F0006946019503942D48FBF7B4FE0520694666
:10D200000007019700950294FBF7ACFE2B480090B5
:10D21000052002946946019503940007FBF7A2FEDE
:10D220002748009002946946019503942148FBF732
:10D2300099FE69461F48009602950194FBF792FEFD
:10D240000320400300900320039001950294694657
:10D250001848FBF787FEE8020090019469460294A3
:10D260001248FBF77FFE6802009001946946029421
:10D270001048FBF777FE002202210520FCF77CF91D
:10D280000520FCF76DF9002211460720FCF774F920
:10D290000720FCF765F90520012210210007FBF7A4
:10D2A00044FF07B0F0BD000000100240000800502D
:10D2B000810400000004005060E0000010990000AC
:10D2C000E184000010B50E480C490160FF210531D2
:10D2D000416000218160C16001614161C161012241
:10D2E000016252024162826181620721C162FCF7E0
:10D2F00011FE002801D072B6FEE710BD00300140DB
:10D300008407002010B586B0002405941E480494BC
:10D310000094019402941B49039401601F218460CE
:10D3200041600461F9214461C160FDF709F90028F9
:10D3300001D072B6FEE7049404A913480594FDF7E2
:10D3400031F8002801D072B6FEE7602000907D2001
:10D35000019002940022694603940B48FDF788F877
:10D36000002801D072B6FEE704210748FDF74AF80D
:10D37000002801D072B6FEE70348FDF751F806B069
:10D3800010BD000000040040DC07002010B50C4870
:10D390000A490160E1214902416000218160C160C8
:10D3A00001618161C1610C22016242614162FDF74C
:10D3B00073FA002801D072B6FEE710BD00380140B4
:10D3C0001C08002010B50C480A4901604B21C90116
:10D3D000416000218160C16001618161C1610C22F5
:10D3E000016242614162FDF757FA002801D072B62E
:10D3F000FEE710BD00440040A408002010B50C4812
:10D400000A490160E1214902416000218160C16057
:10D4100001618161C1610C22016242614162FDF7DB
:10D420003BFA002801D072B6FEE710BD0050004064
:10D430002C090020F8B5FFF773FC02218548FBF7A3
:10D440006FFE854D854E864F002861D038780228C2
:10D4500001D3FCF795F80120824C0027607141024E
:10D460002F707C48FBF75CFE002810D07E4811210D
:10D47000027809027D485A2A016009D97C48076070
:10D480007C4807607C4807600120A07000E0A7701E
:10D49000A079002801D0012809D1FAF7BBFFFFF7D6
:10D4A00065FCFEF765FFFDF783FD04F083FE734D19
:10D4B00028883C2810D9A07900280DD10120A0711E
:10D4C0002F802079002803D06D4804F0E3FE03E0AC
:10D4D00000216C4800F0D0F928881E2807D9A079CF
:10D4E000012804D12F800220A07103F0AFFCA079A5
:10D4F000022803D101210846FCF758F8F08F29884B
:10D500005A38884203DAA079A0E0FCF739F8F8BD70
:10D510005448002444718079022801D3FCF730F884
:10D52000012149024B48FBF7FBFD002811D02C706C
:10D5300000F0DCFAFAF72AFAFFF7F2FBFFF716FC25
:10D54000FEF716FFFDF734FD04F034FE4948046091
:10D55000F8BD4D480078002807D02C7003F076FC09
:10D5600001210846FCF722F8F8BD2878002803D1ED
:10D570004648416B0020884701202870FAF74AFF8F
:10D58000FFF7F4FBFEF7F4FEFDF712FD04F012FEC8
:10D590003F48404D0078002817D03878022801D342
:10D5A000FBF7EEFF28880028DED03C702C8005F0C9
:10D5B0003DFA374D2878810040181330C1B2294810
:10D5C0000C30FFF76DFA2C70F8BD308E01282888DA
:10D5D00005D03C2822D33878002810D01EE001283E
:10D5E000F2D320482C800079002803D0244804F08E
:10D5F00051FEF8BD0021234800F03EF9F8BD01209E
:10D60000387018482C800079002803D01C4804F09A
:10D6100041FE03E000211B4800F02EF928881E2857
:10D6200007D33878012804D1022038702C8003F009
:10D630003FFC3878022803D101210846FBF7B6FFEA
:10D64000308E29883C388842D8DC3878022800D1CE
:10D650005BE7F8BD00040050040000200039002002
:10D6600006000020F401002000000020200000201F
:10D6700018000020140000201C00002010000020D2
:10D68000243D002081CD000801000020044A01084B
:10D69000E102002012000020F8B5FCF745F9644CC7
:10D6A000A062644806F084FB002006F046FB0021DF
:10D6B0001F2006F0FBFA20625F48FBF7EBFEE081DB
:10D6C00064216170FF30913080B20121C903208252
:10D6D000884201D3401A20825748FBF7DBFEA08125
:10D6E000564F574E0AE05448FBF7D4FE80B2A08153
:10D6F000218A884202D3C919884206D300210F200B
:10D7000006F0D4FA05463042EDD06562680476D55D
:10D710006D1C74D08122D20100210F2006F0EDFB98
:10D720000021102006F0C2FAC1B221700022454843
:10D7300006F0F2FA43483E494378421C8B748078E5
:10D74000C8741179217550793E4D60756A7A202A26
:10D7500069D13D4B2A781B789A4264D1EA782271CC
:10D760002A796271EA79A271AA7AE27021756075EC
:10D77000294652000B313548F7F725FDE078420085
:10D780003248511932300B31F7F71DFD0020E0719E
:10D790002F480078002803D111202E49000208608C
:10D7A000A08AFAF7A3F82072607A28283BD22A4888
:10D7B00000260068E27825E071004B19DF7A69469F
:10D7C0000F701B7B4B700988814219D13046F9F7E5
:10D7D000C9FF1E49700032310A5A207A1B4B4100A2
:10D7E000DC335A52627950331A54627A90420BD128
:10D7F000521C62721A46A08AA03A505204E00DE010
:10D80000761CF6B29642D7D3E07886420BD1217AC5
:10D81000627A914207D1F9F7A5FF04E00F4A00218F
:10D820000F2006F06AFB06F06DF906F053F9F8BD1B
:10D83000D8020020B80B000030070020983A000002
:10D8400000D02724883D00208E000020183F0020B3
:10D85000F9010020140000208800002000902724F7
:10D8600000487047601000200048704740100020BA
:10D870000048704750100020034AD1611062012017
:10D880005070002070470000580100200048704789
:10D89000981000200249002248784A707047000022
:10D8A0005801002010B5074B04461A6A002A01D01F
:10D8B000D9699047182221460348F7F784FC0020D5
:10D8C00010BD0000580100208010002002490023F4
:10D8D0000A5C0B5410467047610100200249002386
:10D8E0000A5C0B54104670476401002010B5044ACE
:10D8F000536A002B01D0926A9847002010BD0000A7
:10D9000058010020034A012111540021D21C115456
:10D910000846704761010020034A0121115400218B
:10D92000D21E1154084670476401002010B500282B
:10D9300009D0064A01219170024680210448FEF771
:10D940008EFF002010BD0020C04310BD58010020F4
:10D95000981000200249002288788A7070470000E1
:10D96000580100200020704710B5192904D28A1EE2
:10D9700001460248F7F727FC002010BD6010002088
:10D9800010B5022902D20020C04310BD8C1E102CFD
:10D9900007D2014622460448F7F715FC0249002049
:10D9A0000855002010BD00004010002010B50229CD
:10D9B00002D20020C04310BD8C1E102C07D201469D
:10D9C00022460448F7F7FFFB0249002008550020D3
:10D9D00010BD0000501000200249002208780A7093
:10D9E000704700005801002070B5054C0546A2693B
:10D9F000002A01D0616990470020256170BD0000B8
:10DA000058010020FEE7000070B5114C15466180FA
:10DA10000A4601461E460F48F7F7D5FB25700E4D06
:10DA20006670286B80470B48007804280BD1A088CB
:10DA3000401CA08004F0C4FCFFF72EFE002204214D
:10DA40000648FBF772FB696B0020884770BD000039
:10DA50002A030020F0410020044A01080008005079
:10DA600010B5074C206B80470648162240890721D5
:10DA7000FF30D73003F048FA616B0020884710BDB3
:10DA8000044A0108C038002010B5074C206B8047BD
:10DA90000648162240890721FF30D73003F034FAB8
:10DAA000616B0020884710BD044A0108C03800207F
:10DAB00010B5034C206B8047616B0020884710BD78
:10DAC000044A010810B50648006B80470548162235
:10DAD00040890721FF30D73003F016FA10BD00004F
:10DAE000044A0108C038002070470000F8B5012141
:10DAF00049022748FBF714FB264E274D0024002837
:10DB000016D02878317801270843002803D1032054
:10DB1000F9F7F8FF2F7011273F02012149021C4835
:10DB2000FBF7FEFA002803D0F9F7F8FE032811D01E
:10DB3000AC706C702878002803D00020F9F7E2FF61
:10DB40002C70012149021248FBF7EAFA002800D1A3
:10DB50003470F8BDF9F71AFFFFF7E2F80F480460D8
:10DB6000FFF704F9FEF704FCFDF722FA04F022FBAC
:10DB70000B4800785A280B480760CED90A48046041
:10DB800006480460094804600120A870C5E7000049
:10DB900000040050A6010020F40100201400002021
:10DBA0000000002020000020180000201C000020A1
:10DBB00010B5012149020848FBF7B2FA07490028CD
:10DBC00002D00120087210BD0020087211200A78CE
:10DBD0000002086210BD0000000400500000002098
:10DBE0007CB506F041FB484D0020688147496980BB
:10DBF000EA88322A01D2642103E07D21C9008A42E9
:10DC000000D9E980298F0A2901D902212987E98EC3
:10DC1000432901D94321E986A98A3D4A914201D18C
:10DC20000A21A982A98C3B4A914200D9A884364C8A
:10DC3000394A4034218E4B230E46B43EDB009642D7
:10DC400002D3012938D02386E18FB439914200D321
:10DC5000E387698F782901D9782169872F4AE98F6D
:10DC6000D1702F4908702F48A98801602EA004F0B8
:10DC700045FF6888C2B2010A2FA004F03FFFE18D82
:10DC8000A08D00900191638D228DE18C32A004F073
:10DC900035FF218E38A004F031FFE18F3EA004F063
:10DCA0002DFFE08A01280AD0022813D0002802D1D3
:10DCB00041A004F023FF7CBD01212186C4E7618FD0
:10DCC000208F00900191E38EA28E618E40A004F01F
:10DCD00015FF7CBD49494AA00C4604F00FFF218C7A
:10DCE0004BA004F00BFF45494DA0223104F006FF84
:10DCF000424950A0423104F001FF404952A0623134
:10DD000004F0FCFE7CBD0000C038002001020000D1
:10DD1000FFFF0000102700005D0D0000F40100204F
:10DD20008E00002088000020C9E8B1B849443A209C
:10DD30002578202E0D0A0000B9CCBCFEB0E6B1BE9D
:10DD40003A20CCFAD0ACB6A8CEBB205625642E25FE
:10DD5000642E200D0A000000B7FECEF1C6F7B5D83C
:10DD6000D6B73A2025642E25642E25642E25643AE4
:10DD700025642E0D0A000000B5B1C7B0D4CBB6AFF4
:10DD8000CAB1475053B9A4D7F7BCE4B8F43A202538
:10DD900064202E0D0A000000B5B1C7B0B1BBB2F0CF
:10DDA000CAB1475053B9A4D7F7BCE4B8F43A202518
:10DDB00064202E0D0A000000B5A5B5E3B6A8CEBBC1
:10DDC000C4A3CABDC4A3CABD2E200D0A0000000012
:10DDD0005443505F5254434DC4A3CABD2CB7FECE2A
:10DDE000F1C6F7B5D8D6B73A2025642E25642E257E
:10DDF000642E25643A25642E0D0A0000403B002065
:10DE00004E74726970486F73743A25732E0D0A0050
:10DE10004E74726970506F72743A25642E0D0A0048
:10DE20004E74726970557365726E616D653A2573D3
:10DE30002E0D0A004E7472697050617373776F72A1
:10DE4000643A25732E0D0A004E74726970536F7513
:10DE50007263656E616D653A25732E0D0A000000D0
:10DE600000B5044980208862FF20F53006F0C2FA30
:10DE700000BD000000040050112302461B0200B543
:10DE800019020D489A4202D100F0C0F800BD8A4242
:10DE900002D100F057F809E0112A04D0824205D1DE
:10DEA00000F002F900BD00F009F800BD002AFCD125
:10DEB00000F07AF800BD00001111110000B500F06B
:10DEC0002FF800F02DF800F02BF800F029F800F002
:10DED00027F800F025F800F023F800F021F800F012
:10DEE0001FF800F01DF800F01BF800F019F800F022
:10DEF00017F800F015F800F013F800F011F800F032
:10DF0000B7F800F0B5F800F0B3F800F0B1F800F0A1
:10DF1000AFF800F0ADF800F0ABF800F0A9F800BDE4
:10DF200007488021816100BF00BF00BF00BF00BF64
:10DF300000BF816200BF00BF00BF00BF00BF7047CD
:10DF40000004005000B500F093F800F091F800F0E4
:10DF50008FF800F08DF800F08BF800F089F800F0F1
:10DF600087F800F085F8FFF7DBFFFFF7D9FFFFF731
:10DF7000D7FFFFF7D5FFFFF7D3FFFFF7D1FFFFF77D
:10DF8000CFFFFFF7CDFFFFF7CBFFFFF7C9FFFFF78D
:10DF9000C7FFFFF7C5FFFFF7C3FFFFF7C1FFFFF79D
:10DFA000BFFFFFF7BDFF00BD00B5FFF7B9FFFFF7EB
:10DFB000B7FFFFF7B5FFFFF7B3FFFFF7B1FFFFF7BD
:10DFC000AFFFFFF7ADFFFFF7ABFFFFF7A9FFFFF7CD
:10DFD000A7FFFFF7A5FFFFF7A3FFFFF7A1FFFFF7DD
:10DFE0009FFFFFF79DFFFFF79BFFFFF799FFFFF7ED
:10DFF00097FFFFF795FFFFF793FFFFF791FFFFF7FD
:10E000008FFFFFF78DFFFFF78BFF00BD00B5FFF718
:10E0100087FFFFF785FFFFF783FFFFF781FFFFF71C
:10E020007FFFFFF77DFFFFF77BFFFFF779FF00F032
:10E030001FF800F01DF800F01BF800F019F800F0D0
:10E0400017F800F015F800F013F800F011F8FFF7DA
:10E0500067FFFFF765FFFFF763FFFFF761FFFFF75C
:10E060005FFFFFF75DFFFFF75BFFFFF759FF00BDA5
:10E070000C488021816100BF00BF00BF00BF00BF0E
:10E0800000BF00BF00BF00BF00BF00BF00BF00BF98
:10E0900000BF00BF816200BF00BF00BF00BF00BF64
:10E0A000704700000004005000B5FFF7E1FFFFF7E4
:10E0B000DFFFFFF7DDFFFFF7DBFFFFF7D9FFFFF71C
:10E0C000D7FFFFF7D5FFFFF7D3FFFFF7D1FFFFF72C
:10E0D000CFFFFFF7CDFFFFF7CBFFFFF7C9FFFFF73C
:10E0E000C7FFFFF7C5FFFFF7C3FFFFF7C1FFFFF74C
:10E0F000BFFFFFF7BDFFFFF7BBFFFFF7B9FFFFF75C
:10E10000B7FFFFF7B5FFFFF7B3FF00BDF8B5044653
:10E1100000680025C168490619D4C16880221143EE
:10E12000C160FBF709F827460646203709E0FBF7F0
:10E1300003F8811B7D20C000814202D90420787041
:10E1400001252068C068400601D4002DEFD0284684
:10E15000F8BD70B5044600680025C168802291436F
:10E16000C16020688068800608D42046FBF7B8FEAE
:10E17000002803D00420203460700125284670BD9B
:10E180000120704710B500280DD00A4A0021CB00AD
:10E19000D458844209D89B189B68834205D9C8008B
:10E1A0008018007B10BD1F2010BD491CC9B2152965
:10E1B000EDD3FEE7744A010810B500F025FF0328EF
:10E1C00004D0042803D0052803D0002010BD02206D
:10E1D00010BD012010BD03207047000010B50E4C8B
:10E1E00020610E4800F0A0FF002001F007FA012096
:10E1F00001F07FF90021084601F054F804210020C5
:10E2000001F038FA064800231A46014601F08BF85F
:10E210000020A07010BD00003803002031E300088A
:10E22000FFFF0000F8B5012189023448FAF778FFB2
:10E23000012862D1324C0020A07000F0DBFE0546C0
:10E24000304800F0CDFEE80706D02069002803D052
:10E250000068002800D08047A80718D5FF2269462B
:10E26000294800F01DFF2848143800F0D5FE206929
:10E2700000280CD08668002E09D023480D231438BE
:10E280000C22C3568256684601781F48B04768067C
:10E2900006D52069002803D00069002800D08047F7
:10E2A00028060AD52069002807D08169002904D0F2
:10E2B000E843C005C017401C8847A80514D500F0E6
:10E2C000A3FE042804D000F09FFE052805D00BE033
:10E2D0002069002808D0406803E02069002803D0A6
:10E2E000C068002800D08047A80606D5206900280D
:10E2F00003D0C068002800D08047F8BD0008005057
:10E3000038030020FFFF00000443002070B50C46D6
:10E31000012500F0A5F8204601F0F2F8002000F0F9
:10E3200033F80120FAF7DCFC00F03CFA284670BD17
:10E3300001490120887070473803002070B500251E
:10E34000012000F08DF8002001F006F900240120E2
:10E35000FAF7C6FC00F0BAFEC007C00FA040641C6C
:10E360000543E4B2202CF2D300F01CFA284670BD1D
:10E3700010B500F03FFF10BD10B500F043FF10BD19
:10E3800010B500F0A3FE10BD10B5044600231A46D8
:10E390000649074800F0C7FF06484078002801D02A
:10E3A000054800E0A00101F0D7F810BD020200000E
:10E3B000FFFF000038030020FFFFFF0010B50446F8
:10E3C000074800231A46014600F0ADFF0548407893
:10E3D000002801D0044800E0A00101F0CFF810BDF2
:10E3E000FFFF000038030020FFFFFF0070B5054667
:10E3F0000C480C4600231A46014600F094FF00F03A
:10E4000049FE01460848012909D00472064801F076
:10E4100001F800222146284600F03CFF70BDC4737D
:10E42000F4E70000010200000444002010B501F0F0
:10E4300067F810BD10B5084B084A012808D0D079FC
:10E44000012804D119701172044800F0E3FF10BDD7
:10E450001970D173F8E7000038030020044400204D
:10E4600010B50A4C012805D0002001F02DF800203D
:10E47000607010BD012001F027F86178207881429A
:10E48000F7D0607000F004F810BD00003B030020DE
:10E4900070B504460B48047044700120FFF7E0FF9C
:10E4A0001D208001451C002C04D0342101F0B2F95C
:10E4B000442103E0142101F0ADF92421284601F0A4
:10E4C000A9F970BD3B030020FFB587B01646594936
:10E4D000199A119F149B4A701399002902D055492B
:10E4E0000B7002E05349FF220A70534C014620464C
:10E4F0002830254620350190002918D001296ED1F9
:10E50000002001F08DF81298C0B200F020FF012326
:10E510002B72F0B22876494A0899515C69760A99BB
:10E52000A976089900295CD001295CD05DE0002023
:10E5300001F076F8002028720B20E6622875089812
:10E54000FFF720FE687500202070F800608004202E
:10E550002071182060710020A071139901204140A2
:10E56000344FE171397821721599002900D0F220D9
:10E5700060720020A07201F041F8287A002800D0D3
:10E580000120FFF76DFF019800F0E8FE2A4800F037
:10E5900041FF2BA003C80490059104A801F047F89F
:10E5A000294801F0A7F83046F7F7A4F802460B46D1
:10E5B00000202649F6F7F4FF0322F7F769F804462E
:10E5C0000D461298F7F796F822462B46F6F780FF8D
:10E5D00000221F4BF6F77CFFF7F7AEF8F8600BB0A0
:10E5E000F0BD0B2E09D00C2E07D00021E976237048
:10E5F000052804D0062802D006E01946F6E70C2FBD
:10E6000002D20C20A08100E0A7811398094DA073CD
:10E610002878E07315982074189860740120FFF72B
:10E620001FFF019800F09AFE034800F0F3FE09482E
:10E63000E860D4E73803002004440020704A010851
:10E64000C194C10000000000FF0100000000F03F85
:10E6500000408F40FFFF000010B500F0A9FF10BD83
:10E66000FFB5454D83B00246294628312C460E9E03
:10E670000C9820340291002A02D0012A73D138E08C
:10E6800000272772E8620B2020751846FFF77AFDF5
:10E690006075059828632F70F00068800420287149
:10E6A00018206871AF710F9901204140E9711099EC
:10E6B000002902D0F221697200E06872A87200207D
:10E6C00000F09CFF207A002800D00120FFF7C8FE50
:10E6D000029800F043FE284800F09CFE27A103C9E1
:10E6E00000900191684600F0A2FF264801F002F870
:10E6F00039E001212172C2B2234F2276FF5C677696
:10E700000D9FA776002B02D0012B02D003E00B282F
:10E7100009D00C2807D00020E0762970052A04D003
:10E72000062A02D006E0E176F7E70C2E02D20C2092
:10E73000A88100E0AE810F98A87314480078E873B0
:10E740001098287413986874002000F057FF207AFE
:10E75000002800D00120FFF783FE029800F0FEFDA4
:10E76000054800F057FE049800F0F0FE07491498A1
:10E77000886007B0F0BD000004440020C194C100CF
:10E7800000000000FF010000704A0108380300206B
:10E7900010B50C4600F0B4FE204600F0D7FE00F0A5
:10E7A00061FF10BD08B5002069460090087804217B
:10E7B000084369460870009800F012FF0220FAF73B
:10E7C0008FFA08BD10B5002000F018FF10BD10B57D
:10E7D00000F072FD10BD0000F3B50246002057495D
:10E7E0008BB0002A56D0012A7DD10F462037787E83
:10E7F00030225043524A3C7E80180C22121BD20019
:10E800008018C21FF93A1046466C0846156C80897C
:10E81000F6F770FF00224B4BF6F7A8FD2A46334669
:10E82000F6F756FE07910690B87E8007800F001D10
:10E83000F6F760FF05910490F87E002800D00220D2
:10E84000201A8000F6F742FF07460C980391C0009B
:10E85000A100411A3948027C807B120189180128E5
:10E8600052D00020081A1C30F6F730FF3A46039BBE
:10E87000F6F796FE04F060FF059B049AF6F728FE73
:10E88000002207460C461346F6F788FF3ED238466C
:10E8900021463DE00C46C86AF6F72CFF06460F46B7
:10E8A0000C98F6F727FF0D46069061796088C90835
:10E8B0004018F6F71FFFE279002A1ED00022224BF3
:10E8C000F6F754FD2B46069AF6F750FD627A022AB7
:10E8D00016D000221346F6F749FD0322F6F7D8FEBC
:10E8E00032463B4600E027E0F6F75AFE0022174B7F
:10E8F000F6F7EEFD05F059FD1CE000221346DFE7B8
:10E90000002201239B07E6E71420ABE70020014625
:10E9100000220F4BF6F72AFD2A463346F6F7D8FDBC
:10E92000079B069AF6F722FD0A4A0B4BF6F71EFDE7
:10E9300005F046FBF6F700FF0DB0F0BD04440020E3
:10E9400050030020000011400000F03F00408F40C5
:10E95000000020402B8716D9CEF7EF3F10B500F00E
:10E9600059FF10BD10B500F05BFF10BD70B586B04B
:10E9700014216846F6F740FC01250F4EED030022F6
:10E9800029463046FAF7D1FB012000240190029479
:10E990006946009503943046FAF7E4FA03200190A3
:10E9A00002946946009503943046FAF7DBFA022098
:10E9B00004F026FF06B070BD0004005070B5054697
:10E9C00000F0F7F90024E443002819D1284600F0AC
:10E9D00027F80022C721284600F07AF900282846A7
:10E9E00002D000F00FF80BE000F00CF8284600F021
:10E9F000D1F9002804D1284600F078F9002800D089
:10EA0000204670BD28214843044910B540180189AB
:10EA100040680122FAF789FB10BD0000282400207D
:10EA200028214843044910B5401801894068002254
:10EA3000FAF77BFB10BD000028240020FFB581B051
:10EA40000C46019828214843174900254018406A80
:10EA50001F461646A0420DD9002E0BD0A1198142A7
:10EA600008D8B900114A00915158491E214201D1DC
:10EA7000032F03D30020C04305B0F0BD002C0ED1FE
:10EA8000B0420CD80198FFF799FF0AE061193A46A5
:10EA9000019800F0D5F80549009808584519B54285
:10EAA000F4D30020E8E7000028240020C048010833
:10EAB00038B504460322694600F09EF80025ED4370
:10EAC000002812D168460078FF2810D168464078A7
:10EAD000FF280CD168468078FF2808D103226946B8
:10EAE000204600F089F8002801D0284638BD684645
:10EAF0008278282044430A48012189052018152AD4
:10EB000005D0162A03D0172A04D0182A05D041624E
:10EB1000002038BD0121C905F9E701210906F6E702
:10EB200028240020FFB50E46C8B2FF2181B0013174
:10EB300000250C1A0A9F9C4200D91C46019800F03F
:10EB4000D5F8002842D1019800F033F900283DD1D2
:10EB50000198FFF765FF00220221019800F0B8F844
:10EB600000281FD13002010E0022019800F0B0F8F9
:10EB7000002817D13004010E0022019800F0A8F8F7
:10EB800000280FD1F1B20022019800F0A1F800286E
:10EB900008D10CE003980022415D019800F098F83C
:10EBA000002803D00198FFF72DFF0FE06D1CA54250
:10EBB000F0D30198FFF726FF019800F0EBF800284A
:10EBC00004D1019800F092F8002803D00020C0433F
:10EBD00005B0F0BD002F00D03C600020F8E7000039
:10EBE00010B528246043034CC90000194018426046
:10EBF000038110BD28240020F8B515460E460746AF
:10EC00000024FFF70DFF00229F21384600F060F836
:10EC1000002807D10DE03219FF21384600F058F8DE
:10EC2000002805D03846FFF7EDFE0020C043F8BDB0
:10EC3000641CAC42EFD33846FFF7E4FE0020F8BD79
:10EC4000F8B5064615469000204A1058401E8143EC
:10EC50000C46304600F0ADF80027FF43002833D1C2
:10EC60003046FFF7DDFE19480022001F415D3046A7
:10EC700000F02EF8002816D12002010E00223046A6
:10EC800000F026F800280ED12004010E00223046A4
:10EC900000F01EF8002806D1E1B20022304600F054
:10ECA00017F8002803D03046FFF7ACFE0CE03046E2
:10ECB000FFF7A8FE304600F06DF8002804D130467A
:10ECC00000F014F8002800D03846F8BDC04801080C
:10ECD00007B5114628225043034A0123105C01AABC
:10ECE00000F0A6F80EBD000028240020F8B5054667
:10ECF0000020694608706E462846FFF791FE002204
:10ED000005212846FFF7E4FF040005D13246FF2124
:10ED10002846FFF7DDFF04462846FFF773FE200074
:10ED200003D169460978C907E5D1F8BDFFB583B0BD
:10ED3000002001900D4603982821484314490027DC
:10ED40004018406AFF431C461646A84214D9002EBC
:10ED500012D0002C10D0411E2940401AA04201D2EE
:10ED6000044610E001A80090234632462946039845
:10ED7000FFF7D8FE002802D0384607B0F0BD019852
:10ED80002D183618241A002CECD10020F5E70000CD
:10ED90002824002070B50546FFF742FE002204211A
:10EDA0002846FFF795FF04462846FFF72BFE20462E
:10EDB00070BD70B50546FFF733FE002206212846D8
:10EDC000FFF786FF04462846FFF71CFE204670BD6D
:10EDD000F8B5044615480E46154613490068F6F77F
:10EDE00087F97D21C900484300906068C11FFD3943
:10EDF0000ED13346002280212046009500F038F8DD
:10EE000000280FD0606D2021084360650320F8BD05
:10EE10000098002806D0401E009020688068C043FB
:10EE20000006F5D50020F8BD00366E019C000020DC
:10EE300038B5144600291A460CD064256A4300925E
:10EE4000064A800010580A469BB22146FBF79AF901
:10EE5000002038BD214600F067F838BDB40100201D
:10EE6000024A80001150002070470000B4010020C9
:10EE7000FFB581B01E4604460A9DFAF75DF9401BB6
:10EE8000351AFAF759F90746264800684001000D7F
:10EE9000684339E0701C38D0FAF74EF9C01BA8421D
:10EEA00005D2002D03D0009800282BD02BE020683D
:10EEB0004168E022914341606068C11FFD390CD177
:10EEC0000121A068C903884202D04911884204D1B7
:10EED000206801684022914301600120A16A40033B
:10EEE000814207D121680A6882430A6021680A6862
:10EEF00002430A6001204034607400202074032023
:10EF000005B0F0BD0025401E009020688168029881
:10EF1000884305D0002103988142BBD10020EFE750
:10EF20000121F8E79C00002010B56423534394B2FC
:10EF3000034A800010582246FBF774F8002010BDE9
:10EF4000B40100207047704770470000174908B5AA
:10EF5000884204D9E12168460170E9211EE0144984
:10EF6000884204D9D72168460170D82116E011499A
:10EF7000884204D9C12168460170C5210EE00E49BE
:10EF8000884204D9752168460170812106E00B4949
:10EF9000884204D96B21684601706F2141700222BA
:10EFA0006946982000F010FC08BD000000E9A43577
:10EFB00080F8A9328044E52D000B6B1B40FC5419EE
:10EFC00010B506484078002801D0062803D100F08B
:10EFD000B9FBFFF7B9FF00F0A7FB10BDE00300206D
:10EFE00008B5020A69460A7048700222104600F00D
:10EFF000EBFB08BD08B502226946122000F0D2F8EA
:10F000006846008840BA08BD014840787047000053
:10F01000E00300200220704738B504460322694609
:10F02000142000F0BFF81A4988782070002808D012
:10F03000012816D014212046F6F7DEF80F202070A4
:10F0400038BD6846007820716846407840424010DC
:10F05000A071684680784042401060710020A06036
:10F0600038BD6846007840424010207368464078BA
:10F07000802801D2800802E0FF38013880106073D8
:10F080006846807840424010A0734868206138BDCF
:10F09000E00300200148807870470000E003002072
:10F0A000F8B50C460646002069460870154620460D
:10F0B00000F018F82278AA4201D90120F8BD68466C
:10F0C0003146007800F042F80020F8BD08B5012272
:10F0D0006946152000F066F8684600784042401006
:10F0E00040B208BD38B50D460446022269461320D9
:10F0F00000F058F80A488078012809D1094800F042
:10F1000079F8C00904D00748801E00F073F801E0C8
:10F1100068460078207068464078287038BD000046
:10F12000E00300200407000010B500F099F800F09B
:10F1300009FB002000F062FA012000F0EDF802491E
:10F140000120487010BD0000E0030020F8B515460E
:10F150000E460446FFF734FF00F08CFB104F0022F0
:10F1600004213846F9F7E1FF1E2001F051FE204648
:10F1700001F04EFE002001F04BFE002405E00020CF
:10F1800001F046FE3055641CA4B2AC42F7D3012214
:10F1900004213846F9F7C9FF00F0C6FAF8BD0000AF
:10F1A00000080050F8B515460E460446FFF708FF64
:10F1B00000F060FB0E4F002204213846F9F7B5FF3E
:10F1C000204601F025FE002001F022FE002405E08B
:10F1D000002001F01DFE3055641CA4B2AC42F7D3F0
:10F1E000012204213846F9F7A0FF00F09DFAF8BD8E
:10F1F0000008005008B50122694600F003F868468F
:10F20000007808BDF8B515460E460446FFF7D8FE4F
:10F2100000F030FB114F002204213846F9F785FF3A
:10F220001D2001F0F5FD200A01F0F2FDE0B201F031
:10F23000EFFD002001F0ECFD002405E0002001F0CE
:10F24000E7FD3055641CA4B2AC42F7D3012204217F
:10F250003846F9F76AFF00F067FAF8BD0008005079
:10F2600010B50A20F9F73CFD094C00220821204680
:10F27000F9F75BFF7D200001F8F76FFC0122082100
:10F280002046F9F752FF0A20F9F72AFD10BD0000C9
:10F290000008005010B5144600F024F9204600F094
:10F2A000CFF910BD08B56A46107051700222694648
:10F2B0008F2000F089FA08BD10B500221146C52044
:10F2C00000F082FA01490720487010BDE0030020D9
:10F2D00008B5020A69460A70487004488078002818
:10F2E00003D10222024800F09BFA08BDE00300208F
:10F2F000BE06000008B5020A69460A704870044854
:10F300008078002803D10222024800F089FA08BD63
:10F31000E0030020BC06000001B5012269469D20E3
:10F3200000F052FA08BD7CB5050A6C462570607085
:10F33000080AA070E170100A20716271180AA071A9
:10F340000822E3716946104600F03EFA7CBD01B523
:10F3500001226946A02000F037FA08BD7CB50446BA
:10F36000002000900190224920788978884201D0BD
:10F3700000F0AAF82078002810D001280DD1217CB7
:10F3800068460170617C4170A17C8170E17CC17034
:10F39000042269468B2000F017FA7CBD08256068BE
:10F3A000F6F7A8F902460B4600201249F6F7F8F8DE
:10F3B0000522F6F76DF9F6F7BFF9020C69460A70F7
:10F3C000020A4A708870207BC870607B0871A06850
:10F3D000F6F790F90022084BF6F7E2F8F6F7ACF9E9
:10F3E000020C69464A71020A8A71C8712A46D1E73D
:10F3F000E003002080847E418084EE3F38B56C4677
:10F4000020706170A270E37004226946952000F0BC
:10F41000DBF938BD3EB50446002000900190029013
:10F42000244920788978884201D000F04DF820786E
:10F43000002814D0012811D1A18906220B0A6846A0
:10F4400003704170A17B8170E17BC170217C0171EF
:10F45000617C417169468C2000F0B6F93EBD607A4E
:10F46000F12802D0F22808D00EE01348FFF742FF3F
:10F470001248FFF72DFF022006E01148FFF73AFF80
:10F480001048FFF725FF0620618809220B0A69460C
:10F490000B70A3784B7023798B706379CB70A37951
:10F4A0000B71E3794B71237A8B71C871A07A087262
:10F4B000D0E70000E0030020FFFF0000058000000F
:10F4C0000F1D00002110000001B5684604490078B6
:10F4D0008870012269468A2000F076F908BD000094
:10F4E000E00300200A4610B50146002000F044F970
:10F4F00010BD01B501226946962000F065F908BDEE
:10F5000038B5104C05462078002804D12846FFF76E
:10F510001DFD012020702846F6F7ECF800220A4B6A
:10F52000F6F73EF8F6F708F9020E69460A70020C83
:10F530004A70020A8A70C8700422862000F044F9DA
:10F5400038BD0000E00300208084EE3F10B50221AA
:10F5500000F090F810BD000008B5074A0521517071
:10F56000020C69460A70020A4A70887003228220DF
:10F5700000F02AF908BD0000E003002038B5044679
:10F580000949052048709621084800F043F9210CEC
:10F5900068460170210A4170847003226946822006
:10F5A00000F012F938BD0000E0030020AC080000B4
:10F5B0001CB5030C6A461370030A53709070080C54
:10F5C000D070080A1071517106226946942000F02B
:10F5D000FBF80249062048701CBD0000E003002033
:10F5E00001B5FFF7B0FC01226946842000F0ECF879
:10F5F00001490020487008BDE003002001B5012248
:10F600006946802000F0E0F8684601780348002948
:10F6100002D00221417008BD0121FBE7E003002078
:10F6200001B5012269469F2000F0CEF808BD0146D1
:10F6300010B51B200822800100F0F2F8002010BD58
:10F6400008B5074A04215170020C69460A70020A83
:10F650004A7088700322832000F0B6F808BD0000CD
:10F66000E003002010B500221146D12000F0ACF8D4
:10F6700010BD0000F8B504460D460020FFF7CAFC97
:10F6800002271B4EFF43012809D001230022072136
:10F690000420FFF7B3FE162C19DD16241AE00F2CF8
:10F6A00009D001231A4600210420FFF7A7FE0E2CE3
:10F6B00008DB0E2409E001231A4600210620FFF78B
:10F6C0009DFEF6E7BC4200DA3C46182103E0BC424E
:10F6D00000DA3C463821304600F09CF86846047059
:10F6E0004570022269468E2000F06EF8F8BD0000D9
:10F6F000E708000070B504460A488078002810D159
:10F70000D725ED002846FFF775FD4008E1054000CC
:10F71000C90F0143284600F07DF8E1B2681C00F0F3
:10F7200079F870BDE003002070B50124044DE402B7
:10F7300021462846F9F7F4FC0128F9D070BD0000F5
:10F740000008005010B500F095F80A4C0022042182
:10F750002046F9F7EAFCC02001F05AFB002001F036
:10F7600057FB012204212046F9F7DFFCFFF7DCFFFD
:10F7700010BD000000080050F8B515460E460446BE
:10F78000FFF71EFC00F076F80E4F002204213846E9
:10F79000F9F7CBFC0E2001F03BFB204601F038FBD3
:10F7A000002404E0305D01F033FB641CA4B2AC42E1
:10F7B000F8D3012204213846F9F7B7FCFFF7B4FF6C
:10F7C000F8BD000000080050F8B515460E46074683
:10F7D000FFF7F6FB00F04EF8002204210C48F9F781
:10F7E000A4FC384601F014FB002404E0305D01F075
:10F7F0000FFB641CA4B2AC42F8D3012204210448DC
:10F80000F9F793FC842F01D0FFF78EFFF8BD0000BD
:10F810000008005013B5012201A900F001F81CBD39
:10F82000F8B515460E460446FFF7CAFB00F022F86D
:10F830000F4F002204213846F9F777FC0D2001F024
:10F84000E7FA200A01F0E4FAE0B201F0E1FA00245C
:10F8500004E0305D01F0DCFA641CA4B2AC42F8D3E1
:10F86000012204213846F9F760FCFFF75DFFF8BD7F
:10F870000008005010B50524240710212046F9F790
:10F880004FFC002807D1012210212046F9F74DFC3A
:10F8900001A003F033F910BD7577625F63735F6594
:10F8A00072726F720D0A0000F8B5044600206A46B5
:10F8B00010801A4D55222A70AA226A700322AA705B
:10F8C000661DEE702A716971154A49008918AC717C
:10F8D0002246E81DF5F777FC002007E029186A4664
:10F8E0008978128889186A461180401CB042F5DB7D
:10F8F000611DA81CF7F7ECFF014668460180291935
:10F900000078C8716846407808727D232246DB0083
:10F91000093202490348FBF74EF9F8BD7041002057
:10F92000C03800201C080020F8B516460F460446D3
:10F930001D46012240210A48F9F7F7FBFEF790FA2D
:10F940002846FEF799FA3046FEF796FA3846FEF753
:10F9500093FA2046FEF790FAFEF782FAF8BD00000F
:10F960000004005010B5002240210248F9F7DDFBE9
:10F9700010BD00000004005010B5022813D0FCF7A1
:10F9800057FC00280DD0FCF753FC0B24E4010019B0
:10F990000069002805D0FCF74BFC0019016904A0A0
:10F9A0008847002010BD4868FDF7C0FFF9E7000058
:10F9B0004552524F520D0A000020704710B50220E8
:10F9C000FDF7A0FFFCF734FC00280DD0FCF730FC5D
:10F9D0000B24E40100190069002805D0FCF728FC7D
:10F9E0000019016901A08847002010BD4F4B0D0A86
:10F9F0000000000070B50B24E4010D4602280FD072
:10FA0000FCF716FC00280BD0FCF712FC001900696B
:10FA1000002805D0FCF70CFC001901692AA08847D2
:10FA20006868F5F758FC002815D0012826D0022870
:10FA300036D0FCF7FDFB00280BD0FCF7F9FB0019D2
:10FA40000069002805D0FCF7F3FB001901691FA02D
:10FA50008847002070BD0020F8F754F8FCF7E8FB59
:10FA60000028F6D0FCF7E4FB001900690028F0D06C
:10FA7000FCF7DEFB0019016916A0E9E7FCF7D8FBEB
:10FA800000280BD0FCF7D4FB00190069002805D032
:10FA9000FCF7CEFB001901690EA08847012010E099
:10FAA000FCF7C6FB00280BD0FCF7C2FB001900696D
:10FAB000002805D0FCF7BCFB0019016905A08847A8
:10FAC0000220F8F71FF8C4E7417267204552524FF1
:10FAD000520D0A004F4B0D0A0000000070B5486837
:10FAE000F5F7F9FB7D210446C900F5F701FB050395
:10FAF00064212046F5F7FCFA0A21F5F7F9FA080225
:10FB00002D180A212046F5F7F3FA0C460A21F5F7DD
:10FB1000EFFA0801281800190D4980B288800D49B4
:10FB2000086004F047FCFCF783FB00280DD0FCF7CD
:10FB30007FFB0B24E40100190069002805D0FCF7C5
:10FB400077FB0019016904A08847002070BD000000
:10FB5000C0380020880000204F4B0D0A0000000034
:10FB600010B5022814DAFCF763FB00280DD0FCF76F
:10FB70005FFB0B24E40100190069002805D0FCF7A5
:10FB800057FB0019016903A088470020C04310BD3E
:10FB9000002010BD64656275675F6F666620666CE5
:10FBA00061670D0A0000000010B5022814DAFCF7A6
:10FBB0003FFB00280DD0FCF73BFB0B24E4010019B0
:10FBC0000069002805D0FCF733FB0019016903A088
:10FBD00088470020C04310BD002010BD64656275D9
:10FBE000675F6F6E20666C61670D0A0070B50B254C
:10FBF000ED010C4602280FD0FCF71AFB00280BD0B1
:10FC0000FCF716FB40190069002805D0FCF710FB33
:10FC10004019016911A088476068F5F75CFB04464C
:10FC200000021149000C48828C8204F0C3FB21467B
:10FC3000022002F0ABFCFCF7FBFA00280BD0FCF72B
:10FC4000F7FA40190069002805D0FCF7F1FA4019CD
:10FC5000016906A08847002070BD0000417267203E
:10FC60004552524F520D0A00003900204F4B0D0AE9
:10FC70000000000070B5FCF7DBFA0B24E40100285B
:10FC80000CD0FCF7D5FA00190069002806D0FCF763
:10FC9000CFFA0019026920A122A09047FCF7C8FA08
:10FCA00000280FD0FCF7C4FA00190069002809D019
:10FCB000FDF7DAFD0546FCF7BBFA00190269294693
:10FCC0001EA09047FCF7B4FA00280FD0FCF7B0FA5A
:10FCD00000190069002809D0FDF7C2FD0546FCF7B0
:10FCE000A7FA0019026929461AA09047FCF7A0FA62
:10FCF00000280FD0FCF79CFA00190069002809D0F1
:10FD0000FDF7B6FD0546FCF793FA0019026929468E
:10FD100016A09047002070BD563230323130353158
:10FD20003030300056657273696F6E3A20202020A3
:10FD3000202020202025730D0A000000494D454950
:10FD40003A20202020202020202020202025730D54
:10FD50000A000000434349443A202020202020206C
:10FD6000202020202025730D0A000000494D534912
:10FD70003A20202020202020202020202025730D24
:10FD80000A00000010B527210248FCF7C7F900203F
:10FD900010BD0000CC48010810B50B24E401022876
:10FDA00012D0FCF745FA00280BD0FCF741FA0019F5
:10FDB0000069002805D0FCF73BFA001901690BA087
:10FDC00088470020C04310BDFCF732FA00280BD052
:10FDD000FCF72EFA00190069002805D0FCF728FA74
:10FDE0000019016906A08847002010BD757361677E
:10FDF000653A206C6F6720737472696E670D0A0034
:10FE00004F4B0D0A0000000010B5FCF711FA002856
:10FE10000DD0FCF70DFA0B24E4010019006900284D
:10FE200005D0FCF705FA0019016902A088470020F7
:10FE300010BD00004F4B0D0A0000000010B5032854
:10FE400014D0FCF7F5F900280DD0FCF7F1F90B24DC
:10FE5000E40100190069002805D0FCF7E9F9001950
:10FE6000016903A088470020C04310BD002010BDD9
:10FE700075736167653A206C6F675F7072696E7445
:10FE8000206173635B302D315D20636E740D0A0059
:10FE9000002070477047000010B50220FDF73CFDC0
:10FEA000FCF7C6F900280DD0FCF7C2F90B24E401D9
:10FEB00000190069002805D0FCF7BAF9001901699A
:10FEC00001A08847002010BD4F4B0D0A0000000024
:10FED00010B50020FDF716FDFCF7AAF900280DD09B
:10FEE000FCF7A6F90B24E40100190069002805D0ED
:10FEF000FCF79EF90019016901A08847002010BD98
:10FF00004F4B0D0A0000000010B50020FDF704FD66
:10FF1000FCF78EF900280DD0FCF78AF90B24E401D8
:10FF200000190069002805D0FCF782F90019016961
:10FF300001A08847002010BD4F4B0D0A00000000B3
:10FF400010B50B24E401022812D0FCF771F9002847
:10FF50000BD0FCF76DF900190069002805D0FCF7FB
:10FF600067F9001901690BA088470020C04310BD44
:10FF7000FCF75EF900280BD0FCF75AF9001900696C
:10FF8000002805D0FCF754F90019016908A088473A
:10FF9000002010BD75736167653A207274635F73EA
:10FFA00065745F616C61726D207365630D0A00009A
:10FFB0004F4B0D0A000000000020704710B50728C5
:10FFC00014D0FCF735F900280DD0FCF731F90B24DB
:10FFD000E40100190069002805D0FCF729F900198F
:10FFE000016903A088470020C04310BD002010BD58
:10FFF00075736167653A207274635F736574207905
:020000040801F1
:10000000797979206D6D206464206868206D6D2099
:1000100073730D0A0000000010B5F9F7B1FA002063
:1000200010BD000070B50B24E4010E4603280FD06C
:10003000FCF7FEF800280BD0FCF7FAF8001900696D
:10004000002805D0FCF7F4F80019016920A08847C2
:100050007068F5F740F90546B068F5F73CF90146D8
:10006000681E132821D832291FDC002D1DDD1B4EF0
:100070007D203586C000F5F751F831464039C880FB
:1000800004F098F9FCF7D4F800280BD0FCF7D0F86E
:1000900000190069002805D0FCF7CAF800190169A9
:1000A0000FA08847012030840FE0FCF7C1F800283A
:1000B0000BD0FCF7BDF800190069002805D0FCF74B
:1000C000B7F80019016902A08847002070BD000040
:1000D000417267204552524F520D0A0000390020EC
:1000E0004F4B0D0A0000000070B50B24E4010D46D3
:1000F00002280FD0FCF79CF800280BD0FCF798F8EA
:1001000000190069002805D0FCF792F80019016970
:100110000DA088476868F5F7DEF80E49488304F0BB
:1001200049F9FCF785F800280BD0FCF781F8001995
:100130000069002805D0FCF77BF80019016906A0CA
:100140008847002070BD0000417267204552524F21
:10015000520D0A00003900204F4B0D0A000000002C
:1001600070B50B25ED010C46062812DAFCF760F895
:1001700000280BD0FCF75CF840190069002805D076
:10018000FCF756F8401901691DA088470020C043BC
:1001900070BD1E481CA220210646636802F0BEFC0A
:1001A000A068FCF7ABFB3084184817A2202122304E
:1001B000E36802F0B3FC154813A220214230236902
:1001C00002F0ACFC114810A220216230636902F0F9
:1001D000A5FC04F0EFF8FCF72BF800280BD0FCF797
:1001E00027F840190069002805D0FCF721F84019CC
:1001F000016907A08847084801210184002070BDDB
:100200004552524F520D0A0025730000403B00201A
:100210004F4B0D0A000000000039002070B50B257F
:10022000ED010C46052812DAFCF702F800280BD085
:10023000FBF7FEFF40190069002805D0FBF7F8FF27
:10024000401901691BA088470020C04370BD1BA254
:1002500020211B48636802F061FC194817A2202185
:100260002030A36802F05AFC154814A22021403027
:10027000E36802F053FC124810A220216030236989
:1002800002F04CFC04F096F8FBF7D2FF00280BD0EC
:10029000FBF7CEFF40190069002805D0FBF7C8FF27
:1002A0004019016907A088470848012101840020FE
:1002B00070BD00004552524F520D0A0025730000D8
:1002C000C03A00204F4B0D0A00000000003900200A
:1002D000F8B50B26F6010D46022812DAFBF7A8FF47
:1002E00000280BD0FBF7A4FF80190069002805D077
:1002F000FBF79EFF8019016914A088470020C043C6
:10030000F8BD69466868FCF76DF96868FCF7F6FAAD
:10031000104CE18A884203D06868FCF7EFFAE0826B
:1003200004F048F8FBF784FF00280BD0FBF780FFB0
:1003300080190069002805D0FBF77AFF8019016950
:1003400005A08847012020840020F8BD4552524F67
:10035000520D0A00003900204F4B0D0A000000002A
:10036000F8B50B26F6010D46032812DAFBF760FFFD
:1003700000280BD0FBF75CFF80190069002805D02E
:10038000FBF756FF8019016923A088470020C0436E
:10039000F8BD69466868FCF725F9214C6846007885
:1003A000618E88420ED169464978A28E914209D168
:1003B00069468978E28E914204D16946C978228FD4
:1003C000914209D0608668464078A0866846807869
:1003D000E0866846C0782087A868FCF78FFA618FAE
:1003E000884203D0A868FCF789FA608703F0E2FF2F
:1003F000FBF71EFF00280BD0FBF71AFF80190069DE
:10040000002805D0FBF714FF8019016905A0884773
:10041000012020840020F8BD4552524F520D0A00A1
:10042000003900204F4B0D0A00000000F8B50B26E4
:10043000F6010D46032812DAFBF7FAFE00280BD06E
:10044000FBF7F6FE80190069002805D0FBF7F0FEE7
:100450008019016923A088470020C043F8BD694680
:100460006868FCF7BFF8214C68460078E18C884248
:100470000ED169464978228D914209D16946897821
:10048000628D914204D16946C978A28D914209D00A
:10049000E0846846407820856846807860856846B4
:1004A000C078A085A868FCF729FAE18D884203D0BE
:1004B000A868FCF723FAE08503F07CFFFBF7B8FEA1
:1004C00000280BD0FBF7B4FE80190069002805D086
:1004D000FBF7AEFE8019016905A088470120208442
:1004E0000020F8BD4552524F520D0A00003900203D
:1004F0004F4B0D0A00000000F8B50B26F6010D4623
:10050000022812DAFBF794FE00280BD0FBF790FECE
:1005100080190069002805D0FBF78AFE801901695F
:1005200014A088470020C043F8BD69466868FCF7FE
:1005300059F86868FCF7E2F9104C218B884203D027
:100540006868FCF7DBF9208303F034FFFBF770FEEB
:1005500000280BD0FBF76CFE80190069002805D03D
:10056000FBF766FE8019016905A0884701202084F9
:100570000020F8BD4552524F520D0A0000390020AC
:100580004F4B0D0A0000000070B54868F4F7A3FE59
:100590000C4CE08703F00EFFFBF74AFE00280DD05D
:1005A000FBF746FE0B25ED0140190069002805D038
:1005B000FBF73EFE4019016903A088470120208413
:1005C000002070BD003900204F4B0D0A00000000D4
:1005D00070B54868F4F77FFE0C4C208603F0EAFE05
:1005E000FBF726FE00280DD0FBF722FE0B25ED01C0
:1005F00040190069002805D0FBF71AFE401901696F
:1006000003A0884701202084002070BD003900200D
:100610004F4B0D0A000000000020704710B502A0EB
:10062000FAF71CFE10BD00004576656E743A25751C
:100630000D0A000070B50B24E4010D4602280FD00E
:10064000FBF7F6FD00280BD0FBF7F2FD001900695F
:10065000002805D0FBF7ECFD0019016915A08847BB
:100660006868F4F738FE00F071F9002811D0FBF744
:10067000DFFD00280BD0FBF7DBFD00190069002827
:1006800005D0FBF7D5FD001901690BA088470020B4
:1006900070BDFBF7CDFD0028F9D0FBF7C9FD0019AF
:1006A00000690028F3D0FBF7C3FD0019016904A01D
:1006B000ECE70000417267204552524F520D0A008C
:1006C0004F4B0D0A00000000F8B50B24E4010D4665
:1006D00004280FD0FBF7ACFD00280BD0FBF7A8FDDA
:1006E00000190069002805D0FBF7A2FD0019016977
:1006F00019A088476868F4F7EEFD0746AE68E86819
:10070000F4F7E9FD82B23146384600F059F9002885
:1007100011D0FBF78DFD00280BD0FBF789FD0019E8
:100720000069002805D0FBF783FD001901690BA0C3
:1007300088470020F8BDFBF77BFD0028F9D0FBF7C8
:1007400077FD001900690028F3D0FBF771FD00194F
:10075000016904A0ECE70000417267204552524F46
:10076000520D0A004F4B0D0A0000000038B5002062
:10077000034600901D4A0121684600F041F90B2410
:10078000E401002811D0FBF753FD00280BD0FBF744
:100790004FFD00190069002805D0FBF749FD00193D
:1007A000016913A08847002038BDFBF741FD0028F0
:1007B0000CD0FBF73DFD00190069002806D0FBF7BF
:1007C00037FD001902690CA000999047FBF730FD36
:1007D0000028E8D0FBF72CFD001900690028E2D0C2
:1007E000FBF726FD0019016906A0DBE71D060108DD
:1007F0004552524F520D0A00536F636B49443A25DC
:10080000750D0A004F4B0D0A0000000070B50B2457
:10081000E4010D4603280FD0FBF70AFD00280BD09A
:10082000FBF706FD00190069002805D0FBF700FD65
:100830000019016919A088476868F4F74CFDAD6894
:1008400006462846F4F70DFD02462946304600F0DC
:1008500093FA002811D0FBF7EBFC00280BD0FBF734
:10086000E7FC00190069002805D0FBF7E1FC00193E
:1008700001690BA08847002070BDFBF7D9FC002858
:10088000F9D0FBF7D5FC001900690028F3D0FBF77D
:10089000CFFC0019016904A0ECE700004172672059
:1008A0004552524F520D0A004F4B0D0A00000000F6
:1008B000002070470020704738B51448694608800A
:1008C000FBF7B6FC00280DD0FBF7B2FC0B24E401CB
:1008D00000190069002805D0FBF7AAFC001901697E
:1008E0000BA0884711240023240302222146184626
:1008F000FEF7A4F802236A4621460020FEF716FA06
:10090000064801210184002038BD0000AAAA000089
:10091000757064617465204F4B0D0A00003900202A
:100920000748418F0748C289914205D20649097894
:10093000002901D0012100E0002141707047000032
:10094000C038002000000020F701002009490A4AB1
:100950004143891803280AD2002908D008780028C2
:1009600003D0012801D00520087000207047002026
:10097000C0437047C404000018110020F8B50024DB
:100980000D4D264601270D48604340190178032983
:1009900003D0042901D0062908D186700770836826
:1009A000002B03D0C268022120469847641C032C08
:1009B000E9DB0020F8BD000018110020C40400008D
:1009C00070B515460B4A0C4B4243D41803280DD280
:1009D000002C0BD00B46204608A22A211030FBF732
:1009E0003EFF658703202070002070BD0020C043BB
:1009F00070BD0000C4040000181100202573000021
:100A0000FFB51F4881B01F460E4600251D496943AA
:100A10000C1802D02178002906D06D1C032DF5DBBF
:100A20000020C04305B0F0BD16492046FBF79AFDF3
:100A300065606670022020700398E7601023A06054
:100A40005F01214620463A46C4313C30FCF702F8AB
:100A5000B1208000012E0AD02118204610233A46EA
:100A60006C30FBF7F7FF019805600020DAE72118EA
:100A7000204601233A46B030FAF7F3FAF3E70000D4
:100A800018110020C40400000649074A4143891890
:100A9000032804D2002902D00020087070470020EB
:100AA000C0437047C404000018110020032805DA71
:100AB00003494843034940181030704702A070476B
:100AC000C40400001811002000000000032805DA0B
:100AD0000349484303494018408F7047002070473E
:100AE000C404000018110020032805DA0349484314
:100AF000034940183C30704700207047C404000090
:100B000018110020032804DA034948430349085C0C
:100B10007047002070470000C40400001811002036
:100B2000032805DA034948430349401840787047D1
:100B300000207047C4040000181100200C490D4A21
:100B400041438918002210B5D24303280ED2002950
:100B50000CD00B78042B09D001220A708B68002B73
:100B600002D0CA6802219847002010BD104610BD6F
:100B7000C4040000181100200A490B4A414310B573
:100B8000891803280BD2002909D007220A708B6824
:100B9000002B02D0CA6800219847002010BD002019
:100BA000C04310BDC40400001811002070B50546F4
:100BB0001A481B4968434418032D25D2002C23D022
:100BC0000620207010235E01214620463246C431A3
:100BD0003C30FBF73FFF1149114BB120694362786C
:100BE0008000C9180918012A11D020461023324666
:100BF0006C30FBF72FFFA368002B03D001212846A0
:100C0000E2689847002070BD0020C04370BD2046B8
:100C100001233246B030FAF724FAECE7C4040000AE
:100C20001811002009490A4A414310B589180328C0
:100C300009D2002907D08B68002B02D0CA68032193
:100C40009847002010BD0020C04310BDC404000020
:100C500018110020FFB5014617461F481F4A0024FF
:100C60004843E443801881B01E4603291AD2002865
:100C700018D0002E16D04178012916D06C30009083
:100C8000FBF79CFE05000DD06A68BA4206D22968BF
:100C90000298F4F798FA68680024306029460098B2
:100CA000FBF760FE204605B0F0BD0024B0302546BD
:100CB00000900BE0029801190098FAF7F7F9002864
:100CC00002D000203560EEE7641C6D1CBC42F1D3FD
:100CD00000243560E6E70000C4040000181100207D
:100CE000F7B505461A481B49684300244018671E9B
:100CF0001646032D1FD200281DD04178012910D09F
:100D00006C3007461146FBF777FE040019D03246D7
:100D100020680199F4F757FA38462146FBF738FE68
:100D200013E00546B03509E0019801192846FAF7A5
:100D30007DF9002801D03846FEBD641CB442F3D3CF
:100D400003E0294604A0FAF789FA0020FEBD00005E
:100D5000C404000018110020536F636B65745B2599
:100D6000755D205265637620427566666572204621
:100D7000756C6C0D0A000000F7B505461348144960
:100D8000684300274018FF4382B01646032D16D251
:100D9000002814D0002E12D03C3011460090FBF7F2
:100DA0002BFE04000DD0324620680399F4F70BFAAD
:100DB00021460098FBF7ECFD002005B0F0BD384659
:100DC000FBE7294603A0FAF749FAF8E7C404000054
:100DD00018110020736F636B65745B25645D20736D
:100DE000656E64206275662066756C6C0D0A000085
:100DF000032805DA044A5043044A1154002070477E
:100E00000020C04370470000C404000018110020F7
:100E100001B582B00021684601717D20C0000090BC
:100E2000012301AA02A90348F9F7ACF96846007941
:100E30000EBD000084070020034A1168382389B2E0
:100E400099430143116070470030014000B51348D9
:100E500085B0C17900291ED10121C171F7F7EAFAE5
:100E60000F48F9F79DFB14216846F4F7C5F91020E7
:100E700000901120019000200290039069460948DB
:100E8000F8F770F80121002289020748F8F74DF9B8
:100E90000648C06A804705B000BD0000F40100208C
:100EA000A40800200008005000040050044A010873
:100EB00000B5114885B0017A00291BD101210172CA
:100EC000F7F7B8FA0D48F9F76BFB14216846F4F709
:100ED00093F91020009011200190002002900390BF
:100EE00069460748F8F73EF80121002289020548C3
:100EF000F8F71BF905B000BDF4010020A40800209C
:100F00000008005000040050F7B51A4D0446286B45
:100F10008AB00E468047184920464843E96888470A
:100F200016480121C4800024154808900794082021
:100F300006940290059401910C98039400960494F1
:100F40000223EF6941B222460120B84708200694E7
:100F500007940894099405940294039404940094CB
:100F600001900123AC69324602211846A0470DB01A
:100F7000F0BD0000044A010840420F002A0300208F
:100F8000B80B000010B5FBF76DFAF8F719F910BDB2
:100F900010B59AB034216846F4F72EF9142115A83B
:100FA000F4F72AF920210DA8F4F726F9244801685E
:100FB0000324E402A143C21489180160F8F7EEFA91
:100FC00020480169A14301610E200090FF200130FB
:100FD00002901020049002200990400401210B90FF
:100FE0000001059100240C9003910A946846F8F7DB
:100FF000F7FC002801D072B6FEE70F201590032001
:101000001690179418940121199415A8F8F7BEFBAF
:10101000002801D072B6FEE7A3200D900120400405
:101020000E9003200F948004149010940DA8F8F7EC
:10103000EFFA002801D072B6FEE71AB010BD00002A
:10104000007000404010024002490148886070472B
:101050000050000800ED00E0F0B502680124A4078C
:10106000144D154E154FA04205D0A84203D0B042F2
:1010700001D0B84204D11346702293434A681A4300
:10108000A04205D0A84203D0B04201D0B84204D15A
:1010900003231B029A43CB681A4380239A430B69AC
:1010A0001A4302608A68C262096881620121416153
:1010B000F0BD0000000400400008014000140140A1
:1010C00030B5026A520852000262026A45688369BA
:1010D0007024A3439C080B68A40023430224A2436A
:1010E0008C6845601443836149684163046230BD84
:1010F00030B5026A10239A430262036A4568826926
:1011000073242402A2430C68240214432022934334
:101110008A68456012011A438461496881630262EA
:1011200030BD30B5026AFF2301339A430262026A7E
:101130004568C3697024A3439C080B68A40023433B
:1011400001246402A2438C68456024021443C361F5
:101150004968C163046230BD30B5026A01231B03D4
:101160009A430262036A4568C26973242402A24357
:101170000C68240214430122520393438A68456099
:1011800012031A43C46149680164026230BD10B59C
:10119000818CC90707D001684A6801235B049A4320
:1011A000836A1A434A60818C890707D501684A68B7
:1011B00001231B049A43C36A1A434A60818C49077E
:1011C00007D501684A6801239B049A43036B1A43BD
:1011D0004A60818C090707D501684A680123DB034F
:1011E0009A43436B1A434A60818CC90607D502684B
:1011F000916801231B039943836B19439160818C90
:10120000890607D501688A6801235B039A43C36B8B
:101210001A438A60818C490612D503685A680121F5
:101220000905046C8A4322435A60026C8A4207D142
:101230000268516803235B059943436C194351606D
:10124000818C090607D501684A680123DB04806C9C
:101250009A4302434A6010BDFEB507460025803719
:1012600004467D60F7F768FF019020680068264615
:1012700000076036002819DA274800900121002273
:1012800049052046019B00F03BFC00280ED0EFF3FF
:101290001080012181F3108821680A6880239A4315
:1012A0000A6080F310882020E06729E02068006849
:1012B000400728D5184800900121002289052046C2
:1012C000019B00F01DFC00281DD0EFF310800121D0
:1012D00081F3108821680A68FF2321339A430A604A
:1012E00080F31088EFF31080012181F310882168CA
:1012F0008A68520852008A6080F310882020386083
:1013000035760320FEBD2020E067386025666566DF
:1013100035760020FEBD0000FFFFFF0110B5806A9A
:101320000022014640314A834A82F9F75AF910BD3A
:10133000F8B5846AE06F254680352E682168896893
:1013400000270906002906DA212804D15220075374
:10135000204600F0CCF820688068400606D5222E92
:1013600004D15A200753204600F091F868681021F4
:10137000084368602046F9F734F9F8BD70B50146B6
:101380000968806A096800228906002938DB5A2129
:101390000A52EFF31081012383F3108803681C685D
:1013A000FF250135AC431C6081F31088EFF31081F9
:1013B000012383F3108803689C68640864009C60C0
:1013C00081F31088EFF31081012383F31088036801
:1013D0009C684025AC439C6081F3108820238021C9
:1013E0000B50016E01290BD1EFF31081012383F320
:1013F000108803681C681025AC431C6081F31088BA
:101400004266016E012902D0F9F7D0FB70BD582168
:10141000095AF9F7C3F870BD10B5806A0121416619
:10142000016E012902D0F9F7C5FB10BD5821095AF8
:101430004908F9F7B3F810BD10B501460968806A8C
:10144000096889061BD4002252210A52EFF3108149
:10145000012282F31088026893688024A34393607A
:1014600081F31088EFF31081012282F31088006865
:10147000026840231A43026081F3108810BDF9F717
:101480008DFC10BD10B5806AF9F78CFC10BD10B54D
:10149000EFF31081012282F3108802681368FF24A1
:1014A0002134A343136081F31088EFF310810122EC
:1014B00082F31088026893685B085B00936081F395
:1014C0001088016E01290BD1EFF31081012282F304
:1014D0001088026813681024A343136081F31088F6
:1014E000202280210A5000210166816610BD10B5BE
:1014F000EFF31081012282F3108802681368C02480
:10150000A343136081F310882021C16710BD000040
:1015100070B501464031034680338C8B1D680268EC
:10152000222D04D0906908210843906170BD526A51
:10153000456D22402A80426D921C42654A8B521EA4
:101540004A834A8B002AF1D1EFF31082012484F3FD
:10155000108804682568FF262136B543256082F38C
:101560001088EFF31082012484F310880468A568C2
:101570006D086D00A56082F3108820221A60002398
:1015800083664366174A046894420ED0626812026A
:101590000BD5EFF31082012585F31088256801260D
:1015A000B606B543256082F31088026E012A02D088
:1015B000F9F7FCFA70BD0366EFF31082012383F3A1
:1015C00010880468256810239D43256082F31088E5
:1015D0000268D469E443E40600D41362098BF8F787
:1015E000DDFF70BD0048004070B501464031034644
:1015F00080338C8B1D680268222D04D090690821ED
:101600000843906170BD526A2240446D2270426D61
:10161000521C42654A8B521E4A834A8B002AF1D1E2
:10162000EFF31082012484F3108804682568FF26F4
:101630002136B543256082F31088EFF31082012430
:1016400084F310880468A5686D086D00A56082F3B6
:10165000108820221A60002383664366174A0468B4
:1016600094420ED0626812020BD5EFF3108201256E
:1016700085F3108825680126B606B543256082F3F8
:101680001088026E012A02D0F9F790FA70BD036645
:10169000EFF31082012383F3108804682568102378
:1016A0009D43256082F310880268D469E443E40610
:1016B00000D41362098BF8F771FF70BD0048004039
:1016C000F8B50446016880682269E66910436269DA
:1016D000002532431043754B0A68754E3240024371
:1016E0000A6020684168032212039143E2681143B3
:1016F00041602168A069994201D0226A10438A683A
:101700000B263602B24302438A606A4922686A485D
:101710008A420CD1C0688007800F06D001283FD0D4
:1017200002283BD0032827D124E0012725E0634984
:101730008A420AD1C0680C2108402DD004282FD03D
:1017400008282BD00C2817D114E05D498A4223D0F9
:101750005C498A4220D09A420ED1C168032080029F
:10176000014019D001208002091A19D0091A15D098
:10177000814201D1082700E010274F4952484039E3
:1017800086009A4234D1002F0CD0022F0DD0042FA6
:1017900010D0082F7ED128E00027EEE70227ECE7E3
:1017A0000427EAE7F8F7C0F806E00968C90605D497
:1017B000304603E0F8F7D8F8002872D0626851008C
:1017C0005118814266D81103814263D3010E06028B
:1017D0005008002330185941F3F7B4FC03210902E3
:1017E0003A4A411A91425AD954E00120C003E5E730
:1017F0000122E369D20393422AD13B0001F001FAAE
:101800000906090C4A114A4A4A264A00F8F78CF898
:1018100009E0F8F799F806E00968C90605D43046EA
:1018200003E0F8F7A1F800283BD0616840004A08BF
:101830008018F3F75DFC0146254A1039914229D8FA
:10184000511C01400007400F084328E01046ECE718
:101850003B0001F0D6F90906090C1F111F1F1F21BB
:101860001F00F8F761F809E0F8F76EF806E009687C
:10187000C90605D4304603E0F8F776F8002810D002
:1018800061684A081018F3F733FC02461049103A11
:101890008A4203D9012504E01046F1E780B22168AD
:1018A000C8600020A066E0662846F8BD00480040F9
:1018B000F369FFEF0038014040100240004400404F
:1018C000004C00400050004000093D00FFFC0F00AC
:1018D000EFFF000070B504464165403002830020F0
:1018E00025468035686022212960616F002919D062
:1018F000204BCB62636F20491963636F1F495963A3
:10190000616F13468863666D216832462431606FCB
:10191000F7F7A0F9002805D0102068602020286083
:10192000012070BD206900280CD0EFF31080012148
:1019300081F3108821680A68FF2301331A430A6083
:1019400080F31088EFF31080012181F31088226862
:1019500093680B43936080F31088EFF3108081F35A
:10196000108821688A6840231A438A6080F31088AF
:10197000002070BD7D1301081914010831130108FE
:1019800070B54165014640310A834A83002383666E
:10199000012284681203FF25944204D10469002CBB
:1019A00013D1264C0AE07F26002C09D001252D07F3
:1019B000AC420CD10469002C05D03F248C8307E095
:1019C0000469002C01D08E8302E08D8300E08B83BC
:1019D000014680314B6022230B60EFF3108101231D
:1019E00083F3108803689C6801252C439C6081F375
:1019F00010888168914202D1016900290ED01049F6
:101A00008166016900290BD0EFF31081012282F376
:101A1000108800680268FF23213309E009498166C4
:101A2000EFF31081012282F31088006802682023FE
:101A30001A43026081F31088002070BDFF0100008E
:101A4000E91501081115010810B5C16F212910D140
:101A5000014640314A8A002A0CD0C26C03681288C1
:101A6000D205D20D9A62C26C921CC264488A401E92
:101A7000488210BDEFF31081012282F310880268C2
:101A800013688024A343136081F31088EFF310815F
:101A9000012282F310880068026840231A43026022
:101AA00081F3108810BD10B5C16F21290ED10146F8
:101AB00040314A8A002A0AD0C26C036812789A62BE
:101AC000C26C521CC264488A401E488210BDEFF3AB
:101AD0001081012282F31088026813688024A343D6
:101AE000136081F31088EFF31081012282F31088D4
:101AF0000068026840231A43026081F3108810BD19
:101B0000FFB5064681B080360546044660350A9F1B
:101B10002EE0781C2CD0F7F70FFB0499401AB8423E
:101B200014D8002F12D020680168490720D5C16958
:101B3000C94309070CD4082707622046FFF7A7FC12
:101B4000776000202876012005B0F0BD0320FBE778
:101B5000C069C04300050BD401202168C00208629F
:101B60002046FFF794FC2020706000202876EDE7E7
:101B70002068C1690298884305D0002103988142FA
:101B8000C7D00020E0E70121F8E70000F3B5FFB07F
:101B90008CB0E449E4A0F9F761FB0722E4A18B983B
:101BA000F3F78AFBE54D00272C46E34E403400282E
:101BB00038D00E22E2A18B98F3F77EFB002864D088
:101BC0000822E3A18B98F3F777FB00287ED0082248
:101BD000E2A18B98F3F770FB002878D00922E2A1EC
:101BE0008B98F3F769FB002872D00A22E1A18B9849
:101BF000F3F762FB002814D00922E1A18B98F3F7D8
:101C00005BFB002870D00922E0A18B98F3F754FB0E
:101C100000286AD00A22E0A18B98F3F74DFB002838
:101C20007ED07CE10C2301AA2C218B98FAF740FE90
:101C3000052876D30298FAF7C6FCA9888842F0D125
:101C400000250398FAF75AFE218E814234D020866F
:101C500031E06946C978A28D91420BD0E084684694
:101C6000407820856846807860856846C078A08581
:101C7000012537700598FAF741FEE18D884235D08D
:101C80000598FAF73BFEE085EEE00C2301AA2C2133
:101C90008B98FAF70DFE0528CBD30298FAF793FC40
:101CA000A9888842BDD100250398FAF727FEE18F65
:101CB000814201D0E087012569460498FAF792FC39
:101CC00068460078E18C8842C8D102E011E051E01A
:101CD0005CE069464978228D9142BFD16946897896
:101CE000628D9142BAD1B4E781E09CE0002DCBD166
:101CF00015E10C2301AA2C218B98FAF7D9FD0428B1
:101D000097D30298FAF75FFCA988884289D1A5A1E8
:101D10000498F3F7ADFA0028EADDA548694601E02A
:101D2000A9E0B8E00880A3A0F9F798FA11240023ED
:101D30002403022221461846FCF780FE02236A464D
:101D400021460020FCF7F2FF09240023FF22640350
:101D5000013221461846FCF771FE0398F3F781FA29
:101D6000431C21460020039AFCF7E0FF0A20F6F707
:101D7000A5FFD4E00C2301AA2C218B98FAF798FD3B
:101D8000032889D30298FAF71EFCC8E00C2301AAA5
:101D90002C218B98FAF78CFD03287CD30298FAF754
:101DA00012FCA9888842A3D188A10398F3F760FAAE
:101DB000002803D10498FAF7A1FDB08085A103980B
:101DC000F3F756FA002893D183490420886104026E
:101DD000AB8882A221465348FAF741FD0246514999
:101DE000B068FEF7C9FFAB887CA2214615E00FA8BA
:101DF00000900DAB7EA28C998B98FAF73DFC0228DF
:101E000036D10E990D9847540D98FAF7DCFBAB8844
:101E100098422DD1012171A289024248FAF71FFD93
:101E20000246404978E00C2301AA2C218B98FAF74E
:101E30003FFD00900298FAF7C6FBA9882F4688421A
:101E40006DD10098022826D30398FAF757FD85B282
:101E50000498FAF753FD80B2102D0AD001214902EF
:101E60008D4201D26900785202F0A4FA0120208448
:101E700055E0B08053E00C2301AA2C218B98FAF78F
:101E800017FD04460298FAF79EFB2C498988884280
:101E900045D1022C04D20020C0437FB00EB0F0BD6B
:101EA0000398FAF72BFD84B20498FAF727FD87B25E
:101EB00054A10DA800F04CFE85B2204854A18288A0
:101EC0000DA8401900F044FE281885B23F190BE018
:101ED0001A486100425A0DA840194EA100F038FE80
:101EE0002818641C85B2A4B2A742F1D865210DA8B8
:101EF00041556D1CA9B26E224254491C89B264221C
:101F00004254491C89B20D224254491C89B20A220A
:101F10004254491C8AB20146B068FEF72DFF0020EA
:101F2000BBE70000C034002025730D0A000000004C
:101F3000244750535F532C00D4010020C0380020A8
:101F400024434841494348554750535F532C0000B0
:101F5000247570646174652C00000000246765744A
:101F60006C6F672C0000000024636F6E74726F6CDE
:101F70002C0000002475736572646174612C00008C
:101F800024736574746F6E652C000000247365748F
:101F9000706172612C00000024726561647061726E
:101FA000612C000056323032313035313030300063
:101FB000CCCC0000676F746F204F5441204170708B
:101FC0006C69636174696F6E0D0A0000626565700B
:101FD0006572000054545300000C00502452656395
:101FE00065697665766F6963652C25580D0A000072
:101FF00024736574746F6E652C25702C25700D0A22
:1020000000000000247265706C79706172612C00B0
:1020100025782C0025642C00F0B53A4E002230784B
:102020008DB002286AD1384C384FE08A2546403DB1
:10203000012804D0022821D0002838D05AE0FBF72C
:102040000FFC8446638F228FE18EA08E099306AB2E
:1020500007C3618E6B88B2786046DCB2049205914A
:10206000029403903878190A019100900121AB88FD
:1020700027A289023248FAF7F2FB3AE0FBF7F0FBBD
:102080003049B3780A46223A0493059206910390A8
:1020900068883A78C1B2000A029100920190012149
:1020A000AB8829A289022648FAF7D9FB21E0FBF781
:1020B000D7FB8446638F228FE18EA08E089009A8FB
:1020C0000EC02A4A2A49638EB0781278097804AC87
:1020D0000FC469883B78CAB2090A6046019102922E
:1020E000039000930121AB8822A289021448FAF7D9
:1020F000B6FB02461249B068FEF73EFE00200DB066
:10210000F0BD0000D40100200039002000000020B4
:10211000245854422C25582C2530327525252C2541
:10212000642E25642C25732C25642C333A25642ECB
:1021300025642E25642E25643A25642E00000000B7
:10214000C0340020623B0020245854422C25582CD7
:102150002530327525252C25642E25642C25732CDD
:1021600025642C322573202573000000F90100201E
:1021700008000020245854422C25582C2530327554
:1021800025252C25642E25642C25732C25642C31C3
:102190002E2C25642C25640010B50023034A02214F
:1021A0000348FEF72DFC002010BD0000412201086D
:1021B000DC0100203EB5FAF7D5FD00251849194C81
:1021C000012803D00D60257000203EBD11200002C3
:1021D0000860207800280ED00228F5D1FAF7C2F85E
:1021E000E168114A411A9142EED36570E060FFF751
:1021F00013FFA570E8E701200C4D2070288DAA8DF3
:10220000698D6B4607C30121EB8C09A289020B483B
:10221000FAF725FBEA8D0949A068FEF7D1FBD3E761
:102220001C000020D40100201027000000390020ED
:1022300025752E25752E25752E257500C034002098
:1022400038B5114800240278002914D0012916D08D
:10225000022912D003290DD100946B460B4A0C4978
:102260008068FEF7F7FC002804D10948009944541F
:10227000FFF78CFC38BD012AFCD1047038BD012A5F
:10228000FCD10221017038BDD4010020FF03000001
:10229000C0340020F0B51D4C87B02178022931D11F
:1022A0001B490025097805911A4902950395049563
:1022B0000A78194901278988034601920091BF02D3
:1022C00016A239461C48FAF7CAFA21690646881947
:1022D000B84208D21948324640181749F2F773FF3E
:1022E000206980192061FAF73DF86169401AC82811
:1022F00008D3FAF737F8606110492269A068FEF741
:102300003BFD2561002007B0F0BD0000D401002096
:10231000F901002000000020C038002025732C2582
:10232000582C253032782C25782C25642C25642CCB
:102330002564250D0A000000C0340020C02C0020B8
:1023400070B5114C0D46217802291AD10F49A269A6
:102350008B1801462A461846F2F735FFA069401946
:10236000A061F9F7FFFFE169401AC82809D3F9F71E
:10237000F9FFE0610549A269A068FEF7FDFC0020B5
:10238000A061002070BD0000D4010020C0300020FA
:1023900010B50248F8F72AF910BD00001C0800200B
:1023A00010B50248F8F722F910BD0000A40800207B
:1023B00010B50248F8F71AF910BD00002C090020EA
:1023C00070B5102405252D07AC624B20C000F5F731
:1023D000C4FBAC6101F07EFC044C054D206002E0C2
:1023E00001F078FC2060A842FAD170BDC80200203C
:1023F0003001CADEF8B51D4D0E0034D0042832D2AB
:10240000742148431A494418A078002802D00128B2
:1024100022D028E0E168A068421860680090406F10
:10242000006840682769101A0818C01BF2F760FEA0
:10243000012905D817D100980068C069800612D418
:102440003878307061692069884201D1A06800E065
:10245000401C2061002506E0204618303146F8F780
:1024600025FE0028F6D02846F8BD0000FFFFFFFF3C
:10247000F02A0020002901D0042802D30020C04304
:10248000704774225043034A801840680860002057
:1024900070470000F02A002070B50C00064601D0FD
:1024A000042E02D30020C04370BD7421484321494B
:1024B0000E54227845186A706078A8706068A86029
:1024C000A168E9606278002A02D0012A05D00BE0F9
:1024D00028614018401E686106E028461830012334
:1024E000A2686168F8F7BDFDE068E86220692863CA
:1024F000A0692867606968632078002801D00128F6
:1025000006D121460C310EC928463830FAF7A2FA16
:102510006078002804D0012806D0022804D006E004
:10252000304600F009F802E0304600F021F80020C3
:1025300070BD0000F02A002038B50C4974225043C9
:1025400042185068016804E04C6A6B461C801C8885
:102550001C80CB691B07F7D491681161D368CC1834
:10256000641E54619AB2F8F7BDFA38BDF02A002013
:1025700074214843044910B5401801466831406849
:102580000122F8F7E1FA10BDF02A002070B50E46DE
:10259000044674200A49604345186868F8F700F853
:1025A000686846606868F8F777F9002802D000206C
:1025B000C04370BD204600F005F8002070BD00004B
:1025C000F02A002070B5054674201A496843441863
:1025D000A078002802D0012807D00DE0A068206173
:1025E000E1684018401E606106E020461830012373
:1025F000E268A168F8F735FD6078002801D001286D
:1026000006D121462C310EC920463830FAF722FA7D
:10261000A078002804D0012806D0022804D006E0C3
:102620002846FFF789FF02E02846FFF7A1FF0020B8
:1026300070BD0000F02A002070B50D0001D0042804
:1026400002D30020C04370BD74214843044944189C
:1026500074212046F9F786FF0020656070BD0000F8
:10266000F02A002010B502460E490020742343438F
:102670005B185B6893420FD17422424351188978EA
:10268000002906D0012901D0022901D1FFF770FFEE
:1026900010BDFFF751FF10BD401CC0B20428E5D3A8
:1026A00010BD0000F02A002038B501461348002470
:1026B00074226243121852688A4219D1742161430C
:1026C0000818817801290BD0022908D1016F00294F
:1026D00002D0806EC0B288472046FFF749FF38BD60
:1026E000816E6A46117069461830F8F79FFCF3E76F
:1026F000641CE4B2042CDBD338BD0000F02A0020B7
:10270000F7B582B00021009103991546002903D046
:10271000002D01D0042803D30020C04305B0F0BD34
:10272000742148432B4946187078344638340028C1
:1027300004D0012820D0022842D049E0F9F7B8FCA3
:1027400020462946FAF758F9070033D02046394683
:10275000FAF71EF92A4638680399F2F734FD204645
:10276000FAF72CF90446F9F791FEA088216882B2A5
:102770007068F8F781FA2BE0F9F79AFC20462946B1
:10278000FAF73AF9070015D020463946FAF700F96A
:102790002A4638680399F2F716FD2046FAF70EF933
:1027A0000446F9F773FEA088216882B27068F8F7D2
:1027B000B9FA0DE0F9F76AFE0020C043009007E087
:1027C000134664204343AAB270680399F8F7F3F9FB
:1027D0000098A3E7F02A002070B51F4A0021742357
:1027E0004B439B185B68834231D1742041438C1862
:1027F0006078002816D0012813D1204638300546CD
:10280000FAF7DCF801462846FAF7ACF82846FAF75A
:10281000D5F8002805D081888AB201686068F8F789
:1028200081FA70BD204638300546FAF7C7F80146F0
:102830002846FAF797F82846FAF7C0F80028F0D0AB
:1028400081888AB201686068F8F716FA70BD491C81
:10285000C9B20429C3D370BDF02A0020F8B5002501
:10286000184C194F64280CD0622826D0602807D154
:10287000258401F09FFD6420F5F768F91348C760CF
:10288000F8BD13486946088072B680211148F5F7F3
:10289000EDF9064607E080210E48F5F7E7F9064610
:1028A000C820F5F753F9002EF5D0022269460948F1
:1028B000F5F786FA62B6A584DBE7024865844038FE
:1028C0000580D6E7003900200400FA0500ED00E09D
:1028D000CCCC0000384A0008F8B5414C00232178E0
:1028E000404A1D46082910D007294ED0062957D046
:1028F000052959D004295AD003295BD000295DD07D
:1029000001295FD0022961D062E0A17800264A1F28
:1029100004E0344FBF5DFB189BB2761C9642F8DB97
:10292000627927799B185B18E1785E186378F6184E
:10293000F6198019C00723D0012A1DD0022A1FD101
:1029400028480078012802D10846FFF787FF26486B
:10295000E178627840182349F2F735FC01F02AFD4E
:102960006420F5F7F3F8BFF34F8F21491F48C86083
:10297000BFF34F8F00BFFDE749081846FCF794FFEF
:102980002570E570A570A571F8BDA1795054491C5A
:10299000C8B2A071A178491F8842F5D1082001E092
:1029A000607007202070F8BDE0700620FAE76071C3
:1029B0000520F7E7A070E5700420F3E7552807D15C
:1029C0000120EFE7AA2803D10220EBE7032803D078
:1029D0002570E570A570F8BD032020702071F8BD4A
:1029E000180300200C410020C03800200400FA0524
:1029F00000ED00E010B5084C04212046F6F790FBEE
:102A0000002807D1012204212046F6F78EFB03A0FF
:102A100000F074F810BD0000000800504C4F524107
:102A20005F63735F6572726F720D0A00F8B52648B6
:102A3000264D417904460B0112210C34A1702A78ED
:102A4000910051180F31E1702149098801824189B3
:102A5000A1710E0AE671491C41811E481E49007889
:102A60002072637218480B88C3820020088020738C
:102A70006073A073E073227420465200174911302E
:102A8000F2F7A1FB28781649420010191130F2F72D
:102A90009AFB2A781349900000191130F2F793FB42
:102AA000287881004118A01C0F31F4F711FF694606
:102AB0000880287881004018694600190978417417
:102AC000694649788174F8BDF4010020E1020020D4
:102AD00088000020000000202E030020A43F0020DA
:102AE000F43F00204440002003480179002901D030
:102AF000418A491C41827047000000200FB410B584
:102B000003A9044B044A029800F054FA10BC08BC14
:102B100004B0184789400108BC0600200FB41CB55A
:102B20000246002007AC00290BD0491E01910092FB
:102B3000064B6A462146069800F03CFA009A0021AE
:102B400011701CBC08BC04B018470000ED36010829
:102B50000FB410B504A9074B02AA039800F02AFA93
:102B6000044602A9002000F0CCFD204610BC08BCA1
:102B700004B01847033701087CB51546024600200B
:102B80001C4600290BD0491E00920191044B6A4655
:102B90002146284600F00EFA009A002111707CBDF3
:102BA000ED3601082021020C01D010211046020A46
:102BB00001D010460839020901D01046091F8208C9
:102BC00001D01046891E420801D0881E7047081A9D
:102BD0007047F8B5040C8BB2264682B25E430D0CEA
:102BE0001046370C584336048019002179411646A7
:102BF0006E43370C36048019794126466E43891995
:102C0000F8BD30B47446641E2578641CAB4200D213
:102C10001D46635D5B00E31830BC18478307FF2245
:102C2000DB0E9A408907090E9940002808DB8308CB
:102C300009489B001B1818689043084318607047A8
:102C40000007000F0838830804489B001B18D86948
:102C500090430843D861704700E400E000ED00E0D5
:102C600000487047C0060020014800687047000017
:102C7000C006002002E008C8121F08C1002AFAD1CD
:102C800070477047002001E001C1121F002AFBD1EC
:102C9000704700000149086070470000C00600202E
:102CA00008B50021684601706B46012202212C20E4
:102CB00001F032F90221684601706B4601222C2096
:102CC00001F02AF908BD000038B504466D206946B8
:102CD00008706B46012207492E2001F01DF90649B4
:102CE000002C01D0054A00E0054A2E2001F0FAF838
:102CF00038BD0000060800000618000007060000A6
:102D00000716000038B504466B4602220021362023
:102D100000F0E6FFB3212300FFF773FF0E0F081545
:102D20003A3A3A3A1C273A3A2F34483A0021684650
:102D3000017040784108490014E06946087880082D
:102D40008000401C04E06946087880088000801CF0
:102D500008701DE0684602780A40483202704178E7
:102D6000802001436846417012E0684602780A40BC
:102D7000027040784106490EF4E76946487802211E
:102D8000084303E069464878FD21084069464870D9
:102D90006B4601220021362001F0BEF8012200AB73
:102DA00011463620013301F0B7F838BD694608787E
:102DB000CF21084069462030CAE708B5032168469C
:102DC0004170012101706B4602220021362001F082
:102DD000A3F80122D20306212D2001F083F801205F
:102DE00000F00EFD0120FFF78DFF08BD08B5020AB7
:102DF00069464A7008706B46022204212D2001F0BA
:102E00008BF80320694608706B46012206212D20AD
:102E100001F082F80020694608706B460122062105
:102E20002D2001F079F80A212D2000F03FFF08BD88
:102E3000F0B51FB486B00998089A030D002102432B
:102E400014D05148514A18185043051411980128BC
:102E500010981AD0281A401C00264D4F4D49009654
:102E600001910490002812DA444211E011980124E3
:102E700049A3012801D11098C1430698119A846092
:102E80000360C26041600BB0F0BD4042E4E704461D
:102E9000210500203F4A001C51410391029012E09D
:102EA000E00707D032463B4601990098F2F710FB45
:102EB0000191009032463B4610461946F2F708FB56
:102EC00006460F466410002CEAD10498039B0028A4
:102ED000029A0999089806DAF2F7FAFA019B009A21
:102EE000F2F7F6FA05E0F2F75BFB019B009AF2F7C6
:102EF00057FB04460E460022284BF2F74FFC03D83E
:102F00000020C043014607E00022254B2046314601
:102F1000F2F72CFAF2F7FEFD102409E0002C0ADB90
:102F20000A220023F2F70EF9079B30321A55641E6D
:102F300002460A43F2D11122641C079B121B1C1982
:102F4000119B012B03D0012308430ED10AE0084353
:102F500004D0112010900020119077E71098151AD6
:102F60006D1E0BE01098824202DD00236D1C03E011
:102F7000824201DA00236D1E002BEED006981199D3
:102F80008260C16030C07EE701FCFFFF104D000091
:102F9000000014400000F03F300000000000F0434B
:102FA0000000E03F30380A2801D20120704700209D
:102FB00070470000FFB597B00646002518E22528A7
:102FC00077D100242746FD49049400E00443761C91
:102FD00032780120203A90400842F7D130782A28F0
:102FE0000ED00222307801463039092916D80499CA
:102FF0000A235943303940181443761C0490F1E7F2
:10300000189802C804911890002904DA012040039E
:1030100004434842049002200443761C30782E2852
:1030200014D1042004437078761C2A2809D11898FA
:10303000761C80C8189009E00A214F43303FC71919
:10304000761C3078014630390929F5D930786C285A
:1030500010D006DC4C281AD068280ED06A2817D168
:1030600004E0742813D07A2812D110E00120400522
:1030700004430CE00121090501E0032109050C438B
:103080007178814203D1012000052418761C761C3A
:103090003078119066280BD013DC58287DD009DCDD
:1030A00000287BD04528F6D04628F4D047281AD1EE
:1030B000A5E118E0632835D0642870D0652812D1C6
:1030C0009DE170286CD008DC6728F1D069287BD09E
:1030D0006E280DD06F2806D1BAE073282ED075283F
:1030E00071D0782859D01A9A199990476D1C7EE1B1
:1030F0006002400F022809D003280DD00428189838
:1031000001680DD00D60001D189070E11898EA1745
:1031100001680D604A60F6E7189801680D80F2E7D3
:103120000D70F0E718986A4601781172001D18902A
:103130000020507202A80090012005E0189802C8F3
:10314000189000200091C04361070DD5002101E0D7
:103150000199491C0191B94212DA8142F8DB009AC7
:10316000515C0029F4D10BE0002101E00199491CD8
:1031700001918142FADB019A0099895C0029F5D11D
:10318000019904981A9B471A21463846199A00F06B
:1031900097FA0199401945180BE04FE02CE113E034
:1031A0004EE0009800990078491C00911A9A1999EC
:1031B00090470198401E0190401CF2D121463846AC
:1031C0001A9B199A10E137E00A2000210090019122
:1031D0006002410F022907D0189A01CA1892C2173B
:1031E0009446032908D00AE01898C01DC108C900F8
:1031F00005C91891944607E000B2C2179446042905
:1032000002D140B2C1178C4600226146944506DACD
:103210000A460021404291418C462D2102E02105C1
:1032200004D52B216A461173012103E0E10701D087
:103230002021F7E7029155E00A200AE0102008E07B
:10324000102000900021042004430191082703E08E
:1032500008200021019100906002410F022907D04F
:10326000189A01CA189200229446032908D008E04F
:103270001898C01DC108C90005C91891944603E0FB
:1032800080B2042900D1C0B200210291210729D5C2
:103290001199702906D0009A1021019B4A401A43C7
:1032A00005D00EE040216A461173012108E0614615
:1032B000014306D030216A461173119951730221DE
:1032C0000291009A0821019B4A401A430AD16146A3
:1032D000014301D1610705D530216A4611730121EF
:1032E0007F1E02911199582904D035A10E910DA984
:1032F0000D910DE037A1F9E76146019B009AF1F7C6
:1033000021FF0E9B8C469B5C0D9A521E0D921370F2
:1033100061460143F0D10D9805A9081A20300190AB
:10332000600703D501200004844300E001270198D1
:10333000874201DD381A00E0002001990090411811
:10334000029809180498401A0490E00306D4214614
:103350001A9B199A049800F0B3F94519002706E062
:1033600003A81A9AC05D199990476D1C7F1C02989A
:103370008742F5DBE0030CD521461A9B199A049885
:1033800000F09EF9451904E01A9A302019999047E7
:103390006D1C0099481E00900029F5DC08E00D988E
:1033A0000D990078491C0D911A9A199990476D1C36
:1033B0000199481E01900029F1DC63E10928010010
:1033C000303132333435363738396162636465669B
:1033D000000000003031323334353637383941425D
:1033E000434445460000000000F05AF94519761C98
:1033F0003078002800D0E2E528461BB0F0BD600719
:1034000000D406271898C01DC108C90048680A687A
:103410000831C30FDB071891190001D09CA108E007
:10342000210501D59BA104E0E10701D09AA100E0AC
:103430009AA1430011985B08109165280CD006DC16
:10344000452809D046281DD0472841D141E06628AB
:1034500018D067283CD13CE00021112F01DB11205E
:1034600000E0781C0191009008A911A8FFF7E0FC8A
:10347000139905910021119A15927F1C12980197BA
:10348000009150E00120C00703900120019008A99D
:10349000009711A8FFF7CCFC139A1499059200220B
:1034A000119B009212981593059A0192002901D060
:1034B000104602E0791C40180190381A01D5019895
:1034C00004E04042401E0090781C0190C01B029016
:1034D00043E0012F00DA01270021112F01DD112027
:1034E00000E038460191009008A911A8FFF7A0FC60
:1034F00013990591119A0021129815920091019744
:1035000021070CD40599B94201DB019900E0019132
:10351000012904DD159A491E515C302906D0B842B4
:1035200001DA011D05DA0121029115E00199491E18
:10353000EDE7002805DC0099411800910199091A6E
:1035400003E0019A411C914200DD01910099401A6B
:10355000401C02900120C0070390200706D4029966
:103560000198814202DB0020C0430290002069469E
:10357000C87707AF012103980337C907884224D0D1
:10358000022011902B201290039800280CDA404260
:1035900003902D20129007E00A210398F1F7A8FD6F
:1035A00030317F1E039039701199481E1190002907
:1035B000F2DC03980028EFD1791E12980870307859
:1035C000202108404530BF1E387006A8C01BC01D12
:1035D000039010980078002800D00120019941182C
:1035E0000298C0170918039809180498401A401E39
:1035F0000490E00306D421461A9B199A049800F01F
:103600005FF8451910980078002803D01A9A199984
:1036100090476D1CE00324D521461A9B199A049803
:1036200000F04EF845191CE00098002807DB0099CF
:103630000598884203DD1598405C199901E01999B5
:1036400030201A9A904700986D1C401C00900298F8
:10365000401E0290002804D11A9A2E2019999047F2
:103660006D1C0199481E01900029DDDC05E03878C9
:103670001A9A7F1C199990476D1C0399481E039054
:103680000029F4DC21461A9B199A0498ACE6000044
:103690002D0000002B0000002000000000000000B2
:1036A000F8B5044600251E461746880404D405E0F4
:1036B00039462020B0476D1C641EF9D52846F8BD58
:1036C000FFB50446002581B01E46C80301D530274A
:1036D00000E02027880404D505E038460399B04768
:1036E0006D1C641EF9D5284605B0F0BD4A68002A55
:1036F00006D00A68531C0B6010704868401E486072
:1037000070470A68531C0B601070704730B583B067
:103710000446FFF7A9FA05460020009002460190F2
:1037200021466846F2F7A9F82846FFF7B3FA01994F
:10373000009803B030BD0000F8B54A002B4B520D85
:10374000D6182B4A0C460546142E2BDA002E12DA18
:10375000284BF1F70BFE00221346F2F71FF840D278
:10376000002C03DA0124E40700253AE02046284330
:1037700037D0214C14E0214F0B46F7403B402B4300
:1037800031D01C4BF1F7F2FD00221346F2F706F898
:1037900027D2002C03DD01200005F0400419BC43B2
:1037A00000251EE0332E1EDC33460027143BFF436A
:1037B000DF40384217D00F4BF1F782FE002213464C
:1037C000F1F7ECFF0DD2002C0ADD142E0CD03420C2
:1037D000811B012088404019A84200D2641C054684
:1037E000BD4321462846F8BD641CF9E701FCFFFFF4
:1037F0009C7500883CE4377E0000F03FFFFF0F001F
:103800007D2110B5C9004843F4F7A7F910BD002188
:1038100040E000BF00BF00BF00BF00BF00BF00BF4F
:1038200000BF00BF00BF00BF00BF00BF00BF00BFA0
:1038300000BF00BF00BF00BF00BF00BF00BF00BF90
:1038400000BF00BF00BF00BF00BF00BF00BF00BF80
:1038500000BF00BF00BF00BF00BF00BF00BF00BF70
:1038600000BF00BF00BF00BF00BF00BF00BF00BF60
:1038700000BF00BF00BF00BF00BF00BF00BF00BF50
:1038800000BF00BF00BF00BF00BF00BF00BF00BF40
:1038900000BF491C8142BCD370470000FEB50446FE
:1038A0000020019000906079734940000E5A6178C1
:1038B0002578491E7148CFB20163042D77D0072DBA
:1038C00075D000210291217801736C49E3790122BE
:1038D00092058969002B6CD0914381616748217AF8
:1038E0004173217A82698907890B0A438261002129
:1038F000042000F002FB324661492E2000F0F2FA6B
:103900003846FFF7E1F95F4E0522705D81004018EF
:103910005D49431807212B2000F0FEFA5B4902980D
:1039200001220B180B21282000F0F6FA705D58498F
:1039300080000A580C21282000F0DFFAE079554970
:1039400080004018A1794900425A0221272000F046
:10395000C9FA51487E00825B0421272000F0C2FA98
:10396000E079002829D0A07804282CD028206946A6
:10397000087220220621272000F0B4FA02AB0122AF
:103980002621272000F0C8FA444938014018E17880
:10399000890042580821272000F0AFFAA17A601C64
:1039A000627A0902114313D016E000E001E0012120
:1039B00088E71143F608816190E7642206212720F9
:1039C00000F090FAE0E71020694608720246D1E75D
:1039D00033490172090A4172417A007A0A020243AC
:1039E0002021272000F07EFA2E4F0C2123203A6858
:1039F00000F083FAF01982880421232000F072FA83
:103A0000A07900280BD0E079274901224318002132
:103A1000212000F081FA03200190012000902A0764
:103A2000120F10010243607800218007000B02434F
:103A30000198000502430098400402432079C00623
:103A4000400902436079C00602431F2000F055FA86
:103A5000A07861780123084302040848DB0302616F
:103A6000E179490319430A4302610021082000F06B
:103A700044FA0020FEBD00007C4B010840440020B9
:103A800004280000244B0108E9030020070400205B
:103A90002C4B01084C4B0108584B01085C4B0108AA
:103AA00041100000444B01080904002038B50C46C1
:103AB00007498A8B002102432C2000F013FA684644
:103AC00004706B46012206212C2000F025FA38BD37
:103AD0004044002010B5FFF7E3F810BD10B50446D0
:103AE0000421362000F0E2F80121C902002C01D0A7
:103AF000084300E0884302460421362000F0FDF927
:103B000010BD000038B540206946087000210E2025
:103B100000F0CCF80446002211460E2000F0EDF92A
:103B20006B46012200210D2000F0F6F9074A002122
:103B30000F2000F0E2F900F0BBF9224600210E2030
:103B400000F0DBF902480021017338BDF8FF27249B
:103B5000604400207CB50646042069460870434C4A
:103B60000020607521462031206348710873A083CE
:103B70006063A06300F0AEF83D4D206002E000F00D
:103B8000A9F82060A842FAD10020FFF7BBF8394815
:103B900043210170384A00211E2000F0AEF96B4627
:103BA00001220021242000F0B7F91E20FFF71EF9A2
:103BB00085B2280AA0730420FFF718F90006000E4A
:103BC0000DD002206946087101AB012212212D207F
:103BD00000F0A2F9A08B012109030843A08300F0A3
:103BE00079F820600620FFF701F960600720FFF7F1
:103BF000FDF8A060E806C00E207501D110202075E8
:103C0000C0B200F0C5F9F00707D0FFF7D6F8A08BD7
:103C10000121C9020843A0830AE00521362000F0F3
:103C20002FF81649084002460521362000F05AF9BF
:103C30000120FFF767F80021042000F037F8A061A9
:103C40000021262000F032F815218903084302469E
:103C50000021262000F051F900222621362000F014
:103C600041F900F037F8206000207CBD404400207E
:103C70003001CADEE80300201F1F1F1FFFFD0000E8
:103C800038B5094C89B280B26B46022200F028F8A0
:103C9000002806D168464078010268460078081876
:103CA00084B2204638BD0000FFFF000038B5002474
:103CB000E44389B280B26B46042200F011F8002878
:103CC00006D103216846435C2202D418491EFAD566
:103CD000204638BD10B500210846FFF7E7FF10BDAC
:103CE00038B5002909D0402420436C462070C8B262
:103CF0007F2906D8607002200AE06946087001201A
:103D000006E0802420436C466070C809A070032040
:103D1000694600F00FFB38BD10B5144603460A464D
:103D200021461120FFF7DCFF10BD10B50346052228
:103D300000211520FFF7D4FF10BD38B5054600203F
:103D40006946087000F0B4F8FF2401342246002DC3
:103D500001D00322120200210D2000F0C3F8002D33
:103D600013D06B46012203210F20FFF7B9FF6846ED
:103D70000078000709D5FFF7C5FE224600210D2077
:103D800000F0B0F80020C04338BD002038BD10B5A9
:103D9000024601210A2000F0B0F810BD10B502461D
:103DA00002492E2000F09EF810BD0000041800000B
:103DB000F8B505466B46012203210420FFF790FF6A
:103DC0000126114C3607002D0DD02A4600210C206B
:103DD00000F088F8694608781021084369460870A1
:103DE000A069304307E069460878EF21084069463A
:103DF0000870A069B0430B46A06101220321042092
:103E000000F08AF8F8BD00004044002010B50246DA
:103E10000021182000F066F810BD0000F8B5074634
:103E2000002568460570B807204C2E4600280ADA9F
:103E30008020694608706B46012200210D2000F0A9
:103E40006BF801202073F8076946087821D0062115
:103E50000843694608706B46012200210D2000F0DE
:103E60005BF803210F20FFF70BFF8121C9000842F7
:103E700019D04020694608706B46012200210D20B0
:103E800000F04AF80020FFF729FE00252673ED43D5
:103E900009E002210843694608706B4601220021AF
:103EA0000D2000F039F82846F8BD000060440020DD
:103EB0001CB56B46012203210F20FFF711FF684656
:103EC00000784022C1091040C9014000814208D059
:103ED000012069460871024601AB03210D2000F064
:103EE0001BF81CBD08B56B461A70120A5A7089B2CD
:103EF00080B2022200F010F808BD38B500236C46ED
:103F0000E254120A5B1C042BFADB89B280B223460E
:103F1000042200F001F838BD38B58024002909D00A
:103F2000C02528436D462870C8B27F2907D868701D
:103F3000022009E0204369460870012004E0204384
:103F40006870C809A8700320694600F059FA38BDA6
:103F500010B51446012312189B029A4202D9002080
:103F6000C04310BD0B46821E21460920FFF7D4FF37
:103F7000002010BD10B5054A8905126901430A43A6
:103F800000210820FFF7B9FF002010BD40440020A9
:103F900038B504466B4601220E212B20FFF7A0FE08
:103FA00068460078E10640094001C90E01436846B1
:103FB00001706B4601220E212B20FFF7ADFF38BDAB
:103FC000F8B54A002B4B520DD6182B4A0C46054625
:103FD000142E2BDA002E12DA284BF1F7C7F9002243
:103FE0001346F1F7DBFB40D2002C02DB0024254610
:103FF0003BE060004008284337D0214C14E0214FBB
:104000000B46F7403B402B4331D01C4BF1F7AEF948
:1040100000221346F1F7C2FB27D2002C03DA01205D
:104020000005F0400419BC4300251EE0332E1EDCC1
:1040300033460027143BFF43DF40384217D00F4B75
:10404000F1F73EFA00221346F1F7A8FB0DD2002C3F
:104050000ADA142E0CD03420811B0120884040192C
:10406000A84200D2641C0546BD4321462846F8BD3F
:10407000641CF9E701FCFFFF9C7500883CE4377E77
:104080000000F0BFFFFF0F0013B501231A46694679
:104090000248F6F790FD00981CBD00001C080020A7
:1040A00008B5F5F795F8FCF773FFF9F74DF8624896
:1040B000016B012211430163006B1040002200904C
:1040C00011460A20F5F758FA0A20F5F749FA5B4934
:1040D0005B48002412C07F2101608460C4600461D9
:1040E000FF21446141600838F5F794FE002801D0B3
:1040F00072B6FEE7F9F782F9F9F764F9F9F7E2F831
:10410000F8F7EAFF4E484F49303812C00460846126
:10411000C4614D490462C1600838F5F74BF90028C5
:1041200001D072B6FEE7F9F731F9F9F7EBF8444838
:10413000464940380160062141604549C1608160BF
:10414000F5F700F8002801D072B6FEE73C490020E0
:10415000BC31FEF771FA3F490320FEF76DFA3D4985
:1041600002208839FEF768FA354900202431FAF731
:1041700077FE394C0122920221460020F2F75CFAC8
:10418000012221460220F2F757FA344D0122520350
:1041900029460120F2F750FA102229460020F4F7B0
:1041A00031F90021202322460846FAF719FD0020A4
:1041B000FAF77EFCF3F7B8FBFBF7E4FDF9F710FD27
:1041C000F3F70AFFF8F7C6FDFDF7E6FFF3F70CFD7E
:1041D0000721A015FFF76AFCFFF77CFCF8F736FE15
:1041E000FF24F5342046F4F769FDF8F74BFF144837
:1041F00000221B493038F5F751F9002801D072B67A
:10420000FEE71120000403461A461146FBF78CFB1B
:104210002046F4F753FDFBF7A5FB2046F4F74EFDCF
:10422000F3F79EFE2046F4F749FDF4F77FF90D49B8
:104230000870F9F7FFF8FCE7001002400028004082
:1042400060070020007C0040FFFF000000300040BD
:10425000FF0F00002C09002000040050000800504F
:10426000FF7F000000000020F8B5012292022A49D9
:104270002A48F3F71BFD28482949028804460025EF
:104280007926212740348A4235D001802549818012
:104290007D21C900C1800A2101811E214581C943B8
:1042A00081810121C1818583618302220287782275
:1042B00042878187C187E58225846584A584C5837B
:1042C000A5802721E1846A212185D22161850D21E4
:1042D000A1851549E1856686A786E221E1862A2126
:1042E0002187124961874B21C9002186E187052179
:1042F000818200F05FF86584A5842584608E0C4976
:10430000884207D16686A786E220E0862A20208799
:1043100006486087F8BD0000C038002000F801089A
:10432000AA55000072180000581B00004F2300001F
:10433000FFFF0000FFB581B01D461646074600246A
:10434000FEF758FB102105231B0799620E4808E071
:10435000029A125DC2608268D207FCD0C2682A70DD
:10436000641CBC42F4DB0022174606E0C760846888
:10437000E407FCD0C468AC54521CB242F6D3996135
:10438000002005B0F0BD000000300140F8B5154632
:104390001E4607460024E20028463146F0F702FF99
:1043A0003855641C042CF6DBF8BD10B5F1F774FB2E
:1043B00010BD000070B572B601250C4EAD02294645
:1043C0003046F3F753FC044607E029463046F3F73E
:1043D0004DFC0446C820F3F7B9FB002CF5D02A4663
:1043E00003493046F3F7ECFC62B670BD00F80108F3
:1043F000C0380020002100E0491C8142FCD37047F6
:10440000FFB581B015460F4606460024FEF7F2FAC6
:10441000102205231B079A620D4906E0385DC8602B
:104420008868C007FCD0C868641CB442F6DB002072
:1044300007E0049C245CCC608C68E407FCD0CC686A
:10444000401CA842F5D39A61002005B0F0BD0000E1
:1044500000300140000000000000000001020304E1
:1044600006070809030406080C1018203000000095
:1044700000010203040000002451010802000000B2
:10448000DC500108020000007C4E0108030000001F
:104490003052010803000000084E01080700000028
:1044A000104E010808000000C84E01080900000075
:1044B0006C4E01080A000000844D01080B0000004A
:1044C000584E01080C000000E84E010810000000E2
:1044D000244E010811000000744E01081200000073
:1044E000D4500108180000002851010819000000EC
:1044F000404E0108160000005C4C0108140000004A
:10450000484C01081A000000BC4D010817000000CB
:10451000C84D01081B000000DC5201081C0000000F
:10452000B44E01081D000000344E01081E000000BA
:10453000A84E01081F000000BC4E0108200000002A
:10454000A84D010821000000D04D01082200000004
:10455000E04D010823000000904D010824000000F8
:104560002C4E010825000000684D010826000000BF
:10457000344C0108270000004C4E010828000000C0
:10458000FC4D010829000000604E01082A000000CF
:104590009C4D01082B000000784D01082C00000004
:1045A000884E01082D000000DC4E01082E0000009E
:1045B000D04E01082F000000184E01083000000006
:1045C0009C4E010831000000B44D010815000000A8
:1045D000D453010832000000944E0108330000005B
:1045E000F04D0108340000006C4C0108350000005B
:1045F0008C4C010836000000A44C01083700000074
:10460000BC4C010838000000D44C010839000000FF
:10461000EC4C01083A000000044D01083B0000008A
:104620001C4D01083C000000344D01083D00000015
:104630004C4D01083E000000644D01083F000000A1
:10464000D8530108FC520108105101081C520108FE
:104650006453010800520108FC5001086C50010825
:104660008050010834530108EC510108D051010871
:10467000A451010848530108AC5301084C510108EA
:10468000AC5001085052010838520108244F01086B
:10469000084F0108B04F010890510108C44F0108AC
:1046A000E450010834510108405001089C4F0108B2
:1046B000C45201080853010860510108E45201087E
:1046C0001C530108844F0108D84F0108F44F01081A
:1046D000544F0108C0500108EC4E0108AC520108CB
:1046E0007851010828500108B85101086C4F0108A1
:1046F0003C4F010868520108945301087C5301089B
:104700009450010894520108C053010880520108D6
:104710001050010854500108784C0108904C0108D1
:10472000A84C0108C04C0108D84C0108F04C010805
:10473000084D0108204D0108384D0108504D010871
:104740006054010800000000704701087D6C0008FB
:10475000F0540108404701087047010895690008B6
:10476000845401084047010800000000796B0008EC
:10477000B45401085047010800000000C96B00084C
:10478000205501085047010800000000D9620008C8
:10479000545501085047010800000000D17200087C
:1047A0000C55010850470108000000009561000801
:1047B00078540108404701080000000079690008AA
:1047C00034550108404701087C480108E96C00089D
:1047D000FC540108C04701080000000005670008FC
:1047E00044550108C0470108F04701080169000865
:1047F000A4540108E047010800000000C568000853
:1048000094540108E0470108000000008566000894
:104810003C540108881300000100000028540108DE
:1048200088130000010000001C54010888130000D8
:10483000010000003454010888130000010000004A
:10484000FC53010888130000010000000C5401080B
:104850008813000001000000E453010860EA000032
:10486000030000004854010860EA00000300000053
:1048700054540108E8030000050000006C550108CD
:10488000C047010800000000516D0008B055010844
:10489000E047010800000000616F00089C55010816
:1048A000E0470108000000009D6E000884550108E3
:1048B000E047010800000000FD7000082052D80009
:1048C0000010000000800000000001009457010863
:1048D000B50801088C57010819000108785701082C
:1048E000BDFF0008C856010841FF000870570108C5
:1048F000B9FF0008105701081906010808570108F8
:1049000075FC0008FC55010879F90008E456010817
:10491000A9FB0008A056010861FB000844570108E4
:10492000BDF900085457010899FE0008F056010827
:1049300009FF0008AC560108D1FE00086C560108BA
:10494000B9080108745601086D0701086457010889
:10495000C9060108045601080D080108605601083F
:104960003506010810560108F5F9000880560108BF
:10497000EDFB00089056010825000108F0550108DC
:10498000DDFA0008FC5601082D040108245701082F
:10499000D10501083057010889050108BC560108F6
:1049A000610301083C560108E9000108A857010805
:1049B0001D0201081C560108D10201082C560108ED
:1049C000F90401081857010861010108E0550108C0
:1049D00095FE0008E455010891FE0008B85601084C
:1049E00099FD0008D856010809FE00088057010803
:1049F0003DFE000850560108B9F900089C5701080F
:104A0000B1080108DDE10008B9E1000861E400082F
:104A10002DE400080DE300083DE30008C9E40008A8
:104A200061E6000881E10008D9E70008EDE300082D
:104A3000A5E70008C5E7000889E30008CFE70008FC
:104A400091E7000881E300085DE9000871E30008D0
:104A500065E9000879E3000835E4000891E40008FE
:104A6000D7E1000825E20008BDE3000859E6000888
:104A700004050600C01200001F000000A816000078
:104A800017000000841C00000F000000E425000057
:104A90001E000000B42D00001600000008390000C0
:104AA0000E0000002C4C00001D000000685B0000A0
:104AB00015000000747200000D00000058980000FE
:104AC0001C00000034B7000014000000E8E40000FF
:104AD0000C000000783101001B000000686E01002E
:104AE0001300000034CA01000B000000286202001D
:104AF0001A00000040DB0200120000003C9303009B
:104B00000A000000C0C204001900000060B30500E4
:104B100011000000382007000900000020A1070054
:104B2000000000000000010203040005405C0000DA
:104B3000A05C0400C06C0800805C0400E03F1E0024
:104B4000E07D1E0007A9022570889B880A001600D8
:104B5000010006000100020087008D002D001A31BF
:104B600052001A339A001A351D011A376B003B3177
:104B7000BE003B335E013B3596023B37000099593E
:104B80009959EB518F421E45142E0080EB51F528A8
:104B90003333E13A703DE13AC235852BC2353333C8
:104BA000C235C235AE47E13A5138A33051380040E2
:104BB00040404040404040404141414141404040F0
:104BC0004040404040404040404040404040400520
:104BD0000202020202020202020202020202022097
:104BE0002020202020202020200202020202020297
:104BF00090909090909010101010101010101010B5
:104C000010101010101010101010020202020202F8
:104C10008888888888880808080808080808080814
:104C200008080808080808080808020202024000EC
:104C3000AF4B01082B51495552433A202270647002
:104C400064656163742200002B51495552433A2038
:104C500022636C6F736564222C0000002B51495550
:104C600052433A202272656376222C002B52454330
:104C7000454956452C000000414952373830455FC0
:104C80004556454E545F4E554D5F30003000000094
:104C9000414952373830455F4556454E545F4E5571
:104CA0004D5F310031000000414952373830455FD7
:104CB0004556454E545F4E554D5F32003200000060
:104CC000414952373830455F4556454E545F4E5541
:104CD0004D5F330033000000414952373830455FA3
:104CE0004556454E545F4E554D5F3400340000002C
:104CF000414952373830455F4556454E545F4E5511
:104D00004D5F350035000000414952373830455F6E
:104D10004556454E545F4E554D5F360036000000F7
:104D2000414952373830455F4556454E545F4E55E0
:104D30004D5F370037000000414952373830455F3A
:104D40004556454E545F4E554D5F380038000000C3
:104D5000414952373830455F4556454E545F4E55B0
:104D60004D5F3900390000002B51475053585452C1
:104D700041444154413A00002B514D545355423A5D
:104D8000000000002B43495047534D4C4F433A001D
:104D90002B514750534C4F433A0000002B514D5478
:104DA000444953433A0000002B5148545450524553
:104DB00041443A002B434349443A00002B514953A4
:104DC000454E443A000000002B514952443A00003D
:104DD0002B51485454505245414446494C453A00A1
:104DE0002B5148545450504F535446494C453A0067
:104DF0002B514C544F4E453A000000002B514D545E
:104E0000434C4F53453A00002B435245473A00006C
:104E10002B43475245473A002B514D5450494E477A
:104E20003A0000002B434D54493A00002B43434CB9
:104E30004B3A00002B51464F50454E3A00000000BF
:104E40002B51494F50454E3A000000002B514D5414
:104E50004F50454E3A0000002B4350494E3A000057
:104E60002B514D54434F4E4E3A0000002B435351AB
:104E70003A0000002B434D47523A00002B434D456A
:104E8000204552524F523A002B514D54554E533AF1
:104E9000000000002B435454533A00002B514D5452
:104EA000535441543A0000002B5148545450474544
:104EB000543A00002B51464C53543A002B5148545D
:104EC0005450504F53543A002B43474154543A00E6
:104ED0002B514D54524543563A0000002B514D542E
:104EE00050554245583A00003E00000041495237B3
:104EF0003830455F4556454E545F514750535854DE
:104F00005241444154410000414952373830455FD5
:104F10004556454E545F4E45575F49505F44415496
:104F200041000000414952373830455F4556454EF3
:104F3000545F534D535F444154410000414952373F
:104F40003830455F4556454E545F514D5453554298
:104F500000000000414952373830455F4556454E04
:104F6000545F514750534C4F430000004149523762
:104F70003830455F4556454E545F514D5444495372
:104F800043000000414952373830455F4556454E91
:104F9000545F51485454505245414400414952379E
:104FA0003830455F4556454E545F524541440000F8
:104FB000414952373830455F4556454E545F43436B
:104FC00049440000414952373830455F4556454E07
:104FD000545F53454E440000414952373830455FD5
:104FE0004556454E545F51485454505245414446ED
:104FF000494C4500414952373830455F4556454E8A
:10500000545F5148545450504F535446494C4500F6
:10501000414952373830455F4556454E545F514CF3
:10502000544F4E4500000000414952373830455F2B
:105030004556454E545F514D54434C4F5345000027
:10504000414952373830455F4556454E545F434CD1
:105050004F534500414952373830455F4556454E1C
:10506000545F524543454956450000004149523777
:105070003830455F4556454E545F43524547000022
:10508000414952373830455F4556454E545F434796
:1050900052454700414952373830455F4556454EE5
:1050A000545F514D5450494E47000000414952371A
:1050B0003830455F4556454E545F41434B00000034
:1050C000414952373830455F4556454E545F43435A
:1050D0004C4B000053454E44204F4B005348555411
:1050E000204F4B00414952373830455F4556454EB9
:1050F000545F53454E445F4F4B00000041495237C7
:105100003830455F4556454E545F4F4B0000000018
:105110004849444F5F41545F4556454E545F4F4B9D
:10512000000000004F4B000053454E4420464149CB
:105130004C000000414952373830455F4556454ED6
:10514000545F53454E445F4641494C002D414952FE
:10515000373830455F4556454E545F504F4C4C00F4
:10516000414952373830455F4556454E545F5146A8
:105170004F50454E00000000414952373830455FDE
:105180004556454E545F514D544F50454E0000001A
:10519000414952373830455F4556454E545F4F5070
:1051A000454E0000414952373830455F4556454E1F
:1051B000545F4350494E0000414952373830455FF3
:1051C0004556454E545F514D54434F4E4E000000DE
:1051D000414952373830455F4556454E545F4C4241
:1051E000535F4C4F434154494F4E000041495237A1
:1051F0003830455F4556454E545F435351000000DB
:105200004849444F5F41545F4556454E545F5345AE
:105210004E445F4552524F52000000004849444FEF
:105220005F41545F4556454E545F4552524F5200C0
:105230004552524F52000000414952373830455FC5
:105240004556454E545F524541445F534D5300000F
:10525000414952373830455F4556454E545F4E45BB
:10526000575F534D53000000414952373830455F76
:105270004556454E545F514D54554E530000000065
:10528000414952373830455F4556454E545F515479
:1052900054530000414952373830455F4556454E1A
:1052A000545F514D5453544154000000414952370A
:1052B0003830455F4556454E545F50445044454153
:1052C00043540000414952373830455F4556454EFA
:1052D000545F434F4E4E454354000000434F4E4EE3
:1052E00045435400414952373830455F4556454E95
:1052F000545F514854545047455400004556454E5C
:10530000545F455849540000414952373830455F91
:105310004556454E545F51464C535400414952370F
:105320003830455F4556454E545F514854545050AF
:105330004F535400414952373830455F4556454E2A
:10534000545F434741545400414952373830455F18
:105350004556454E545F494E49545F54494D454F5B
:10536000555400004849444F5F41545F4556454EEF
:10537000545F54494D454F55540000004149523740
:105380003830455F4556454E545F514D5452454364
:1053900056000000414952373830455F4556454E6A
:1053A000545F514D545055424558000041495237C1
:1053B0003830455F4556454E545F44454C41590091
:1053C000414952373830455F4556454E545F524447
:1053D00059000000524459004556454E545F454E11
:1053E0005452590041542B435354543D22257322A7
:1053F0002C22222C22220D0A0000000041542B43B3
:1054000049505258463D310D0A00000041542B438B
:1054100049504D55583D310D0A00000041542B4371
:105420004349440D0A00000041542B43494D490DA6
:105430000A0000004154490D0A00000041542B436A
:1054400047534E0D0A00000041542B434949435233
:105450000D0A000041542B43494653520D0A0000E7
:10546000414952373830450041495237383045526A
:10547000756E4154436D6400414952373830454997
:10548000646C650041495237383045506F7765721A
:105490004F66660041495237383045495043686588
:1054A000636B0000414952373830454950506F6CAA
:1054B0006C00000041495237383045506F776572B3
:1054C0004F6E000041495237383045436C6F736569
:1054D000576972656C65737300000000414952376B
:1054E0003830454F70656E576972656C657373002F
:1054F00041495237383045496E6974004149523745
:105500003830454950496E697400000041495237AE
:105510003830454154436D64496E697400000000A1
:10552000414952373830454154436D645465737472
:1055300000000000414952373830455265616479B6
:1055400000000000414952373830454950526561EA
:1055500064790000414952373830455761697453C6
:10556000696D4361726452656164790041495237E3
:10557000383045536561726368696E674E6574774C
:105580006F726B0041495237383045536F636B651A
:105590007453656E64446174610000004149523780
:1055A000383045536F636B6574436C6F73650000EF
:1055B00041495237383045536F636B6574436F6EA2
:1055C0006E6563740000000041495237383045432E
:1055D00053510000414952373830454C6F63000049
:1055E0006F7461006C6F675F75706C6F6164000051
:1055F0006465766963655F696400000061745F6378
:105600006D6400007463705F73656E640000000079
:105610006462675F6D6F6465000000007365745FAE
:105620007274636D6D6F6465000000007365745F74
:10563000757762656E61626C650000007365745F0A
:1056400067707375706461746574696D65000000DE
:10565000617564696F5F766F6C756D650000000041
:105660007463705F636C6F736500000075706461D4
:10567000746500007463705F637265617465000037
:105680006770735F626175645F72617465000000CA
:105690007365745F64617461726174650000000019
:1056A00064656275675F6F666600000034675F70EF
:1056B0006F7765726F6666006C6F67007365745F05
:1056C0007274636D000000007274635F7365745FD1
:1056D000616C61726D0000006C6F675F636C656187
:1056E0006E00000064656275675F6F6E0000000009
:1056F00034675F706F7765726F6E000073657276E6
:1057000065725F696E666F00696E666F000000000B
:10571000736C6565700000007365745F6E74726908
:10572000700000007365745F6770735F7300000042
:105730007365745F636861696368756770735F73CD
:1057400000000000636C6F73655F776972656C655C
:10575000737300006F70656E5F776972656C657357
:10576000730000007463705F636F6E6E6563740036
:105770007274635F676574007274635F736574004D
:105780006C6F675F7072696E740000007265626FA3
:105790006F74000074657374000000007474735FAC
:1057A000706C6179000000007365745F7178777ABE
:1057B00000000000636C6561720000006C73000003
:1057C000E057010800000020C4060000A86000089F
:1057D000DC580108C4060020BC480000842C0108E5
:1057E000012458152443434D53472C524D432C312B
:1057F0002C302C2A30340D0A145C475341149A443F
:10580000144A56148B3141145B4C4C147A46145C88
:105810005458543C84300D0A32019204025D2085B4
:105820006854010813F96C9B08C41013BD649B08ED
:10583000DC1013256B790C01148BC8552C0B1CF54F
:10584000632C01149AD440CBB969400217017A0144
:10585000194BC842040132036255AA000C5D24476B
:105860004E4747412C4C42532C140502141509098C
:105870000102024781E2010A15FF0CC14809FCA997
:10588000F1D24D624040085A30085A20085A100898
:105890001159080B2CF03F285AE00809262893D00C
:1058A0003F130704380D091E08054008260910405B
:1058B00008560A131D043B08BE050624D8BC401038
:1058C00008320217B4570108E1C01B08BC08133D99
:0C58D000C209233801FF01FF0152B201A0
:04000005080050C1DE
:00000001FF
